:020000040800F2
:20000000E8120020DD1B0008F91B0008FD1B0008011C0008051C0008091C0008000000000F
:200020000000000000000000000000000D1C0008111C000800000000151C0008191C0008E4
:200040001D1C0008211C0008251C0008291C00082D1C0008311C0008351C0008391C000828
:200060003D1C0008411C0008451C0008491C00084D1C0008511C0008551C0008591C000808
:200080005D1C0008611C0008651C0008691C00086D1C0008711C0008751C0008791C0008E8
:2000A0007D1C0008811C0008851C0008891C0008A11A0008BD1A000800000000951C000849
:2000C000991C000800000000000000009D1C000800000000370F00088D0F0008A91C0008E3
:2000E000AD1C0008B11C0008B51C000800B587B0012141F2040000F04FFCE020ADF800005C
:2001000003208DF8020018208DF8030000A9DFF88C0700F073FC1020ADF8000003208DF886
:20012000020010208DF8030000A9DFF8700700F065FC1021DFF8640700F0C6FC0020ADF8D3
:2001400004004FF48270ADF806000020ADF808000220ADF80A000120ADF80C004FF4007098
:20016000ADF80E000020ADF810000020ADF812000720ADF8140001A9DFF8240700F0EEFCBA
:200180000121DFF81C0700F009FD4FF6FF7007B000BD00B587B00121082000F0FDFB0121E5
:2001A0004FF4804000F008FC4FF42040ADF8000003208DF802001C208DF8030000A9DFF812
:2001C000E40600F01BFC4FF48040ADF8000003208DF8020004208DF8030000A9DFF8C406E6
:2001E00000F00CFC4FF48050ADF8000003208DF8020014208DF8030000A9DFF8A80600F0CB
:20020000FDFB4FF48051DFF89C0600F05DFC0020ADF804004FF48270ADF806000020ADF8A2
:2002200008000020ADF80A000120ADF80C004FF40070ADF80E003820ADF810000020ADF8DD
:2002400012000720ADF8140001A9DFF85C0600F085FC0121DFF8500600F0A0FC4FF6FF70C9
:2002600007B000BD00B587B00121012000F094FB0121DFF8380600F02DFC01210C2000F0CE
:200280008BFB01214FF4004000F096FB3820ADF8000003208DF8020018208DF8030000A9A2
:2002A000DFF8000600F0AAFB4FF40040ADF8000003208DF8020010208DF8030000A9DFF8C2
:2002C000DC0500F09BFB4FF40041DFF8D00500F0FBFB0020ADF804004FF48270ADF80600F8
:2002E0000020ADF808000220ADF80A000120ADF80C004FF40070ADF80E000020ADF8100053
:200300000020ADF812000720ADF8140001A9DFF8A00500F023FC0121DFF8940500F03EFC35
:200320004FF6FF7007B000BD80B51021DFF86C0500F0CDFB062000F05CFA1021DFF85C055A
:2003400000F0C2FB01BD80B54FF40041DFF84C0500F0BDFB062000F088FA4FF40041DFF8B6
:200360003C0500F0B1FB01BD80B51021DFF82C0500F0ADFB042000F03CFA1021DFF81C0569
:2003800000F0A2FB00F05AF801BD80B54FF40041DFF8080500F09BFB042000F066FA4FF4F6
:2003A0000041DFF8F80400F08FFB00F057F801BD80B51021DFF8E40400F089FB502000F0B9
:2003C00018FA1021DFF8D40400F07EFB1021DFF8CC0400F07CFB012000F00BFA002000F05D
:2003E00008FA1021DFF8B40400F06EFB00F026F801BD80B54FF40041DFF8A00400F067FB90
:20040000502000F032FA4FF40041DFF8900400F05BFB4FF40041DFF8840400F058FB0120D4
:2004200000F023FA002000F020FA4FF40041DFF86C0400F049FB00F011F801BD10B50120E9
:20044000002401E000F01AF8C0B2C00705D52000441C42F210718842F4D310BD10B5012009
:20046000002401E000F01EF8C0B2C00705D52000441C42F210718842F4D310BD10B51021D5
:20048000DFF8180400F023FB052000F0B2F900F0ABF904001021DFF8040400F015FB2000D3
:2004A000C0B210BD10B54FF40041DFF8F00300F00EFB052000F0D9F900F0D2F904004FF408
:2004C0000041DFF8D80300F0FFFA2000C0B210BDF8B504000D00160000271021DFF8BC031F
:2004E00000F0F5FA0B2000F084F9200CC0B200F080F9200AC0B200F07CF92000C0B200F0FB
:2005000078F9002000F075F904E000F06DF9BFB278557F1CBFB2B6B2B742F6D31021DFF836
:200520007C0300F0D1FA4FF6FF70F2BD70B504000D0000264FF48051DFF8680300F0C7FABB
:2005400014F07F0000F073F904E000F06BF9B6B27055761CB6B2032EF7D34FF48051DFF877
:20056000440300F0B1FA4FF6FF7070BDF8B504000D00160000274FF40041C84800F0A7FA98
:200580000B2000F072F9200CC0B200F06EF9200AC0B200F06AF92000C0B200F066F90020F0
:2005A00000F063F904E000F05BF9BFB278557F1CBFB2B6B2B742F6D34FF40041B74800F0E0
:2005C00083FA4FF6FF70F2BDF8B504000D0016000027200000F0C6F8FFF7EAFEFFF7A4FEFC
:2005E0001021AE4800F073FAAD2000F002F9200CC0B200F0FEF8200AC0B200F0FAF820009D
:20060000C0B200F0F6F8287800F0F3F8687800F0F0F81021A14800F057FA0220070015E0DE
:20062000401E0028FCD110219C4800F050FAAD2000F0DFF8785D00F0DCF87F1C785D00F08B
:20064000D8F87F1C1021954800F03EFAB6B2B74201D27820E5E7642000E0401E0028FCD1AA
:20066000FFF782FE10218D4800F031FAFFF7E6FE4FF6FF70F2BD38B504000D004FF4805194
:20068000884800F024FA54F08000C0B200F0CFF8287800F0CCF8687800F0C9F8A87800F09A
:2006A000C6F84FF480517F4800F00EFA4FF6FF7032BDF8B504000D0016000027FFF799FE7E
:2006C000FFF741FE4FF40041744800F000FAAD2000F0CBF8200CC0B200F0C7F8200AC0B252
:2006E00000F0C3F82000C0B200F0BFF8287800F0BCF8687800F0B9F84FF40041674800F02E
:20070000E3F90220070017E0401E0028FCD14FF40041624800F0DBF9AD2000F0A6F8785D68
:2007200000F0A3F87F1C785D00F09FF87F1C4FF400415A4800F0C8F9B6B2B74201D27820F9
:20074000E3E7642000E0401E0028FCD1FFF71DFE4FF40041514800F0BAF9FFF77FFE4FF68F
:20076000FF70F2BD10B50400FFF722FEFFF7DCFD10214A4800F0ABF9202000F03AF8200CC8
:20078000C0B200F036F8200AC0B200F032F82000C0B200F02EF81021404800F095F9FFF73E
:2007A0004DFE10BD10B50400FFF723FEFFF7CBFD4FF40041394800F08AF9202000F055F88E
:2007C000200CC0B200F051F8200AC0B200F04DF82000C0B200F049F84FF400412F4800F0C3
:2007E00073F9FFF73BFE10BD80B5002000F001F802BD10B504000221294800F0E1F9002845
:20080000F9D0E4B2210089B2254800F0D5F90121234800F0D5F90028F9D0214800F0CEF996
:20082000C0B210BD80B5002000F001F802BD10B5040002211C4800F0C3F90028F9D0E4B2F9
:20084000210089B2184800F0B7F90121164800F0B7F90028F9D0144800F0B0F9C0B210BDF7
:2008600080B5002000F001F802BD10B5040002210F4800F0A5F90028F9D0E4B2210089B2C7
:200880000B4800F099F90121094800F099F90028F9D0074800F092F9C0B210BD000801404B
:2008A00000300140000C01400038004000023000003C0040ED000008D1040008C9050008AC
:2008C000930100082D05000877060008650200086D050008B306000830B4002200210023C9
:2008E00000243D4D2D6815F00C052A00002A04D0042A05D0082A06D021E03849016020E089
:20090000374901601DE03449096811F47011324A126812F48033890C891C002B03D1314A22
:20092000514301600AE02C4A1268920303D52E4A5143016002E02A4A5143016001E0274972
:2009400001602549096811F0F00212092749545C0168E14041602049096811F4E062120AC1
:200960002249545C4168E14081601B49096811F46052D20A1D49545C4168E140C1601649E9
:20098000096811F44042920B1949545CC168B1FBF4F1016130BC7047C9B2002905D015491A
:2009A000096808431349086005E01249096831EA0000104908607047C9B2002905D00E49A3
:2009C000096808430C49086005E00B49096831EA00000949086070470410024000127A0086
:2009E000001BB70000093D00808D5B004800002060000020181002401C100240F0B40022F1
:200A00000026002400250023002791F803C01CF00F0C624691F803C05FEACC6C01D58B785C
:200A20001A430B781B0621D00368002406E0CD78482D02D10125A5400561641C082C14D2B7
:200A40000125A5400E882E40AE42F6D1A5000F2616FA05F7BB4312FA05F52B43CD78282DDE
:200A6000E5D10125A5404561E7E703600B884FF48074A34226D34368002420E0012514F13C
:200A80000806B5400E882E40AE4217D1A5000F2616FA05F7BB4312FA05F52B43CD78282D85
:200AA00004D1012514F10806B5404561CD78482D04D1012514F10806B5400561641C082CB6
:200AC000DCD34360F0BC704789B20161704789B24161704770B4002200240023002500289F
:200AE00002D51C4A136801E01B4A1368C0F3034582B210F44014B4F5401F08D133F070631F
:200B0000154C246834F07064134D2C600FE0C40205D50324AC40A34353F0706307E0440D2E
:200B2000E4B2240112FA04F4A34353F07063C9B2002905D0410DC9B2090112FA01F10B4362
:200B4000002802D50348036001E00348036070BC704700001C0001400400014010B40022EE
:200B600003881A0012F441520B884C8823438C882343CC8823430C8923434C8923438C89EB
:200B80002343CC8923431A430280828B4FF2FF731A408283098A018210BC7047C9B20029F9
:200BA00004D0018851F04001018004E001884FF6BF721140018070478181704780897047F0
:200BC00000220089084201D0012200E000221000C0B2704770477047704710B4019CDBB2DE
:200BE000012B03D14FF48063038108E0DBB2022B03D14FF4C063038101E000230381E4B2CD
:200C0000012C02D10023C38016E0E4B2022C03D14FF40053C3800FE0E4B2032C03D14FF43C
:200C20008053C38008E0E4B2042C03D14FF44053C38001E00023C380D2B2082A09D10289A1
:200C4000002A02D10022828013E04FF4805282800FE0D2B2092A03D14FF48052828008E0F0
:200C60000289002A02D10022828002E04FF480528280B1F5966F15D0B1F5166F16D0B1F588
:200C8000965F17D0B1F5165F18D0B1F5964F19D0B1F5164F1AD0B1F5614F1BD0B1F5E13F05
:200CA0001CD01FE04FF4966101601EE04FF4166101601AE04FF49651016016E04FF4165170
:200CC000016012E04FF4964101600EE04FF4164101600AE04FF46141016006E05FF4E131E2
:200CE000016002E04FF41651016010BC7047F0B589B004000D0016001F00012144F20400A3
:200D0000FFF74AFE4FF40070ADF8040003208DF8060018208DF8070001A9B248FFF76EFEC1
:200D20004FF48060ADF8040004208DF8070001A9AC48FFF763FEFFB200973300DBB22A0010
:200D4000D2B2210005A8FFF748FF0020ADF820000C20ADF81E0005A9A34800F053F900203B
:200D6000ADF80C000020ADF80E004FF40070ADF810000020ADF8120003A99B4800F0A4F994
:200D8000012240F22551984800F0BEF90121964800F0ACF925208DF8080000208DF80900EC
:200DA00000208DF80A0001208DF80B0002A800F000FA4FF6FF7009B0F0BDF0B589B0040043
:200DC0000D0016001F0001210420FFF7E5FD01215FF40030FFF7F0FD0420ADF80400182026
:200DE0008DF8070003208DF8060001A97D48FFF705FE0820ADF8040004208DF8070001A926
:200E00007848FFF7FBFDFFB200973300DBB22A00D2B2210005A8FFF7E0FE0020ADF82000E7
:200E20000C20ADF81E0005A9704800F0EBF80020ADF80C000020ADF80E004FF40070ADF88E
:200E400010000020ADF8120003A9684800F03CF9012240F22551654800F056F901216348A6
:200E600000F044F926208DF8080000208DF8090000208DF80A0001208DF80B0002A800F0CA
:200E800098F94FF6FF7009B0F0BD10B5040040F22661554800F077F9E4B2210089B252489C
:200EA00000F05BF9012240F226614F4800F02CF94F480078AA28FBD14D485521017000221B
:200EC00040F22661484800F01FF94FF6FF7010BD10B5040040F22661444800F054F9E4B25F
:200EE000210089B2414800F038F9012240F226613E4800F009F93F480078AA28FBD13D4876
:200F000055210170002240F22661384800F0FCF84FF6FF7010BD384A127802700120088003
:200F20004FF6FF707047354A12780270012008804FF6FF70704780B520212B4800F015F9D0
:200F4000C0B201280CD1284800F00BF92A49087040F22551244800F016F929480069804716
:200F60004021214800F001F9C0B201280DD1002240F226611C4800F0C7F840F226611A483B
:200F800000F001F91A48AA21017001BD80B52021164800F0EAF8C0B201280CD1134800F0A2
:200FA000E0F81649087040F22551104800F0EBF81348806A804740210C4800F0D6F8C0B2BE
:200FC00001280DD1002240F22661084800F09CF840F22661054800F0D6F80648AA2101700D
:200FE00001BD00000008014000380140004400406400002065000020E0100020E1100020C3
:2010000000000020F0B585B004000D0000200021002200230026AF89002F2600208A4CF6A0
:20102000FF710840E98808432082A0894EF6F3110840A9882A8911436A8911430843A081F6
:20104000A08A4FF6FF410840A9890843A08200A8FFF742FC1B48864201D1039900E002990A
:20106000A089000407D5192000FB01F029684900B0FBF1F206E0192000FB01F029688900B5
:20108000B0FBF1F26420B2FBF0F000010109642303FB1123A189090408D5D9003231642217
:2010A000B1FBF2F111F00701084307E0190132316422B1FBF2F111F00F010843208105B022
:2010C000F0BD00000038014010B40022038A1A004FF2FF031A400B884C8823438C88234379
:2010E000C98819430A43028210BC7047C9B2002904D0818951F40051818104E081894DF6A4
:20110000FF72114081817047F0B4002300240025002640F66A1789B2B94206000800C0B2B1
:201120004309DBB289B211F01F04012010FA04F5012B01D10C3604E0022B01D1103600E00A
:201140001436D2B2002A03D030682843306002E03068A8433060F0BC7047C905C90D818034
:2011600070478088C005C00D704700224FF4007389B299420088084201D0012200E00022B1
:201180001000C0B2704710B40022002340F66A1489B2A14289B20A0A012111FA02F39BB27D
:2011A000D943018010BC70471E4908431E490860704710B4002100220F23C478002C1ED048
:2011C0001949096811F4E061D1F5E061090AD1F10402CB404178914082781A4011430901CD
:2011E0000278124BD15401784911114A0123007810F01F0013FA00F042F821000AE001784F
:2012000049110C4A0123007810F01F0013FA00F042F8210010BC7047074A1140084307494B
:20122000086070470000FA050CED00E000E400E000E100E080E100E080FFFF1F08ED00E07F
:2012400080B501214020FFF7A7FB0220ADF8000010208DF8030002208DF8020000A97F48A7
:20126000FFF7CCFB02217D48FFF72EFC01BD000080B500F003F900F025F900F044F902206D
:2012800000F054F9FFF7DCFF1423754A0021022000F061F973480021016004E0714800687B
:2012A000401C704908606F480068042805D26D4800686B49405C5A28F0D06A48006804289A
:2012C00040F0B4806648007965494979090451EA00606349897950EA01206149C97908432B
:2012E0006149086060480068B0F5483F03D25E485FF4962101605A4800795949097A08185A
:2013000080B2FF2840F09280554840795449497A081880B2FF2840F089805148807950499F
:20132000897A081880B2FF2840F080804C48C0794B49C97A081880B2FF2877D100F028F98B
:201340004948006810F50051484800F006FA02214248FFF7BCFB43480021016023E04FF411
:201360008052FF213E4800F02EFA4FF480533C4A3C480068401C4FF4805101FB00F10220D6
:2013800000F0E9F84FF48052364800684FF48051364B01FB0031324800F0B8F931480068C3
:2013A000401C304908602F4800682F490968B0EB113FD4D32B4800684FF4805148432A49A9
:2013C000096888422BD24FF48052FF21244800F0FAF925480068234909684FF4805202FB8D
:2013E00011039BB21E4A1F480068401C4FF4805101FB00F1022000F0AEF81B480068194913
:2014000009684FF4805202FB1102164800684FF48051164B01FB0031114800F077F90020F5
:20142000FFF7C0F902210D48FFF74EFB4FF400515FF00060FFF7F0FE4FF4005080F3088889
:20144000DDF800D00A480B49096801600A4808490968016008480068804701BD0018014064
:2014600068000020D8100020D410002000200008D010002004200008CC10002080B500F063
:20148000C3F94FF4C060FFF78FFE01BD80B5214A2148008821494118012000F099FA1E488E
:2014A0000088642804D21C480088401C1A49088019480088642802D117480021018001BD08
:2014C0007047704780B514480021018011480021018001200090002308225FF4E1310120EC
:2014E00000F052FA002801D100200BE00C4B0D4A0D49012000F07EFA002801D1002001E023
:201500004FF6FF7002BD0348002101800248002101807047DE100020DC1000206810002016
:20152000C3140008C11400088D14000810B50024C0B203280CD2C0B20C21144A01FB0020C9
:20154000006880474FF6FF71884201D14FF6FF74200080B210BD70B50400080011001A00D8
:201560000025E4B2032C0DD292B2E4B20C23074E03FB04635B6898474FF6FF71884201D1EC
:201580004FF6FF75280080B270BD0000B4080008DFF83401DFF834110160DFF82C01DFF8E3
:2015A000301101607047DFF82C01006850F08000DFF820110860704738B5040004255FF412
:2015C000302000F08DF80500EDB2042D20D1DFF80401006850F00200DFF8F8100860DFF8DC
:2015E000F8000460DFF8EC00006850F04000DFF8E41008605FF4302000F072F80500DFF8D8
:20160000D400006841F6FD710840DFF8C81008602800C0B232BD70B582B005000C0004266F
:20162000002000904FF4005000F05AF80600F6B2042E2DD1DFF89C00006850F00100DFF854
:20164000941008602C804FF4005000F049F80600F6B2042E13D1A81C0090200C00990880A9
:201660004FF4005000F03CF80600DFF86800006841F6FE710840DFF85C10086008E0DFF8AE
:201680005400006841F6FE710840DFF8481008603000C0B276BD11490860704704200F493F
:2016A0000968C90701D501200CE00C480068400701D5022006E009480068C00601D50320AD
:2016C00000E00420C0B270470420024023016745AB89EFCD10200240142002400C20024061
:2016E00038B504000425FFF7D9FF050003E0FFF7D5FF0500641EEDB2012D01D1002CF6D137
:20170000002C00D105252800C0B232BDF8B505000C00170004208DF80000FFF739FFBE08A7
:201720000420B7FBF0F101FB1071002909D0761C07E029682000FFF76EFF8DF80000241D20
:201740002D1D3000461E80B2002803D09DF800000428EED0FFF727FFF1BD70B582B00400DA
:201760000D0004208DF800004FF48060B4FBF0F101FB1041002901D0002023E0FFF708FF99
:20178000AE0A4FF48060B5FBF0F101FB1051002900D0761C3520FFF77EFF002508E04FF4DD
:2017A000806000FB0540FFF707FF8DF800006D1CB54203D29DF800000428F0D0FFF7F3FECB
:2017C0004FF6FF7076BD10B5040010000A000100200000F031F9200010BD10B450F8041BEC
:2017E00081B102681218001D50F8043BDC0744BFA9F10104E31852F8044B43F8044B091FB4
:20180000F9D1EBE710BC704780B54F48006850F001004D4908604D4800684D4908404B49C7
:201820000860494800684B490840474908604648006830F48020444908604448006830F4AC
:20184000FE004249086044485FF41F01016000F005F842485FF00061016001BD80B500F0CC
:2018600001F801BD82B000200190002000903648006850F48030344908603348006810F478
:20188000003000900198401C01900098002803D10198B0F5A06FF0D12B480068800302D52B
:2018A0000120009001E0002000900098012847D12B48006850F01000294908602848006830
:2018C00080088000264908602548006850F00200234908601D481D49096801601B481B49DA
:2018E000096801601948006850F48060174908601648006830F47C10144908601348006863
:2019000050F48810114908600F48006850F080700D4908600C4800688001FBD50B480068B4
:2019200080088000094908600848006850F00200064908600548006810F00C000828F9D179
:2019400002B070470000000000100240041002400000FFF8FFFFF6FE0810024008ED00E05E
:20196000002002400749002201E01831521C0B78FF2B01D1002004E00B78C0B28342F4D1F9
:2019800008007047000000202DE9F0410E0017009846069CC0B2FFF7E5FF0500002D01D12C
:2019A000002013E02300DBB24246D2B23900C9B230006C682468A047002129724FF6FF71BC
:2019C00080B2884201D10121297280B2BDE8F08138B50C001500C0B2FFF7C4FF0200002ACF
:2019E00001D1002005E02900200052689268904780B232BD70B50C0015001E00C0B2FFF74F
:201A0000B1FF002801D1002004E004614661C5604FF6FF7070BD50F8041B61B150F8042B16
:201A2000D30744BFA9F101039A18002342F8043B091FFAD1EFE7704762F30F2262F31F4221
:201A4000401810F0030308D0C91A1FD3DB0748BF00F8012D28BF20F8022D130030B41446ED
:201A60001546103928BF20E93C00FAD8490728BF20E90C0048BF40F8042D890028BF20F880
:201A8000022D48BF00F8012D30BC7047C91818BF00F8012DCB0728BF00F8012D70470000D3
:201AA00080B501215FF0804000F016F8002804D001215FF0804000F026F801BD80B5012172
:201AC000044800F009F8002803D00121014800F01AF801BD0004004030B400220023002412
:201AE000058A0D402B008089084004009BB2002B04D0A4B2002C01D0012200E000221000B6
:201B0000C0B230BC704789B2C94301827047000080B500F015F802000023DB431068984268
:201B200004D011000220ABBE002010605068984204D0111D0220ABBE0020506001BD0000F8
:201B4000004870475800002010B5084979441C31074C7C441A34A14206D0081D0A685118D4
:201B600088470146A142F8D110BD00BF0800000028000000A3FEFFFF7C1000006800002034
:201B80000000000057FCFFFF680000002C010000000000200000000000F009F8002801D055
:201BA000FFF7D2FF0020FFF763FB00F002F80120704780B500F002B800BF000007463846BF
:201BC00000F002F8FBE7000080B5FFF7A1FF024A11001820ABBEFBE7260002000148804756
:201BE0000148004709180008ED1B0008C046C046C046C046FFF7D0FFFFF7FEBFFFF7FEBFD9
:201C0000FFF7FEBFFFF7FEBFFFF7FEBFFFF7FEBFFFF7FEBFFFF7FEBFFFF7FEBFFFF7FEBF2C
:201C2000FFF7FEBFFFF7FEBFFFF7FEBFFFF7FEBFFFF7FEBFFFF7FEBFFFF7FEBFFFF7FEBF0C
:201C4000FFF7FEBFFFF7FEBFFFF7FEBFFFF7FEBFFFF7FEBFFFF7FEBFFFF7FEBFFFF7FEBFEC
:201C6000FFF7FEBFFFF7FEBFFFF7FEBFFFF7FEBFFFF7FEBFFFF7FEBFFFF7FEBFFFF7FEBFCC
:201C8000FFF7FEBFFFF7FEBFFFF7FEBFFFF708BFFFF714BFFFF7FEBFFFF7FEBFFFF7FEBF8C
:201CA000FFF749B9FFF772B9FFF7FEBFFFF7FEBFFFF7FEBFFFF7FEBF0000000030000020EF
:201CC00000000000D70B0008D50B0008D90B0008010000003C00002000000000D70B0008FF
:201CE000D50B0008D90B0008EF0C00088B0E0008170F0008BB0D0008D10E0008270F000849
:201D000000000000010203040102030406070809FFFFFFFFFFFFFFFF02040608AAAA000031
:201D2000FFFFFFFFFFFFFFFFFFFFFFFFFFFFFFFFFFFFFFFFFFFFFFFFFFFFFFFFFFFFFFFFC3
:201D4000FFFFFFFFFFFFFFFFFFFFFFFFFFFFFFFFFFFFFFFFFFFFFFFFFFFFFFFFFFFFFFFFA3
:201D6000FFFFFFFFFFFFFFFFFFFFFFFFFFFFFFFFFFFFFFFFFFFFFFFFFFFFFFFFFFFFFFFF83
:201D8000FFFFFFFFFFFFFFFFFFFFFFFFFFFFFFFFFFFFFFFFFFFFFFFFFFFFFFFFFFFFFFFF63
:201DA000FFFFFFFFFFFFFFFFFFFFFFFFFFFFFFFFFFFFFFFFFFFFFFFFFFFFFFFFFFFFFFFF43
:201DC000FFFFFFFFFFFFFFFFFFFFFFFFFFFFFFFFFFFFFFFFFFFFFFFFFFFFFFFFFFFFFFFF23
:201DE000FFFFFFFFFFFFFFFFFFFFFFFFFFFFFFFFFFFFFFFFFFFFFFFFFFFFFFFFFFFFFFFF03
:201E0000FFFFFFFFFFFFFFFFFFFFFFFFFFFFFFFFFFFFFFFFFFFFFFFFFFFFFFFFFFFFFFFFE2
:201E2000FFFFFFFFFFFFFFFFFFFFFFFFFFFFFFFFFFFFFFFFFFFFFFFFFFFFFFFFFFFFFFFFC2
:201E4000FFFFFFFFFFFFFFFFFFFFFFFFFFFFFFFFFFFFFFFFFFFFFFFFFFFFFFFFFFFFFFFFA2
:201E6000FFFFFFFFFFFFFFFFFFFFFFFFFFFFFFFFFFFFFFFFFFFFFFFFFFFFFFFFFFFFFFFF82
:201E8000FFFFFFFFFFFFFFFFFFFFFFFFFFFFFFFFFFFFFFFFFFFFFFFFFFFFFFFFFFFFFFFF62
:201EA000FFFFFFFFFFFFFFFFFFFFFFFFFFFFFFFFFFFFFFFFFFFFFFFFFFFFFFFFFFFFFFFF42
:201EC000FFFFFFFFFFFFFFFFFFFFFFFFFFFFFFFFFFFFFFFFFFFFFFFFFFFFFFFFFFFFFFFF22
:201EE000FFFFFFFFFFFFFFFFFFFFFFFFFFFFFFFFFFFFFFFFFFFFFFFFFFFFFFFFFFFFFFFF02
:201F0000FFFFFFFFFFFFFFFFFFFFFFFFFFFFFFFFFFFFFFFFFFFFFFFFFFFFFFFFFFFFFFFFE1
:201F2000FFFFFFFFFFFFFFFFFFFFFFFFFFFFFFFFFFFFFFFFFFFFFFFFFFFFFFFFFFFFFFFFC1
:201F4000FFFFFFFFFFFFFFFFFFFFFFFFFFFFFFFFFFFFFFFFFFFFFFFFFFFFFFFFFFFFFFFFA1
:201F6000FFFFFFFFFFFFFFFFFFFFFFFFFFFFFFFFFFFFFFFFFFFFFFFFFFFFFFFFFFFFFFFF81
:201F8000FFFFFFFFFFFFFFFFFFFFFFFFFFFFFFFFFFFFFFFFFFFFFFFFFFFFFFFFFFFFFFFF61
:201FA000FFFFFFFFFFFFFFFFFFFFFFFFFFFFFFFFFFFFFFFFFFFFFFFFFFFFFFFFFFFFFFFF41
:201FC000FFFFFFFFFFFFFFFFFFFFFFFFFFFFFFFFFFFFFFFFFFFFFFFFFFFFFFFFFFFFFFFF21
:201FE000FFFFFFFFFFFFFFFFFFFFFFFFFFFFFFFFFFFFFFFFFFFFFFFFFFFFFFFFFFFFFFFF01
:2020000048A10020A51E040807CD000809CD00080FCD00080BCD00080DCD000811CD0008A2
:2020200011CD000811CD000811CD000811CD000811CD000811CD00086B3601080B3101084D
:202040006B4B0108754B01087F4B0108894B0108934B01089D4B0108A74B0108B14B010870
:20206000BB4B0108C54B0108CF4B0108D94B0108E34B0108ED4B0108F74B0108014C0108CF
:202080000B4C0108154C01081F4C0108294C0108334C01083D4C0108474C0108514C010828
:2020A0005B4C0108654C01086F4C0108794C0108834C01088D4C0108974C0108A14C010888
:2020C000AB4C0108B54C0108BF4C0108C94C0108D34C0108DD4C0108E74C0108F14C0108E8
:2020E000FB4C0108054D01080F4D010813CD000813CD000813CD000813CD000813CD000848
:2021000013CD000813CD0008194D0108234D01082D4D0108374D0108414D01084B4D0108BF
:20212000554D01085F4D0108694D0108734D01087D4D0108874D0108914D01089B4D01082F
:20214000A54D0108AF4D0108B94D0108C34D01080000000000000000000000000000000057
:2021600000000000000000000000000000000000000000000000000000000000000000005F
:2021800000000000000000000000000000000000000000000000000000000000000000003F
:2021A00000000000000000000000000000000000000000000000000000000000000000001F
:2021C0000000000000000000000000000000000000000000000000000000000000000000FF
:2021E0000000000000000000000000000000000000000000000000000000000000000000DF
:2022000058444A32322D424759542D442D56312E3030330000B585B04FF4FA6006F03AF87C
:2022200006F04CFB66E00422DFF8301A2B2007F046F90222DFF8281A1F2007F040F9012284
:20224000DFF8B8161B2007F03AF9DFF8B416002007F085FB0422DFF8041A2B2007F02FF9B7
:202260000322DFF8A016222007F029F90222DFF89816212007F023F90222DFF89016232070
:2022800007F01DF90022DFF88816382007F017F90022DFF88016392007F011F90022DFF859
:2022A00078163A2007F00BF90022DFF870163B2007F005F9DFF868060088052190FBF1F20B
:2022C00001FB1200002801D100F005FA00200090042200A92B2007F0F2F80098C00407D524
:2022E000DFF8780D00210180DFF8740D0021018000F058FB642005F0CDFFDFF824060088D5
:20230000401CDFF81C16088006F01EF9002803D006F01AF9012886D101A807F0A0FBDFF82D
:202320000406008800287FF47EAF9DF8080002287FF479AF9DF8090002287FF474AF9DF8EE
:202340000A0000287FF46FAF9DF80B00002808D09DF80B00012804D09DF80B0002287FF440
:2023600062AFFEE730B400230022002810D000230AE092B2DBB21C5CA4184FF4807594FB5D
:20238000F5F202FB15425B1CDBB2C9B28B42F0D3100080B230BC704710B4002300220028DD
:2023A0000AD00278012303E09BB21C5C62405B1C9BB289B28B42F7D3D2B2100080B210BC33
:2023C000704770B40023002200280FD0022309E0DBB21C5C4FF4807594FBF5F606FB1546B5
:2023E000B2185B1CDBB2C9B28B42F1D31000C0B270BC70470FB410B40021002000221100A3
:2024000018E0C9B201AA8A1852780A2392FBF3F403FB14223032C0B2DFF80C35C254401CFF
:20242000C9B2032905D2C0B2DFF8FC242E238354401C491CC9B2042957D2C9B201AA8A1833
:202440005278642A2ED3C9B201AA8A185278642392FBF3F23032C0B2DFF8CC34C254401C7B
:20246000C9B201AA8A1852780A2392FBF3F20A2392FBF3F403FB14223032C0B2DFF8A834CF
:20248000C254401CC9B201AA8A1852780A2392FBF3F403FB14223032C0B2DFF88C34C254E2
:2024A000401CBDE7C9B201AA8A1852780A2AA8D3C9B201AA8A1852780A2392FBF3F2303248
:2024C000C0B2DFF86434C254401CC9B201AA8A1852780A2392FBF3F403FB14223032C0B26E
:2024E000DFF84434C254401C9AE7C0B2DFF8381422224254401CC0B2DFF82C142C22425462
:20250000401CC0B2DFF8201420224254401CBDF80A1042F2107291424AD3BDF80A1042F236
:20252000107291FBF2F13031C0B2DFF8FC238154401CBDF80A104FF47A7291FBF2F10A2217
:2025400091FBF2F302FB13113031C0B2DFF8D8238154401CBDF80A10642291FBF2F10A2223
:2025600091FBF2F302FB13113031C0B2DFF8B8238154401CBDF80A100A2291FBF2F10A227D
:2025800091FBF2F302FB13113031C0B2DFF898238154401CBDF80A100A2291FBF2F302FBAA
:2025A00013113031C0B2DFF880238154401C8EE0BDF80A104FF47A72914237D3BDF80A1061
:2025C0004FF47A7291FBF2F13031C0B2DFF858238154401CBDF80A10642291FBF2F10A2217
:2025E00091FBF2F302FB13113031C0B2DFF838238154401CBDF80A100A2291FBF2F10A227D
:2026000091FBF2F302FB13113031C0B2C64A8154401CBDF80A100A2291FBF2F302FB131187
:202620003031C0B2C04A8154401C50E0BDF80A10642925D3BDF80A10642291FBF2F13031E3
:20264000C0B2B94A8154401CBDF80A100A2291FBF2F10A2291FBF2F302FB13113031C0B2D9
:20266000B14A8154401CBDF80A100A2291FBF2F302FB13113031C0B2AB4A8154401C26E0A2
:20268000BDF80A100A2916D3BDF80A100A2291FBF2F13031C0B2A44A8154401CBDF80A1024
:2026A0000A2291FBF2F302FB13113031C0B29E4A8154401C0BE0BDF80A100A2291FBF2F319
:2026C00002FB13113031C0B2974A8154401CC0B210BC04B0704780B594480078102805D2B3
:2026E00092480078401C9149087002E08F48002101708F4800788F490978884209D08C4870
:202700008C49097801708948002101708A480021018005F019FF212800F0C080DFF83C057D
:20272000006843F2F301084203D184480078AA282ED106F0E4F8DFF824050078C00703D5EC
:202740007C480121017014E0DFF810050078800603D57848022101700BE0DFF800050078D9
:20276000400603D573480321017002E071480721017072480078AA2802D16E480521017093
:202780006F480078AA280ED16A48062101700AE006F0BAF8654800210170664800210170FE
:2027A00065480021018067480078012803D1022007F02DFE1BE063480078022814D162488B
:2027C00000884FF6FF71884206D1022007F01FFE5D48002101800AE0022007F030FE5A48CB
:2027E0004FF6FF71018002E0022007F028FE57480078012803D056480078AA2803D1012092
:2028000007F005FE1BE051480078022814D1514800884FF6FF71884206D1012007F0F7FD20
:202820004C48002101800AE0012007F008FE49484FF6FF71018002E0012007F000FE46480D
:202840000078012803D1002007F0E1FD26E04248007802281FD13548007836490978B0EB5C
:20286000410F14DA344800884FF6FF71884206D1002007F0CCFD3048002101800EE00020B8
:2028800007F0DDFD2C484FF6FF71018006E0002007F0BDFD02E0002007F0D1FD01BD2F480A
:2028A000002101802E484FF6FF7101802D48002101802D48002101802C48002101802C4812
:2028C000002101802B48002101802B48002101802A48002101802A48002101802948002172
:2028E000018029480021018028480021016028480021018027480021017070478C7F00205D
:2029000044750020507F00202280002023800020607E0020647E0020687E00206C7E00205A
:202920008A7F0020687F002064760020368000203580002034800020927F00206E09002026
:20294000700900201D8000208E7F00201E8000206F090020907F00201F800020B27F00205F
:202960004E090020A27F0020A47F0020A67F0020A87F0020AA7F0020B07F0020AC7F0020ED
:202980006E7F0020707F0020B47F0020A47E00206A7F00203A80002080B507F08BFD07F0F8
:2029A000B7FD01BD2DE9F04FADF2B44D5FF0000A00245FF00009002253A9002006F07FFD2B
:2029C000002252A9152006F07AFD002251A9162006F075FD002250A9052006F070FD0322B6
:2029E000DFF8101E5D2006F06AFDA7A9002006F0B6FF5398DFF8001E07F0B6FD07F020FE3E
:202A000080465298DFF8F01D07F0AEFD07F018FE06005198DFF8E41D07F0A6FD07F010FE0D
:202A200007005098DFF8D41D07F09EFD07F008FE05008B480078012802D15FF001080FE0BD
:202A400087480078022802D15FF0020808E084480078002802D15FF0000801E05FF0030820
:202A6000DFF89C0D0078012803D10120ADF8040002E00020ADF80400DFF8880D00210170EE
:202A80009DF89D02002802D15FF0020935E09DF89D02062828D1DFF8700D0078022802D174
:202AA0005FF0100929E0DFF8600D0078032802D15FF0110921E0DFF8500D0078042802D1D6
:202AC0005FF0120919E05FF001096448006843F2F301084211D1DFF82C0D007850F0800089
:202AE000DFF8201D087008E09DF89D02052802D15FF0040901E05FF00309584800788007F7
:202B000007D5DFF8000D007850F00100DFF8F41C087052480078400707D5DFF8E80C007865
:202B200050F00200DFF8DC1C08704C480078C00707D5DFF8D00C007850F00400DFF8C41C37
:202B4000087046480078400607D5DFF8B80C007850F00800DFF8AC1C0870404800788006DD
:202B600007D5DFF8A00C007850F01000DFF8941C08703A480078000607D5DFF8880C007870
:202B800050F02000DFF87C1C087034480068C00407D5DFF8700C007850F08000DFF8641C88
:202BA0000870DFF8E80D008840F22621884208D3DFF8D80D008840F22621401ADFF8CC1D54
:202BC0000880DFF8CC0D0088DFF8C01D098880B2884204D3DFF8B41D0988441A05E000F2AF
:202BE0002620DFF8A81D0988441AA4B2062CC2F01184DFF8980DB0F800A01FFA8AFADFF8FD
:202C0000940D1AF80000682842F062801AF1010A40F226201FFA8AFA824503D340F226201D
:202C2000BAEB000A1FFA8AFADFF8680D1AF800B0BBF1040080B2FA2881F0FA87A4B21FFAD5
:202C40008BFB1BF102008442C1F2EA874FF48C72002156A807F006FD002422E0987E002040
:202C6000328000201AF1010A40F226201FFA8AFA824503D340F22620BAEB000AA4B256A83F
:202C80001FFA8AFADFF80C1D1AF801102154A4B2042C05D2A4B200A8A4B256A9615C21541D
:202CA000641CA4B21FFA8BFB5C45DBD30021002007F0F0FC1AF1010A40F226201FFA8AFA01
:202CC000824503D340F22620BAEB000ADFF8BC0CA0F800A09DF8000007282DD19DF8010001
:202CE000002829D19DF80200002825D19DF80300002821D14FF48072002104A807F0B2FCA4
:202D000068208DF8100004208DF811000B208DF8120000208DF8130000208DF81400002089
:202D20008DF81500CD484FF6FF7101809DF81100811C04A807F0DFFB9DF80000132853D1FA
:202D40009DF8010000284FD19DF8020000284BD19DF80300002847D14FF48072002104A8E0
:202D600007F080FC68208DF8100004208DF8110023208DF8120000208DF8130000208DF8D2
:202D8000140000208DF81500B44800210180B448002101809DF81100811C04A807F0ABFB9D
:202DA0004FF48072002104A807F05CFC68208DF8100001208DF8110002208DF8120008220B
:202DC000DFF8481E0DF1130007F02EFD00208DF81B0000208DF81C000D2104A807F08BFBAB
:202DE0000121002007F056FC9DF8000083280FD19DF8010000280BD19DF80200002807D1F7
:202E00009DF80300002803D10021002007F042FC9DF8000043280FD19DF8010000280BD12E
:202E20009DF80200002807D19DF80300002803D10021002007F02EFC9DF85C01642840F057
:202E40001F81864800884FF6FF71884240F018814FF48072002104A807F004FC9DF80100A5
:202E6000DFF86C1E0880DFF8680E00880002DFF8601E0880DFF8580E00889DF80010084300
:202E8000DFF84C1E0880DFF8480E008880B24008DFF83C1E088068208DF810000E208DF8B1
:202EA0001100DFF8300E008840008DF81200DFF8240E008880B2C0098DF81300DFF8100E74
:202EC000008840008DF81400DFF8040E008880B2C0098DF81500DFF8FC0D0088401CDFF8F0
:202EE000F41D088064208DF8160001208DF8170007208DF8180000208DF8190000208DF836
:202F00001A0000208DF81B0000208DF81C0000208DF81D0000208DF81E0014208DF81F00B9
:202F20009DF81100811C04A807F0E5FA142005F0B1F9DFF8A40D80F80090DFF8A00D80F86D
:202F4000008068208DF8100020208DF81100DFF8840D008840008DF81200DFF8780D008853
:202F600080B2C0098DF81300DFF8640D008840008DF81400DFF8580D008880B2C0098DF8D1
:202F80001500DFF8500D0088401CDFF8481D088086208DF8160000208DF8170003208DF89B
:202FA000180000208DF8190000208DF81A0000208DF81B0001208DF81C0030008DF81D0028
:202FC000B6B2300A8DF81E0038008DF81F00BFB2380A8DF82000BDF804008DF821008DF894
:202FE000228028008DF82300280A8DF82400280C8DF82500280E8DF826000822DFF80C1C9C
:203000000DF1270007F010FC5FFA88F8B8F1020F02D0BFB2012F03D301208DF82F0002E0F5
:2030200000208DF82F009DF89D02002808D102208DF83000DFF8CC0700788DF8310019E0DF
:203040009DF89D0206280DD101208DF83000DFF8B40700788DF831000CE000BF867F0020CA
:20306000887F002003208DF83000DFF8980700788DF831009DF81100811C04A807F03BFA92
:203080009DF85C01852841F01F859DF80100DFF8401C0880DFF8380C00880002DFF8301CA3
:2030A0000880DFF82C0C00889DF800100843DFF8201C0880DFF8180C008880B24008DFF892
:2030C000101C08809DF86201012831D0022800F0A382032800F0A282042800F028840F289D
:2030E00000F04184152800F05784162800F0D8841A2800F061871B2801F0A0801C2801F0E6
:203100008F811D2801F091821E2801F095821F2801F03083212800F0E585222800F0798641
:20312000232801F09383352801F09F8401F0CCBC5FF0010A46A80021002206C008389DF82D
:203140007401182802D316208DF87401002414E0DFF85C0E0088401EDFF8541E0880022281
:20316000DFF84C1E4FF4137007F0CFFE0322DFF8401E282006F0C8F9641C9DF87401A4B24B
:2031800080B2844280F0D0810821A4B2092056AA00FB04201D3007F02FFC0222DFF8101E17
:2031A0004FF4137007F09CFEDFF8040E00884FF49671884280F0DB80A4B2092056A900FBEF
:2031C000041090F8250001285ED15FF0010A01E01AF1010ADFF8D80D00881FFA8AFA50450F
:2031E0001CD31FFA8AFA4AF2EA3010EBCA00DFF8C41D0860082246A9DFF8B80D006807F0F4
:203200006FFE0822A4B2092056A900FB041010F11D0146A807F08EFE0028D9D1DFF8900DB4
:2032200000881FFA8AFA5045A6D2DFF8840D00884AF2F23111EBC000DFF8781D0860082253
:20324000A4B2092056A900FB041010F11D01DFF8640D006807F059FE0A2005F01BF8DFF8BB
:20326000500D0088401CDFF8481D08800222DFF8401D4FF4137007F048FE0322DFF8301DA5
:20328000282006F041F977E7A4B2092056A900FB041090F8250002287FF46EAF5FF0010A0A
:2032A00001E01AF1010ADFF8080D00881FFA8AFA5045FFF461AF1FFA8AFA4AF2EA3010EB80
:2032C000CA00DFF8F01C0860082246A9DFF8E40C006807F005FE0822A4B2092056A900FBF4
:2032E000041010F11D0146A807F024FE0028D8D1DFF8BC0C00881FFA8AFA504522D31FFA5C
:203300008AFA4AF2F23010EBCA00DFF8A81C0860082246A9DFF89C0C006807F0E1FD1FFA15
:203320008AFA4AF2EA3010EBCA00DFF8881C0860082246A9DFF87C0C006807F0E6FD1AF146
:20334000010AD5E7DFF8680C0088401EDFF8601C08800222DFF8581C4FF4137007F0D5FD9C
:203360000322DFF84C1C282006F0CEF804E7A4B2092056A900FB041090F82500012874D152
:203380005FF0010A01E01AF1010ADFF8240C00881FFA8AFA50451CD31FFA8AFA4AF2EA3039
:2033A00010EBCA00DFF80C1C0860082246A9DFF8040C006807F094FD0822A4B2092056A949
:2033C00000FB041010F11D0146A807F0B3FD0028D9D1DFF8DC0B00881FFA8AFA5045BFF42D
:2033E000CBAE5FF0010A21E01FFA8AFA4AF2F23010EBCA00DFF8BC1B0860082246A9DFF833
:20340000B40B006807F06CFD1FFA8AFA4AF2EA3010EBCA00DFF89C1B0860082246A9DFF887
:20342000940B006807F071FD1AF1010ADFF8800B0088401E1FFA8AFA5045D5DA1FFA8AFA44
:203440004AF2EA3010EBCA00DFF8681B08600822A4B2092056A900FB041010F11D01DFF8E2
:20346000540B006807F051FD86E6A4B2092056A900FB041090F8250002287FF47DAE5FF083
:20348000010A01E01AF1010ADFF8240B00881FFA8AFA5045FFF470AE1FFA8AFA4AF2EA3066
:2034A00010EBCA00DFF80C1B0860082246A9DFF8040B006807F014FD0822A4B2092056A9CA
:2034C00000FB041010F11D0146A807F033FD0028D8D1DFF8DC0A00881FFA8AFA5045FFF46E
:2034E00037AE1FFA8AFA4AF2F23010EBCA00DFF8C41A0860082246A9DFF8B80A006807F0F9
:20350000EFFC1FFA8AFA4AF2EA3010EBCA00DFF8A41A0860082246A9DFF8980A006807F01A
:20352000F4FC1AF1010AD4E7DFF8880A4AF2E031016009215AA8C01C07F05EFA09225AA92E
:20354000C91CDFF8700A006807F0DFFC4FF48072002104A807F086F868208DF810001D202A
:203560008DF81100DFF86C07008840008DF81200DFF86007008880B2C0098DF81300DFF8DC
:203580005007008840008DF81400DFF84407008880B2C0098DF81500DFF838070088401C3A
:2035A000DFF83017088082208DF8160000208DF8170003208DF8180000208DF819000020CE
:2035C0008DF81A0000208DF81B000C208DF81C000D240822DFF83416A4B204A8201807F012
:2035E00023F9083409215AA8C01C07F005FA09225AA9C91CA4B204A8201807F0CCFC09342C
:20360000A4B204A8002121549DF81100811C04A806F071FF01F058BA01F056BADFF87C0E58
:2036200000210180042266A9C91CDFF8740E07F0B2FC9DF89F01112840F080804FF48072FD
:20364000002104A807F00EF804F07EFF002825D100208DF8250008225AA9C91CDFF8780ED8
:2036600007F099FC20225CA9C91CDFF8700E07F092FC10220DF5D171DFF8640E07F08BFC7B
:20368000DFF8600E11210170DFF85C0E2A210170DFF8541E012004F06CFD02E001208DF8F6
:2036A000250068208DF8100014208DF81100DFF82406008840008DF81200DFF81806008821
:2036C00080B2C0098DF81300DFF80406008840008DF81400DFF8F805008880B2C0098DF839
:2036E0001500DFF8F0050088401CDFF8E815088082208DF8160000208DF8170003208DF808
:20370000180000208DF8190000208DF81A0000208DF81B000D208DF81C000D240822DFF854
:20372000EC14A4B204A8201807F07EF808349DF81100811C04A806F0DEFEF6E09DF89F01DA
:20374000102863D14FF48072002104A806F08AFF68208DF8100014208DF81100DFF8740545
:20376000008840008DF81200DFF86805008880B2C0098DF81300DFF85805008840008DF80A
:203780001400DFF84C05008880B2C0098DF81500DFF840050088401CDFF838150880822082
:2037A0008DF8160000208DF8170003208DF8180000208DF8190000208DF81A0000208DF8D0
:2037C0001B000D208DF81C000D240822DFF83C14A4B204A8201807F027F80834A4B204A8F0
:2037E000012121549DF81100811C04A806F083FE9BE000BF5E7F0020000020410000C8422A
:20380000EF7F00203B800020288000209DF89F01212827D104F098FE032840F086800822EC
:203820005AA9C91CDFF8B00C07F0B5FB20225CA9C91CDFF8A80C07F0AEFB10220DF5D17199
:20384000DFF89C0C07F0A7FBDFF8980C21210170DFF8940C2B210170DFF88C1C012004F05A
:2038600088FC62E09DF89F0120285ED104F06CFE03285AD1022268A9DFF8B80D07F08BFBD4
:20388000DFF8640C202101709DF8A001012804D1DFF8540C2021017042E09DF8A001022890
:2038A00004D1DFF8440C2121017039E09DF8A001032804D1DFF8300C2221017030E09DF89E
:2038C000A001042804D1DFF8200C2321017027E09DF8A001052804D1DFF80C0C24210170AA
:2038E0001EE09DF8A001062804D1DFF8FC0B2521017015E09DF8A001072804D1DFF8E80B03
:20390000262101700CE09DF8A001082804D1DFF8D80B2721017003E0DFF8CC0B272101700B
:20392000DFF8C41B012004F024FC01F0CDB8DFF8340E00210180DFF8300E4FF6FF71018020
:203940009DF87B01012807D09DF87B01002803D09DF87B01022804D1DFF8101E012004F020
:2039600008FC01F0B1B89DF86B01012807D09DF86B01002803D09DF86B01022803D1DFF816
:20398000F00D0021016001F09FB800BF9C7F0020FC7E0020DC500020002408215AA8C01C55
:2039A00006F07EFF4FF6FF71884223D108225AA9C91C964806F056FF0C2294495E2005F068
:2039C000A3FD3B21CCA807F0EDFA10228F49CCA807F0B0FA00280DD03B218C4807F001FB52
:2039E000DFF8940E00210180DFF8900E002101804FF6FF744FF48072002104A806F032FEB5
:203A000068208DF810001B208DF81100B148008840008DF81200AF48008880B2C0098DF861
:203A20001300AB48008840008DF81400A848008880B2C0098DF81500A6480088401CA54952
:203A4000088082208DF8160000208DF8170003208DF8180000208DF8190000208DF81A00A8
:203A600000208DF81B0015208DF81C00082267490DF11D0006F0D8FE082264490DF12500F5
:203A800006F0D2FE9DF81100811C04A806F033FD4FF6FF70A4B2844200D1FEE701F014B808
:203AA00000245FF0000A4FF48072022104A806F0D9FD9DF89D02002804D09DF89D02062827
:203AC00040F0AD809DF86B01012830D106225BA954A807F060FA00208DF8560154A806F0F7
:203AE000F7FE4FF6FF7188421ED108214CA807F059FA54A808F09EFBDFF86C1E0860042280
:203B0000DFF8641E292005F0FFFC4C98DFF8581E0968884204D00821DFF84C0E07F061FA27
:203B200000208DF8250002E001208DF825009DF87201012821D13C23FFAA78325FF4C8110D
:203B4000022008F090FB3C225CA9C91CFFA8783007F0F0F900280DD05FF4C81008F016FF0C
:203B60003C235CAAD21C5FF4C811022008F095FB4FF6FF7400208DF826009DF8AF0101282B
:203B80004AD1A4B2002C43D14521C6A807F00AFA4521DFF8D80D07F005FADFF8D00D9DF844
:203BA000B0114170DFF8C40D9DF8B1118170DFF8BC0D9DF8B211C170DFF8B00D9DF8B3118D
:203BC00001719DF8B4019DF8B51110EB0120DFF89C1DC8801622C6A9DFF8900D07F0AAF925
:203BE00000280ED04521DFF8840D07F0FAF9DFF8880C00210180DFF8840C002101804FF6AC
:203C0000FF7A00208DF8270009E000BF347C002001208DF8270002E002208DF827006820E2
:203C20008DF8100016208DF811002A48008840008DF812002748008880B2C0098DF81300C8
:203C40002348008840008DF814002148008880B2C0098DF815001F480088401C1D490880D9
:203C600082208DF8160000208DF8170003208DF8180000208DF8190000208DF81A000020EE
:203C80008DF81B0016208DF81C000822DFF8241E0DF11D0006F0C8FD9DF81100811C04A8A5
:203CA00006F029FC4FF6FF701FFA8AFA824509D1DFF8040E4FF6FF710180DFF8000E4FF6AE
:203CC000FF7101804FF6FF70A4B2844208D1FEE79E7F0020A07F002037800020388000203A
:203CE00000F0F2BE0422DFF8801C292005F0E7FB4FF48072002104A806F0B4FC68208DF8B6
:203D000010005B208DF81100DFF8B40D008840008DF81200DFF8A80D008880B2C0098DF8F7
:203D20001300DFF8A00D008840008DF81400DFF8940D008880B2C0098DF81500DFF8800D92
:203D40000088401CDFF8781D088082208DF8160000208DF8170003208DF8180000208DF82D
:203D6000190000208DF81A0000208DF81B0021208DF81C000822DFF83C1D0DF11D0006F05E
:203D800053FD1524DFF8E00B0268DFF8901EA4B204A8201808F094FEA41D3C230DF12B02DA
:203DA0005FF4C811022008F05EFA572004004521A1A807F0F7F8A4B204A89DF885122154B2
:203DC000641CA4B204A89DF886122154641CA4B204A89DF887122154641CA4B204A89DF883
:203DE00088122154641CA4B204A8BDF88A122154641CA4B204A8BDF88A1289B2090A2154D6
:203E0000641C9DF81100811C04A806F074FB00F05BBE4FF48072002104A806F023FC682026
:203E20008DF8100023208DF81100DFF8940C008840008DF81200DFF8880C008880B2C00950
:203E40008DF81300DFF87C0C008840008DF81400DFF8700C008880B2C0098DF81500DFF8C3
:203E6000600C0088401CDFF8581C088082208DF8160000208DF8170003208DF81800002046
:203E80008DF8190000208DF81A0000208DF81B0022208DF81C000822DFF8181C0DF11D00D2
:203EA00006F0C2FC1524002245A9382005F007FB4598DFF8F81D06F057FB06F0C1FBA4B29D
:203EC00004A96054641CA4B204A9020A6254641CA4B204A9020C6254641CA4B204A9000E64
:203EE0006054641C002245A9392005F0E8FA4598DFF8B81D06F038FB06F0A2FBA4B204A906
:203F00006054641CA4B204A9020A6254641CA4B204A9020C6254641CA4B204A9000E60541C
:203F2000641C002245A93A2005F0C9FA4598DFF87C1D06F019FB06F083FBA4B204A960545D
:203F4000641CA4B204A9020A6254641CA4B204A9020C6254641CA4B204A9000E6054641C10
:203F6000002245A93B2005F0AAFA4598DFF83C1D06F0FAFA06F064FBA4B204A96054641CBA
:203F8000A4B204A9020A6254641CA4B204A9020C6254641CA4B204A9000E6054641C9DF8BB
:203FA0001100811C04A806F0A6FA00F08DBD00BF627F0020A07E00205FF0000A1624002026
:203FC000A4B256A9615C0800641E0002A4B256A9615C0818641E0002A4B256A9615C08185B
:203FE000641E0002A4B256A9615C0818641E08F08BFDDFF8B81C08F095FD02900298DFF8D1
:20400000741E08F00DFE12D2002202A9382005F07BFA092144A806F0C5FF4498029908F059
:2040200011FE06D0092102A806F0DBFF01E05FF0010A1A240020A4B256A9615C0800641EC2
:204040000002A4B256A9615C0818641E0002A4B256A9615C0818641E0002A4B256A9615CE0
:204060000818641E08F050FDDFF8401C08F05AFD02900298DFF8FC1D08F0D2FD12D20022EE
:2040800002A9392005F040FA0A2144A806F08AFF4498029908F0D6FD06D00A2102A806F074
:2040A000A0FF01E05FF0010A1E240020A4B256A9615C0800641E0002A4B256A9615C0818F4
:2040C000641E0002A4B256A9615C0818641E0002A4B256A9615C0818641E08F015FDDFF811
:2040E000CC1B08F01FFD02900298DFF8881D08F097FD12D2002202A93A2005F005FA0B2166
:2041000044A806F04FFF4498029908F09BFD06D00B2102A806F065FF01E05FF0010A2224E1
:204120000020A4B256A9615C0800641E0002A4B256A9615C0818641E0002A4B256A9615CF9
:204140000818641E0002A4B256A9615C0818641E08F0DAFCDFF8541B08F0E4FC02900298EF
:20416000DFF8101D08F05CFD12D2002202A93B2005F0CAF90C2144A806F014FF449802998D
:2041800008F060FD06D00C2102A806F02AFF01E05FF0010A4FF48072002104A806F062FA6F
:2041A00068208DF8100014208DF81100DFF81009008840008DF81200DFF80409008880B22B
:2041C000C0098DF81300DFF8FC08008840008DF81400DFF8F008008880B2C0098DF8150056
:2041E000DFF8DC080088401CDFF8D418088082208DF8160000208DF8170003208DF818001C
:2042000000208DF8190000208DF81A0000208DF81B001A208DF81C000822DFF898180DF1D7
:204220001D0006F001FB00208DF825009DF81100811C04A806F05FF900F046BC4FF4807241
:20424000002104A806F00EFA68208DF8100015208DF81100DFF86808008840008DF8120005
:20426000DFF85C08008880B2C0098DF81300DFF85408008840008DF81400DFF848080088A5
:2042800080B2C0098DF81500DFF834080088401CDFF82C18088082208DF8160000208DF80D
:2042A000170003208DF8180000208DF8190000208DF81A0000208DF81B001B208DF81C000E
:2042C0000822DFF8F0170DF11D0006F0ADFA1524A4B204A89DF86B112154641CA4B204A8DB
:2042E000012121549DF86B01002804D1A4B204A8002121547CE09DF86B0102280FD09DF896
:204300006B0103280BD09DF86B01042807D09DF86B01052803D09DF86B01062844D19DF84D
:204320009D02002803D09DF89D02062837D19DF86B01022807D09DF86B01032803D09DF8E3
:204340006B01042821D19DF86B01DFF8241E08700222DFF81C1E692005F0D6F800208DF81B
:204360000D0048210DF10D0006F01CFE8DF80D009DF80D00DFF8F81D097888420AD04821FE
:20438000DFF8EC0D06F02DFE04E09DF86B01DFF8E41D0870A4B204A80021215428E0A4B201
:2043A00004A80121215423E09DF86B01DFF8C01D08700222DFF8B81D692005F0A5F800207F
:2043C0008DF80C00482103A806F0ECFD8DF80C009DF80C00DFF8981D0978884204D0482113
:2043E000DFF88C0D06F0FDFDA4B204A8002121549DF81100811C04A806F07DF8DFF8740D13
:204400000078052800D1FEE7DFF8680D0078062805D107F04FFE212008F032FCFEE753E3B3
:204420009DF86B01012861D10020DFF84C1D00220A709DF86C1104290BD29DF86C01DFF82F
:204440003C1D08709DF86E0100029DF86D11081803E0DFF8281D00220A70DFF8201D097822
:2044600001290AD180B208F04FFBDFF87C1E08F059FBDFF8781E086038E0DFF8001D0978A4
:2044800002290FD180B208F03FFBDFF85C1E08F049FBDFF87C1E086028E000BF947F00204D
:2044A000787E0020DFF8D41C097803291ED1DFF8641E00228A7080B23C2190FBF1F201FB15
:2044C0001201DFF8502E517080B23C2190FBF1F0DFF8401E087009E0A1740020A9740020B0
:2044E000C9740020A07400207B0900204FF48072002104A806F0B6F89DF86B01012821D1C5
:2045000004F022F80C2803D004F01EF80E2816D1DFF8040E0078012804D0DFF8FC0D0078A9
:2045200002280CD1DFF8F40D2C210170DFF8EC1D012003F01EFE00208DF8260002E0012000
:204540008DF826009DF86B01022820D1DFF8400E0078AA2818D103F0F7FF0E2807D003F053
:20456000F3FF0F2803D003F0EFFF11280CD1DFF8AC0D2D210170DFF8A41D012003F0F9FD57
:2045800000208DF8260002E001208DF8260068208DF8100015208DF81100DFF82405008832
:2045A00040008DF81200DFF81805008880B2C0098DF81300DFF80C05008840008DF81400CC
:2045C000DFF80005008880B2C0098DF81500DFF8F0040088401CDFF8E814088082208DF8B1
:2045E000160000208DF8170003208DF8180000208DF8190000208DF81A0000208DF81B00EC
:204600001C208DF81C000822DFF8A8140DF11D0006F00AF99DF86B018DF825009DF811009B
:20462000811C04A805F067FF4EE2DFF8740D0021018049E2667F00200020002108009DF89E
:204640006C11080000029DF86B110818411E89B2B1F5616F02D2DFF84C1D088000209DF841
:204660006E11080000029DF86D110818411E89B2B1F5616F02D2DFF8301D088000209DF839
:204680007011080000029DF86F110818411E89B2B1F5616F02D2DFF8141D088000209DF831
:2046A0007211080000029DF871110818411E89B2B1F5616F02D2DFF8F81C08804FF48072AA
:2046C000002104A805F0CEFF68208DF8100013208DF81100DFF8E803008840008DF8120044
:2046E000DFF8DC03008880B2C0098DF81300DFF8D403008840008DF81400DFF8C8030088B0
:2047000080B2C0098DF81500DFF8B4030088401CDFF8AC13088082208DF8160000208DF892
:20472000170003208DF8180000208DF8190000208DF81A0000208DF81B001E208DF81C0086
:204740000822DC490DF11D0006F06EF89DF81100811C04A805F0CFFE0121002005F09AFF12
:20476000B2E100BF967F0020467F00207C090020300900204FF48072002104A805F072FF67
:2047800068208DF810003D208DF81100CC48008840008DF81200CA48008880B2C0098DF87C
:2047A0001300C848008840008DF81400C548008880B2C0098DF81500C1480088401CC04955
:2047C000088082208DF8160000208DF8170003208DF8180000208DF8190000208DF81A001B
:2047E00000208DF81B001F208DF81C000822B1490DF11D0006F018F815241122DFF8B41BC2
:20480000A4B204A8201806F0C6FB29241122DFF8A81BA4B204A8201806F0BDFB3D24A4B2EE
:2048200004A8DFF8981B09882154641CA4B204A8DFF8881B098889B2090A2154641C9DF8D7
:204840001100811C04A805F056FE3DE15FF0000A65220021DFF8680B05F004FF15220021FC
:20486000DFF8600B05F0FEFE15220021DFF8580B05F0F8FE002410E0867F0020887F002028
:20488000A4B256A82018C07C5FFA8AFADFF8301B0AF801001AF1010A641CA4B2142C05D24B
:2048A000A4B256A82018C07C0028E9D15FFA8AFADFF80C0B3A210AF800101AF1010A0024DC
:2048C0000DE0A4B256A8201890F827005FFA8AFADFF8EC1A0AF801001AF1010A641CA4B207
:2048E000052C06D2A4B256A8201890F827000028E7D100240DE0A4B256A8201890F8680007
:204900005FFA8AFADFF8B81A0AF801001AF1010A641CA4B2462C06D2A4B256A8201890F8C4
:2049200068000028E7D100245FF0000A0DE0A4B256A8201890F82C005FFA8AFADFF8841A33
:204940000AF801001AF1010A641CA4B2142C06D2A4B256A8201890F82C000028E7D100240C
:204960005FF0000A12E000BF707E002098760020A4B256A8201890F840005FFA8AFADFF8E9
:20498000481A0AF801001AF1010A641CA4B2142C06D2A4B256A8201890F840000028E7D17A
:2049A0004FF48072002104A805F05CFE68208DF8100014208DF811004148008840008DF8E9
:2049C00012003F48008880B2C0098DF813003D48008840008DF814003A48008880B2C00938
:2049E0008DF8150036480088401C3549088082208DF8160000208DF8170003208DF81800FC
:204A000000208DF8190000208DF81A0000208DF81B0023208DF81C00082226490DF11D00C1
:204A200005F002FF03F090FD002803D003F08CFD01280CD1DFF8EC0B4FF6FF710180DFF8A8
:204A4000E80B0421017000208DF8250002E001208DF825009DF81100811C04A805F04BFD2A
:204A60000121002005F016FE2EE0DFF8BC0B00210170DFF8B80B00210180DFF8B40B4AF69B
:204A8000AA2101800322DFF8A81B5D2004F03CFD3A210DF10E0006F085FABDF80E00DFF8EB
:204AA000901B0988884204D03A21DFF8840B06F098FA09E0347C0020527F0020587F002032
:204AC000A07F00209E7F00209DF85C01672840F0A1849DF80100DFF85C1B0880DFF8540BE2
:204AE00000880002DFF84C1B0880DFF8480B00889DF800100843DFF83C1B0880DFF8340BF8
:204B0000008880B24008DFF82C1B08809DF86B0110F5FA60ADF834019DF86A018DF83601F7
:204B20009DF869018DF837019DF868018DF839019DF867018DF83A019DF8660100029DF8AC
:204B4000651108184FF47A71B0FBF1F08DF83B019DF89D02002804D09DF89D02062840F082
:204B600059844DA805F096F94FF6FF71884240F051844DA804F048FF4FF48072002104A829
:204B800005F070FD68208DF8100012208DF81100DFF8A40A008840008DF81200DFF8980A71
:204BA000008880B2C0098DF81300DFF8880A008840008DF81400DFF87C0A008880B2C00930
:204BC0008DF81500DFF8700A0088401CDFF8681A088067208DF8160000208DF81700032024
:204BE0008DF8180000208DF8190000208DF81A0000208DF81B0001208DF81C00072259A9EE
:204C0000491C0DF11D0006F0C6F99DF81100811C04A805F070FC00F0FDBB00BF28800008F8
:204C2000DFF8180A0088401CDFF8101A0880F1E31FFA8BFBBBF1010F42D11AF1010A40F284
:204C400026201FFA8AFA824503D340F22620BAEB000A1FFA8AFADFF8E8091AF8000002280C
:204C600026D100240CE01AF1010A40F226201FFA8AFA824503D340F22620BAEB000A641CBE
:204C8000A4B2092CEFD3DFF8B409A0F800A0DFF8B4094FF6FF710180DFF8AC094FF6FF71F0
:204CA00001800021002005F0F5FCB3E30050C347DFF888090088401CDFF880190880A9E38C
:204CC000DFF878090088401CDFF870190880A1E31FFA8AFADFF868091AF80000552840F088
:204CE00059831AF1010A40F226201FFA8AFA824503D340F22620BAEB000A1FFA8AFADFF875
:204D000040091AF80000BC2840F0F8804FF48C72002156A805F0A6FC002415E01AF1010A86
:204D200040F226201FFA8AFA824503D340F22620BAEB000AA4B256A81FFA8AFADFF80019B9
:204D40001AF801102154641CA4B21E2CE6D31AF1010A40F226201FFA8AFA824503D340F2E8
:204D60002620BAEB000ADFF8D408A0F800A01D2156A8FDF7F7FA9DF8751189B280B28142E7
:204D80007AD1DFF8C8089DF85B114170DFF8BC089DF85A118170DFF8B4089DF85911C17020
:204DA000DFF8A8089DF8581101719DF85C019DF85D1110EB0120DFF89418C880DFF88C08B5
:204DC0009DF861110172DFF884089DF860114172DFF878089DF85F118172DFF870089DF80A
:204DE0005E11C1729DF862019DF8631110EB0120DFF858188881DFF854089DF86711817370
:204E0000DFF848089DF86611C173DFF840089DF865110174DFF834089DF864114174DFF8E3
:204E20002C089DF873118174DFF820089DF87211C174DFF818089DF871110175DFF80C0875
:204E40009DF870114175DFF80408012101704521C0A806F0A7F81622DFF8F017C0A806F039
:204E600069F8002800F0D6824521DFF8E00706F0B8F8CFE20100C842DFF8C0070088401C59
:204E8000DFF8B817088006E0DFF8B0070088401CDFF8A8170880DFF8A4070088DFF8B017C6
:204EA0000988884200F0B682DFF89007008840F22621884208D3DFF88407008840F22621F8
:204EC000401ADFF878170880DFF870070088DFF880170988884200F09D82DFF86007008816
:204EE000DFF85C17405C682807D0DFF850070088DFF84C17405C5528C6D18BE21FFA8AFABB
:204F0000DFF83C071AF80000002808D01FFA8AFADFF82C071AF80000012840F008821FFAB0
:204F20008AFADFF81C071AF800005FEA002B1AF1010A40F226201FFA8AFA824503D340F273
:204F40002620BAEB000A1FFA8AFADFF8F4061AF8000010EB0B0BBBF1040040F20B1180B29B
:204F6000884280F0DE81A4B21FFA8BFB1BF101008442C0F24F824FF48C72002156A805F0F8
:204F800071FB55208DF858011FFA8BFB5FEA1B208DF8590158468DF85A0100240320040087
:204FA00015E01AF1010A40F226201FFA8AFA824503D340F22620BAEB000AA4B256A81FFAA0
:204FC0008AFADFF87C161AF801102154641CA4B21FFA8BFB1BF101008442E2DB1AF1010A31
:204FE00040F226201FFA8AFA824503D340F22620BAEB000ADFF84406A0F800A0594689B2A5
:2050000056A8FDF7C9F91FFA8BFB56A91BF8011089B280B2814240F0FD819DF85B01A02883
:205020000CD0A12821D0A22836D0A3284BD0A42800F0B680AF2800F05B8171E19DF85C014B
:20504000012811D1DFF80C06008800280CD1DFF8080600210180DFF804064FF6FF71018031
:20506000DFF8FC0500210180D4E19DF85C01012811D1DFF8E005008800280CD1DFF8DC0503
:2050800000210180DFF8DC054FF6FF710180DFF8D00500210180BDE19DF85C01012811D197
:2050A000DFF8B005008800280CD1DFF8B80500210180DFF8B4054FF6FF710180DFF8A0055F
:2050C00000210180A6E19DF85C01012867D1DFF884050088002862D1DFF88C050021018007
:2050E000DFF888054FF6FF710180DFF868054FF6FF7101809DF86001DFF874150860DFF807
:20510000700500689DF85F1110EB0120DFF860150860DFF85C0500689DF85E1110EB0140FD
:20512000DFF84C150860DFF8480500689DF85D1110EB0160DFF838150860DFF834050068E0
:205140004FF48071B0FBF1F202FB1102002A04D1DFF81C050068000A04E0DFF814050068D8
:20516000000A401CDFF80C150880002410E000BF28800020720900201B8000201C8000209C
:20518000A4B24FF4805000FB04F007F0FFFB641CA4B2502CF4D3DFF8C8040021018039E14E
:2051A0009DF85901012840F09D809DF85A01082840F098809DF85C019DF85D1111EB002011
:2051C000DFF8B014098880B2814208D0DFF8A8044FF6FF710180DFF8940400210180DFF835
:2051E0009C040088401C9DF85E119DF85F2112EB0121884276D19DF85E019DF85F1111EBED
:205200000020DFF878140880DFF87404DFF86C1409880180DFF8480400210180DFF85C04CF
:205220000088DFF850140988884229D10023DFF840040068DFF83C140988491E4FF480725C
:205240005143401A0300DBB29BB258AADFF82C0400884FF48071484310F57061022007F044
:205260001CF8DFF820044FF6FF710180DFF808044FF6FF710180DFF8F4030021018031E04F
:20528000DFF8F8030088032815D10C22DFF8F81358A805F04FFE002816D0DFF88C030121BB
:2052A0000170DFF8D4034FF6FF710180DFF8BC030021018008E0DFF8C4030088042803D351
:2052C000DFF86403032101704FF4807358AADFF8AC0300884FF48071484310F570610220FE
:2052E00006F0DBFF96E000BF0000C8423C7E00209DF85C0101280AD1DFF87C0300210180D7
:20530000C84800210180DFF858030021018081E0407E0020F07C0020328000207D090020C4
:2053200078E0C6480088401CC449088072E0C3480088401CC149088004E0C0480088401CEB
:20534000BE490880BD480088C1490988884261D0BA48008840F22621884206D3B74800886E
:2053600040F22621401AB5490880B4480088B849098888424ED0B1480088B149405C68282F
:2053800005D0AE480088AE49405C5528D5D141E073090020A9480088401CA84908801AE0FF
:2053A0009A7F002046090020480900204A0900204C0900205880000830800008647F002051
:2053C000A8720020B0760020C87600209B480088401C9A490880994800889D490988884213
:2053E00018D09648008840F22621884206D39348008840F22621401A904908808F4800884D
:2054000093490988884205D08C4800888C49405C6828DBD183480088002842F07182894806
:20542000008800282FD1DFF8300E0088974909880A22514390FBF1F201FB1200002822D157
:205440004FF48072002104A805F00CF968208DF8100001208DF8110002208DF81200082299
:205460008B490DF1130005F0DFF900208DF81B0000208DF81C000D2104A805F03CF80121D4
:20548000002005F007F9DFF8D00D0088814909880A22514390FBF1F201FB1200002825D106
:2054A000694800884FF6FF7188421FD14FF48072002104A805F0D6F868208DF8100004203E
:2054C0008DF8110043208DF8120000208DF8130000208DF8140000208DF81500062104A83E
:2054E00005F009F80121002005F0D4F8DFF8680D0088694909880A22514390FBF1F201FB72
:205500001200002813D0654800785FFA89F948450DD1634800785FFA88F8404507D1614801
:205520000078DFF8981E0978884200F0CD80464800884FF6FF71884240F0C680574880F8BC
:205540000090574880F800805648DFF8701E0978017068208DF8100020208DF811003648BE
:20556000008840008DF812003348008880B2C0098DF813002F48008840008DF814002D48E9
:20558000008880B2C0098DF815002B480088401C2949088086208DF8160000208DF81700A0
:2055A00003208DF8180000208DF8190000208DF81A0000208DF81B0001208DF81C003000FC
:2055C0008DF81D00B6B2300A8DF81E0038008DF81F00BFB2380A8DF82000BDF804008DF872
:2055E00021008DF8228028008DF82300280A8DF82400280C8DF82500280E8DF826000822CF
:2056000023490DF1270005F00FF95FFA88F8B8F1020F02D0BFB2012F46D301208DF82F0008
:2056200045E000BF687F002030800020727F00205E7F00209E7F0020A07F00209C7F0020EA
:20564000DC500020887F0020867F002098760020FC7E0020B07F00204E090020A27F0020E3
:20566000B27F0020A47F0020A67F0020A87F0020A47E00206E7F0020AA7F0020707F002063
:205680006C7F0020AC7F00200022000846090020347C0020480900204A0900203780002090
:2056A000388000203980002000208DF82F008DF83090DFF8080D00788DF831009DF8110060
:2056C000811C04A804F017FFDFF8D00E00884FF6FF71884240F0D480DFF8C40E00884FF6C1
:2056E000FF71884240F0CC80DFF86C0B00884FF4FA7190FBF1F201FB1200002840F0C0805C
:205700004FF48072002104A804F0ACFF68208DF8100013208DF81100DFF8880E00884000CD
:205720008DF81200DFF87C0E008880B2C0098DF81300DFF8740E008840008DF81400DFF8C5
:20574000680E008880B2C0098DF81500DFF8540E0088401CDFF84C1E088082208DF8160093
:2057600000208DF8170003208DF8180000208DF8190000208DF81A0000208DF81B0005204B
:205780008DF81C000D240822DFF8201EA4B204A8201805F049F89DF81100811C04A804F0A5
:2057A000AAFE0121002004F075FF4FF48072002104A804F057FF68208DF810001D208DF86C
:2057C0001100DFF8E00D008840008DF81200DFF8D40D008880B2C0098DF81300DFF8C80D16
:2057E000008840008DF81400DFF8BC0D008880B2C0098DF81500DFF8AC0D0088401CDFF840
:20580000A41D088082208DF8160000208DF8170003208DF8180000208DF8190000208DF823
:205820001A0000208DF81B000C208DF81C000D240822DFF8781DA4B204A8201804F0F4FFD9
:205840000834DFF86C0D4AF2E03101600922A4B204A82118DFF8580D006805F041FB0921A9
:20586000A4B204A8201805F0C7F80934A4B204A8002121549DF81100811C04A804F03BFE49
:20588000DFF8080F00884FF6FF71884240F0B780DFF80C0D00884FF6FF71884240F0AF8056
:2058A000DFF8E80E002101804FF48072002104A804F0D8FE68208DF8100079208DF8110061
:2058C000DFF8E00C008840008DF81200DFF8D40C008880B2C0098DF81300DFF8CC0C00889D
:2058E00040008DF81400DFF8C00C008880B2C0098DF81500DFF8AC0C0088401CDFF8A41C05
:20590000088082208DF8160000208DF8170003208DF8180000208DF8190000208DF81A00C9
:2059200000208DF81B0001208DF81C000822DFF87C1C0DF11D0004F077FFDFF8541E4AA88C
:2059400005F040F808224AA90DF1250005F023FB08210DF1250005F04FF8062200210DF1F8
:205960002D0004F07FFE06210DF12D0005F044F80A2200210DF1330004F074FE0622DFF823
:20598000141E0DF13D0005F006FB0A2200210DF1430004F067FE042200210DF14D0004F037
:2059A00061FE022200210DF1510004F05BFE202200210DF1530004F055FE082200210DF163
:2059C000730004F04FFE0822DFF8CC1D0DF17B0005F0E1FA082200210DF1830004F042FEE0
:2059E00008210DF1830005F007F89DF81100811C04A804F080FD0121002004F04BFEDFF853
:205A00009C0D00884FF6FF71884263D1DFF8900B00884FF6FF7188425CD1DFF83C08008859
:205A2000142190FBF1F201FB1200002852D14FF48072002104A804F015FE68208DF8100044
:205A400013208DF81100DFF85C0B008840008DF81200DFF8500B008880B2C0098DF8130093
:205A6000DFF8440B008840008DF81400DFF8380B008880B2C0098DF81500DFF8280B0088D6
:205A8000401CDFF8201B088082208DF8160000208DF8170003208DF8180000208DF8190099
:205AA00000208DF81A0000208DF81B001D208DF81C000822DFF8F41A0DF11D0004F0B4FEB9
:205AC0009DF81100811C04A804F015FD0121002004F0E0FDDFF8C80C00884FF6FF7188420C
:205AE00040F0F782DFF8B80A00884FF6FF71884240F0EF82DFF8A80C002101804FF480725A
:205B0000002104A804F0AEFD68208DF81000A8208DF81100DFF88C0A008840008DF81200D2
:205B2000DFF8800A008880B2C0098DF81300DFF8780A008840008DF81400DFF86C0A00885A
:205B400080B2C0098DF81500DFF8580A0088401CDFF8501A088082208DF8160000208DF8E8
:205B6000170003208DF8180000208DF8190000208DF81A0000208DF81B0002208DF81C004E
:205B80000322DFF88C1E4FF4097005F0A9F9DFF8800E4078BC21484300F25020DFF8101A24
:205BA0000860BC22DFF86C1EDFF8040A006805F097F90D240822DFF8F419A4B204A82018F3
:205BC00004F032FE0834DFF84C0E806A04F0A6FEA4B204A96054641CA4B204A9000A6054BA
:205BE000641CDFF8300E90F83E0004F097FEA4B204A96054641CDFF81C0E90F83D0004F0D0
:205C00008DFEA4B204A96054641CDFF8080E90F83C0004F083FEA4B204A96054641CDFF88E
:205C2000F40D90F83B0004F079FEA4B204A96054641CDFF8E00D90F83A0004F06FFEA4B2C1
:205C400004A96054641CDFF8CC0D008FB0F5FA6004F064FEA4B204A96054641C0822DFF897
:205C60004C19A4B204A8201804F0DEFD0834A4B204A8DFF8A01D91F895102154641CA4B26B
:205C800004A800212154641C0822DFF80C1BA4B204A8201805F07FF908340822DFF8481ED0
:205CA000A4B204A8201805F076F90834DFF8640D90F83E004FF47A714843A4B204A960548C
:205CC000641CA4B204A9000A6054641CA4B204A8DFF8401D91F83D102154641CA4B204A800
:205CE000DFF8301D91F83C102154641CA4B204A8DFF8201D91F83B102154641CA4B204A8D5
:205D0000DFF8101D91F83A102154641CA4B204A8DFF8001D098F30312154641CDFF8F40CFC
:205D200090F846004FF47A714843A4B204A96054641CA4B204A9000A6054641CA4B204A862
:205D4000DFF8D01C91F845102154641CA4B204A8DFF8C01C91F844102154641CA4B204A824
:205D6000DFF8B01C91F843102154641CA4B204A8DFF8A01C91F842102154641CA4B204A848
:205D8000DFF8901CB1F8401030312154641CDFF8840C406FDFF8541D04F0E6FB04F050FCBE
:205DA000A4B204A96054641CA4B204A9020A6254641CA4B204A9020C6254641CA4B204A91D
:205DC000000E6054641CDFF84C0CD0F88400DFF81C1D04F0C9FB04F033FCA4B204A9605464
:205DE000641CA4B204A9020A6254641CA4B204A9020C6254641CA4B204A9000E6054641C52
:205E0000DFF8100C806FDFF8E41C04F0ADFB04F017FCA4B204A96054641CA4B204A9020AE0
:205E20006254641CA4B204A9020C6254641CA4B204A9000E6054641CDFF8D80BD0F8880096
:205E4000DFF8A81C04F090FB04F0FAFBA4B204A96054641CA4B204A9020A6254641CA4B26D
:205E600004A9020C6254641CA4B204A9000E6054641CDFF8A00BC06FDFF8701C04F074FB75
:205E800004F0DEFBA4B204A96054641CA4B204A9020A6254641CA4B204A9020C6254641C72
:205EA000A4B204A9000E6054641CDFF8680BD0F88C00DFF8381C04F057FB04F0C1FBA4B288
:205EC00004A96054641CA4B204A9020A6254641CA4B204A9020C6254641CA4B204A9000E44
:205EE0006054641CDFF82C0BD0F88000DFF8FC1B04F03AFB04F0A4FBA4B204A96054641C37
:205F0000A4B204A9020A6254641CA4B204A9020C6254641CA4B204A9000E6054641CDFF8D9
:205F2000F40AD0F89000DFF8C41B04F01DFB04F087FBA4B204A96054641CA4B204A9020A8D
:205F40006254641CA4B204A9020C6254641CA4B204A9000E6054641CDFF8B80A406DDFF862
:205F60008C1B04F001FB04F06BFBA4B204A96054641CA4B204A9020A6254641CA4B204A9B1
:205F8000020C6254641CA4B204A9000E6054641CDFF8800A806DDFF8541B04F0E5FA04F01D
:205FA0004FFBA4B204A96054641CA4B204A9020A6254641CA4B204A9020C6254641CA4B27E
:205FC00004A9000E6054641CDFF8480AC06DDFF81C1B04F0C9FA04F033FBA4B204A96054DE
:205FE000641CA4B204A9020A6254641CA4B204A9020C6254641CA4B204A9000E6054641C50
:20600000DFF8100A006EDFF8E41A04F0ADFA04F017FBA4B204A96054641CA4B204A9020A65
:206020006254641CA4B204A9020C6254641CA4B204A9000E6054641CDFF8D809006DDFF8A2
:20604000AC1A04F091FA04F0FBFAA4B204A96054641CA4B204A9020A6254641CA4B204A993
:20606000020C6254641CA4B204A9000E6054641CA4B204A802212154641CA4B204A800215A
:206080002154641C241D241DA4B204A800212154641CA4B204A800212154641CA4B204A857
:2060A000DFF8701991F894102154641C241D2022DFF83C1AA4B204A8201804F06CFF9DF880
:2060C0001100811C04A804F016FA0121002004F0E1FA02F039FA60490988DFF8182A12883F
:2060E0000A235A4391FBF2F302FB1311002941F02C8180B2112801F02881DFF8A404008831
:206100004FF6FF71884241F020810322DFF800194FF4097004F0E4FE0222DFF8DC19262051
:2061200003F0F2F9DFF8E80880780128C0F07484DFF8C809006800284DD1DFF8080F007835
:20614000BC21484300F25020DFF864140860BC22DFF8C018DFF85804006804F0C1FE0621BC
:20616000DFF8940904F03DFFDFF8A8080079AA2823D0DFF8A008AA210171BC22DFF8941899
:20618000DFF82C04006804F0C0FEDFF884088078012812D3DFF878088078401EDFF8701869
:2061A00088700322DFF868184FF4097004F0ADFE0621DFF8440904F014FFDFF8880E0078D9
:2061C000401CDFF8801E0870DFF8300942F20F71016001F0BAB8DFF86C0E0078BF2803D368
:2061E000DFF8600E01210170DFF8580E0078BC21484300F25020EE490860BC22DFF81418C8
:20620000EB48006804F06CFEDFF8E00E00210170DFF80008007955282FD0DFF8280E0078D5
:20622000401CDFF8201E0870DFF8180E0078BF2803D3DFF8100E01210170DFF8080E007856
:20624000BC21484300F25020D9490860BC22DFF8C417D74802E000BF8A7F0020006804F015
:206260003FFEDFF8880E0078401CDFF8801E0870DFF8780E0078BF28CAD3DFF8980700796B
:20628000AA2801F06280DFF88C07806ADFF86C1808604FF48072002104A804F0E3F96820E8
:2062A0008DF81000E5208DF81100BE48008840008DF81200BB48008880B2C0098DF813002B
:2062C000B948008840008DF81400B748008880B2C0098DF81500B3480088401CB1490880DF
:2062E00082208DF8160000208DF8170003208DF8180000208DF8190000208DF81A00002048
:206300008DF81B0003208DF81C000822A7490DF11D0004F089FADFF8FC06806A04F0FEFABE
:2063200001008DF82510000A8DF82600DFF8E40690F83E0004F0F2FA8DF82700DFF8D40629
:2063400090F83D0004F0EAFA8DF82800DFF8C40690F83C0004F0E2FA8DF82900DFF8B4067F
:2063600090F83B0004F0DAFA8DF82A00DFF8A40690F83A0004F0D2FA8DF82B00DFF89406BF
:20638000008FB0F5FA6004F0C9FA8DF82C00082286490DF12D0004F047FA0822DFF8201F6E
:2063A0004AA804F0F8FD08224AA90DF1350004F0F2FD0822DFF8301702E000BF3B8000200B
:2063C0000DF13D0004F0E7FDDFF8480690F83E004FF47A71484301008DF84610000A8DF89B
:2063E0004700DFF8300690F83D008DF84800DFF8240690F83C008DF84900DFF8180690F8A7
:206400003B008DF84A00DFF80C0690F83A008DF84B00DFF80006008F30308DF84C00DFF883
:20642000F40590F846004FF47A71484301008DF84D10000A8DF84E00DFF8D80590F845009B
:206440008DF84F00DFF8CC0590F844008DF85000DFF8C00590F843008DF85100DFF8B40552
:2064600090F842008DF85200DFF8A805B0F8400030308DF853004424DFF89805406FDFF875
:206480006C1604F071F804F0DBF8A4B204A96054641CA4B204A9020A6254641CA4B204A9D7
:2064A000020C6254641CA4B204A9000E6054641CDFF86005D0F88400DFF8301604F054F86E
:2064C00004F0BEF8A4B204A96054641CA4B204A9020A6254641CA4B204A9020C6254641C4F
:2064E000A4B204A9000E6054641CDFF82805806FDFF8F81504F038F804F0A2F8A4B204A9CB
:206500006054641CA4B204A9020A6254641CA4B204A9020C6254641CA4B204A9000E6054F6
:20652000641CDFF8F004D0F88800DFF8C01504F01BF804F085F8A4B204A96054641CA4B20F
:2065400004A9020A6254641CA4B204A9020C6254641CA4B204A9000E6054641CDFF8B40431
:20656000C06FDFF8881503F0FFFF04F069F8A4B204A96054641CA4B204A9020A6254641CB6
:20658000A4B204A9020C6254641CA4B204A9000E6054641CDFF87C040CE000BF987F002036
:2065A000867F0020A07F00209E7F0020347C0020A07E0020D0F88C00DFF8301503F0D4FFF6
:2065C00004F03EF8A4B204A96054641CA4B204A9020A6254641CA4B204A9020C6254641CCE
:2065E000A4B204A9000E6054641CDFF82804D0F88000DFF8F81403F0B7FF04F021F8A4B21C
:2066000004A96054641CA4B204A9020A6254641CA4B204A9020C6254641CA4B204A9000EFC
:206620006054641CDFF8EC03D0F89000DFF8BC1403F09AFF04F004F8A4B204A96054641CAE
:20664000A4B204A9020A6254641CA4B204A9020C6254641CA4B204A9000E6054641CA4B213
:2066600004A802212154641CA4B204A800212154641C0834DFF81C0E0068DFF81C1E03F095
:2066800073FF03F0DDFFA4B204A96054641CA4B204A9020A6254641CA4B204A9020C625476
:2066A000641CA4B204A9000E6054641CD948406DDFF8381403F058FF03F0C2FFA4B204A923
:2066C0006054641CA4B204A9020A6254641CA4B204A9020C6254641CA4B204A9000E605435
:2066E000641CCC48406EDFF8041403F03DFF03F0A7FFA4B204A96054641CA4B204A9020A5B
:206700006254641CA4B204A9020C6254641CA4B204A9000E6054641CDFF8800D0068DFF814
:20672000781D03F021FF03F08BFFA4B204A96054641CA4B204A9020A6254641CA4B204A9B5
:20674000020C6254641CA4B204A9000E6054641CB048806DE54903F007FF03F071FFA4B2EB
:2067600004A96054641CA4B204A9020A6254641CA4B204A9020C6254641CA4B204A9000E9B
:206780006054641CA348806ED8490BE0947F00207A7400206A7400208A7400209A7F00204A
:2067A000967F002003F0E0FE03F04AFFA4B204A96054641CA4B204A9020A6254641CA4B2C5
:2067C00004A9020C6254641CA4B204A9000E6054641CDFF8980E0068DFF8BC1C03F0C4FE3A
:2067E00003F02EFFA4B204A96054641CA4B204A9020A6254641CA4B204A9020C6254641CB6
:20680000A4B204A9000E6054641C8248C06DB74903F0AAFE03F014FFA4B204A96054641C64
:20682000A4B204A9020A6254641CA4B204A9020C6254641CA4B204A9000E6054641C7548CA
:20684000C06EAA4903F090FE03F0FAFEA4B204A96054641CA4B204A9020A6254641CA4B2D9
:2068600004A9020C6254641CA4B204A9000E6054641CDFF8FC0D0068DFF81C1C03F074FE26
:2068800003F0DEFEA4B204A96054641CA4B204A9020A6254641CA4B204A9020C6254641C66
:2068A000A4B204A9000E6054641C5A48006E8F4903F05AFE03F0C4FEA4B204A96054641C74
:2068C000A4B204A9020A6254641CA4B204A9020C6254641CA4B204A9000E6054641C4D4852
:2068E000006F824903F040FE03F0AAFEA4B204A96054641CA4B204A9020A6254641CA4B2C0
:2069000004A9020C6254641CA4B204A9000E6054641C4048006D754903F026FE03F090FEF6
:20692000A4B204A96054641CA4B204A9020A6254641CA4B204A9020C6254641CA4B204A991
:20694000000E6054641CA4B204A8324991F895102154641CA4B204A800212154641C00201D
:2069600049902C48406B614903F0FEFD03F068FE4990042249A9A4B204A8201804F00BFB09
:20698000241D241D2348C06C584903F0EDFD03F057FEA4B204A96054641CA4B204A9020AD2
:2069A0006254641CA4B204A9020C6254641CA4B204A9000E6054641CA4B204A8154991F82C
:2069C00095102154641CA4B204A800212154641CA4B204A800212154641CA4B204A80D4995
:2069E00091F894102154641C20224149A4B204A8201804F0D0FA9DF81100811C04A803F0CF
:206A00007AFD0121002003F045FE00F09EBC00BF9C7E0020F06E00200322DFF8141F4FF454
:206A20000D7004F05DFA02223349272002F06CFDDFF8FC0E80780128C0F087842F480068B0
:206A400000285DD1DFF8FC050078BC2148F6D85201FB0020DFF8DC1E0860BC22DFF8D81E4B
:206A6000DFF8D00E006804F03BFA0721224804F0B8FADFF8C40E0079AA2827D0DFF8B80E10
:206A8000AA210171BC22DFF8B01EDFF8A80E006804F03BFADFF8980E8078012816D3DFF8BA
:206AA000900E8078401EDFF8881E88700322DFF8801E4FF40D7004F028FA02220E4927203B
:206AC00002F022FD07210C4804F08BFADFF874050078401CDFF86C150870084842F20F71B8
:206AE000016000F032BC00BFF56E00200000C8428A6F00204C0900209E7E002030090020E8
:206B0000DFF8400500780B2803D3DFF8380501210170DFF830050078BC2148F6D85201FB6C
:206B20000020DFF8101E0860BC22DFF80C1EDFF8040E006804F0D4F9DFF8B00500210170B9
:206B4000DFF8F40D007955282ED0DFF8F8040078401CDFF8F0140870DFF8E80400780B2801
:206B600003D3DFF8E00401210170DFF8D8040078BC2148F6D85201FB0020DFF8B81D086051
:206B8000BC22DFF8B41DDFF8AC0D006804F0A8F9DFF858050078401CDFF850150870DFF84F
:206BA0004C0500780B28CBD3DFF88C0D0079AA2800F0CB83DFF8800D806ADFF8801D086018
:206BC0004FF48072002104A803F04CFD68208DF81000E5208DF81100DFF8640D00884000AF
:206BE0008DF81200DFF8580D008880B2C0098DF81300DFF8500D008840008DF81400DFF83B
:206C0000440D008880B2C0098DF81500DFF8300D0088401CDFF8281D088082208DF816002D
:206C200000208DF8170003208DF8180000208DF8190000208DF81A0000208DF81B00032078
:206C40008DF81C000822DFF8001D0DF11D0003F0EBFDDFF8E40C806A03F060FE01008DF8F7
:206C60002510000A8DF82600DFF8CC0C90F83E0003F054FE8DF82700DFF8BC0C90F83D0060
:206C800003F04CFE8DF82800DFF8AC0C90F83C0003F044FE8DF82900DFF89C0C90F83B0092
:206CA00003F03CFE8DF82A00DFF88C0C90F83A0003F034FE8DF82B00DFF87C0C008FB0F55F
:206CC000FA6003F02BFE8DF82C000822DFF8781C0DF12D0003F0A8FD0822DFF8E4154AA849
:206CE00004F059F908224AA90DF1350004F053F90822DFF8C81E0DF13D0004F04CF9DFF88C
:206D0000380C90F83E004FF47A71484301008DF84610000A8DF84700DFF81C0C90F83D003A
:206D20008DF84800DFF8100C90F83C008DF84900DFF8040C90F83B008DF84A00DFF8F80BAE
:206D400090F83A008DF84B00DFF8EC0B008F30308DF84C00DFF8E00B90F846004FF47A7155
:206D6000484301008DF84D10000A8DF84E00DFF8C80B90F845008DF84F00DFF8BC0B90F857
:206D800044008DF85000DFF8B00B90F843008DF85100DFF8A40B90F842008DF85200DFF8A9
:206DA000980BB0F8400030308DF853004424DFF8880B406FDFF8081E03F0D6FB03F040FC9F
:206DC000A4B204A96054641CA4B204A9020A6254641CA4B204A9020C6254641CA4B204A9ED
:206DE000000E6054641CDFF8500BD0F88400DFF8D01D03F0B9FB03F023FCA4B204A960549F
:206E0000641CA4B204A9020A6254641CA4B204A9020C6254641CA4B204A9000E6054641C21
:206E2000DFF8140B806FDFF8981D03F09DFB03F007FCA4B204A96054641CA4B204A9020A1A
:206E40006254641CA4B204A9020C6254641CA4B204A9000E6054641CDFF8DC0AD0F8880063
:206E6000DFF85C1D03F080FB03F0EAFBA4B204A96054641CA4B204A9020A6254641CA4B2AA
:206E800004A9020C6254641CA4B204A9000E6054641CDFF8A40AC06FDFF8241D03F064FB9E
:206EA00003F0CEFBA4B204A96054641CA4B204A9020A6254641CA4B204A9020C6254641C53
:206EC000A4B204A9000E6054641CDFF86C0AD0F88C00DFF8EC1C03F047FB03F0B1FBA4B2C3
:206EE00004A96054641CA4B204A9020A6254641CA4B204A9020C6254641CA4B204A9000E14
:206F00006054641CDFF8300AD0F88000DFF8B01C03F02AFB03F094FBA4B204A96054641C70
:206F2000A4B204A9020A6254641CA4B204A9020C6254641CA4B204A9000E6054641CDFF8A9
:206F4000F809D0F89000DFF8781C03F00DFB03F077FBA4B204A96054641CA4B204A9020AC7
:206F60006254641CA4B204A9020C6254641CA4B204A9000E6054641CA4B204A802212154B5
:206F8000641CA4B204A800212154641C0834DFF804050068DFF8001503F0E6FA03F050FBD8
:206FA000A4B204A96054641CA4B204A9020A6254641CA4B204A9020C6254641CA4B204A90B
:206FC000000E6054641CDFF87009406DDFF8F01B03F0CAFA03F034FBA4B204A96054641C80
:206FE000A4B204A9020A6254641CA4B204A9020C6254641CA4B204A9000E6054641CDFF8E9
:207000003809406EDFF8B81B03F0AEFA03F018FBA4B204A96054641CA4B204A9020A62543A
:20702000641CA4B204A9020C6254641CA4B204A9000E6054641CDFF864040068DFF858145A
:2070400002E000BF7A09002003F08EFA03F0F8FAA4B204A96054641CA4B204A9020A625490
:20706000641CA4B204A9020C6254641CA4B204A9000E6054641CDFF8C008806DDFF8401B46
:2070800003F072FA03F0DCFAA4B204A96054641CA4B204A9020A6254641CA4B204A9020C3B
:2070A0006254641CA4B204A9000E6054641CDFF88808806EDFF8081B03F056FA03F0C0FA16
:2070C000A4B204A96054641CA4B204A9020A6254641CA4B204A9020C6254641CA4B204A9EA
:2070E000000E6054641CDFF8840501E0338000200068E94903F038FA03F0A2FAA4B204A9E9
:207100006054641CA4B204A9020A6254641CA4B204A9020C6254641CA4B204A9000E6054EA
:20712000641CDFF81408C06DDFF8941A03F01CFA03F086FAA4B204A96054641CA4B204A974
:20714000020A6254641CA4B204A9020C6254641CA4B204A9000E6054641CDFF8DC07C06E79
:20716000DFF85C1A03F000FA03F06AFAA4B204A96054641CA4B204A9020A6254641CA4B2AC
:2071800004A9020C6254641CA4B204A9000E6054641CDFF8DC040068BF4903F0E5F903F0CE
:2071A0004FFAA4B204A96054641CA4B204A9020A6254641CA4B204A9020C6254641CA4B26D
:2071C00004A9000E6054641CDFF86C07006EDFF8F01903F0C9F903F033FAA4B204A960549C
:2071E000641CA4B204A9020A6254641CA4B204A9020C6254641CA4B204A9000E6054641C3E
:20720000DFF83407006FDFF8B81903F0ADF903F017FAA4B204A96054641CA4B204A9020A62
:207220006254641CA4B204A9020C6254641CA4B204A9000E6054641CDFF8FC06006DDFF86F
:20724000801903F091F903F0FBF9A4B204A96054641CA4B204A9020A6254641CA4B204A9B2
:20726000020C6254641CA4B204A9000E6054641CA4B204A8DFF8C01691F895102154641CB3
:20728000A4B204A800212154641C00204890DFF8A806406BDFF8281903F066F903F0D0F988
:2072A0004890042248A9A4B204A8201803F073FE241D241DDFF88006C06CDFF8041901E061
:2072C000056F002003F050F903F0BAF9A4B204A96054641CA4B204A9020A6254641CA4B266
:2072E00004A9020C6254641CA4B204A9000E6054641CA4B204A8DFF8401691F89510215486
:20730000641CA4B204A800212154641CA4B204A800212154641CA4B204A8DFF81C1691F829
:2073200094102154641C2022DFF85C1CA4B204A8201803F030FE9DF81100811C04A803F0E6
:20734000DAF80121002003F0A5F9DFF8400C00884AF6AA21884206D1DFF8340C00884FF64D
:20736000FF7188426FD1DFF82C0C00884FF6FF71884268D1DFF8200C0088642190FBF1F2C6
:2073800001FB120000285ED14FF48072002104A803F068F968208DF8100028208DF8110037
:2073A000DFF89C05008840008DF81200DFF89005008880B2C0098DF81300DFF88805008883
:2073C00040008DF81400DFF87C05008880B2C0098DF81500DFF868050088401CDFF86015EB
:2073E000088082208DF8160000208DF8170003208DF8180000208DF8190000208DF81A00CF
:2074000000208DF81B0035208DF81C000822DFF838150DF11D0003F007FA1122DFF87C1BB8
:207420000DF1250003F0B7FDDFF8740B00788DF839009DF81100811C04A803F05CF801219E
:20744000002003F027F9DFF85C0B00884FF6FF71884213D1DFF84C0B002101804FF48072CB
:20746000002104A803F0FEF855208DF81000BC208DF81100022104A803F03DF8DFF8280BD9
:2074800000884FF6FF71884240F0D080DFF8180B06E000BF607E00200050C347647E00206C
:2074A000002101804521BAA803F07CFD1622DFF8FC1ABAA803F03EFD002804D04521DFF808
:2074C000EC0A03F08EFD4FF48072002104A803F0C9F855208DF81000BA208DF81100DFF831
:2074E000CC0A00798DF81200DFF8C00AC0788DF81300DFF8B80A80788DF81400DFF8AC0A7E
:2075000040788DF81500DFF8A40AC0888DF81600DFF8980AC08880B2000A8DF81700DFF841
:207520008C0AC07A8DF81800DFF8800A807A8DF81900DFF8780A407A8DF81A00DFF86C0AE6
:20754000007A8DF81B00DFF8640A80898DF81C00DFF8580A808980B2000A8DF81D00DFF82B
:207560004C0A407C8DF81E00DFF8400A007C8DF81F00DFF8380AC07B8DF82000DFF82C0A0F
:20758000807B8DF8210001208DF8220000208DF82300C2208DF8240001208DF82500032041
:2075A0008DF8260000208DF8270000208DF8280004208DF82900DFF8F409407D8DF82A0075
:2075C000DFF8E809007D8DF82B00DFF8E009C07C8DF82C00DFF8D409807C8DF82D001E2168
:2075E00004A8FAF7EEFE8DF82E001F2104A802F082FF4FF47A7000F04DFE1F2104A802F0AA
:207600007AFF4FF47A7000F045FE1F2104A802F072FF4FF47A7000F03DFE1F2104A802F00C
:207620006AFFDFF88C094FF6FF710180DFF8800900884FF6FF71884247D1DFF85C090088FC
:207640001E2190FBF1F201FB120000283DD14FF48072002104A803F005F855208DF810003D
:20766000FF208DF81100002409E000BF687E00206C7E0020A4B204A820188470641CA4B275
:207680001C2CF7D37A208DF82E001F2104A802F032FF4FF47A7000F0FDFD1F2104A802F087
:2076A0002AFF4FF47A7000F0F5FD1F2104A802F022FF4FF47A7000F0EDFD1F2104A802F0AE
:2076C0001AFFDFF8EC0800210180DFF8E80800884FF6FF71884240F0B780DFF8D808002117
:2076E0000180DFF8C808002101704521B4A803F059FC1622DFF8B418B4A803F01BFC00285D
:2077000004D04521DFF8A40803F06BFC4FF48072002104A802F0A6FF1222DFF89C1804A84E
:2077200003F039FC31208DF822002C208DF8230022208DF8240054208DF8250043208DF844
:20774000260050208DF8270022208DF828002C208DF8290022208DF82A0000244521DFF8AC
:207760004C0803F01FFCDFF8441884B06846162205F08EFA0FBCFAF73DFE0400E4B222002A
:20778000DFF838180DF12B0003F005FCE4B204A820182C21C176E4B204A820183121017763
:2077A000E4B204A820180D214177E4B204A820180A218177E4B214F11F0104A802F09BFEDA
:2077C0004FF47A7000F066FDE4B214F11F0104A802F091FE4FF47A7000F05CFDE4B214F130
:2077E0001F0104A802F087FE0DF58860342105F087FAE4B214F119020DF116010DF58860DC
:2078000003F0C9FBE4B214F119010DF5886002F072FE4FF47A7000F03DFDE4B214F11901A4
:207820000DF5886002F067FE4FF47A7000F032FDE4B214F119010DF5886002F05CFEDFF8F9
:2078400080074FF6FF710180DFF8740700884FF6FF71884251D1DFF840070088142190FB8A
:20786000F1F201FB1200002847D14FF48072002104A802F0F7FE1022DFF8481704A803F0E7
:207880008AFB0D208DF820000A208DF82100122104A802F030FE40F2DC5000F0FBFC12214A
:2078A00004A802F028FE40F2DC5000F0F3FC122104A802F020FE9CA8142105F021FA0C2221
:2078C0000DF116019CA803F066FB0C219CA802F012FE40F2DC5000F0DDFC0C219CA802F0FE
:2078E0000AFE40F2DC5000F0D5FC0C219CA802F002FEDFF8CC0600210180FAF7D0FF3EE3D2
:207900000021002002F0C6FEDFF8BC06008864281CD3DFF8B80600210180DFF8B4064FF6C7
:20792000FF710180DFF868064FF6FF7101801EE09C7E0020A07E0020F06E0020300900208E
:20794000A07F00209E7F0020347C0020DFF8480600880A2190FBF1F201FB1200002806D188
:20796000DFF864060088401CDFF85C160880DFF8640600884FF6FF71884231D1DFF81806D2
:207980000088322190FBF1F201FB1200002827D14FF48072002104A802F064FE55208DF820
:2079A000100000208DF8110004208DF81200A0208DF813009DF811009DF8121011EB002174
:2079C00089B204A8FAF7E8FC8DF814009DF811009DF8121011EB0020411C04A802F08BFD56
:2079E000DFF8F40500884FF6FF71884250D1DFF8A80500880A2190FBF1F201FB12000028B4
:207A000046D14FF48072002104A802F02BFE55208DF81000002401222F21DFF8C00502F003
:207A200021FE01220021DFF8B80502F01BFE08E0E4B204A82018E4B2DFF8A815615C017189
:207A4000641CE4B2DFF89C05205C2F28F0D100208DF81100201D8DF81200A1208DF8130021
:207A60009DF811009DF8121011EB002189B204A8FAF792FCE4B204A9611808719DF811004B
:207A80009DF8121011EB0020411C04A802F033FDDFF8540500884FF6FF71884264D1DFF8A5
:207AA000F80400880A2190FBF1F201FB120000285AD14FF48072002104A802F0D3FD55200F
:207AC0008DF810000024002501220021DFF81C0502F0C8FDDFF8180505F01CF90400E4B23D
:207AE0002200DFF80C1505A803F055FAE4B204A820180021417101220021DFF8F80402F027
:207B0000B1FDDFF8F40405F005F90500EDB22A00DFF8E414E4B204A82018401D03F03BFA59
:207B200000208DF811002819401D8DF81200A2208DF81300E4B2EDB2281904A944189DF8EC
:207B400011009DF8121011EB002189B204A8FAF723FC60719DF811009DF8121011EB0020FF
:207B6000411C04A802F0C7FCDFF8900400884FF6FF71884260D1DFF8200400880A2190FB6B
:207B8000F1F201FB1200002856D14FF48072002104A802F067FD55208DF8100000250024FA
:207BA00001222F21DFF8340402F05CFD01220021DFF82C0402F056FD05E000BFF56E002041
:207BC0000000C8426D1CEDB2DFF81804285C2F28F8D1EDB2DFF80C042818401C05F09AF833
:207BE0000400E4B22200EDB2DFF8F8032818411C05A803F0D0F900208DF81100201D8DF8DA
:207C00001200A3208DF813009DF811009DF8121011EB002189B204A8FAF7BEFBE4B204A9A9
:207C2000611808719DF811009DF8121011EB0020411C04A802F05FFCDFF8C40300884FF618
:207C4000FF7188426CD1D4480088022190FBF1F202FB1102002A63D14FF48072002104A808
:207C600002F000FD55208DF8100000208DF8110009208DF81200A4208DF8130001208DF893
:207C80001400E048008880B2000A8DF81500DD4800888DF816000020DB490988491C0800C0
:207CA00080B2010A8DF817108DF818009DF811009DF8121011EB002189B204A8FAF76CFB85
:207CC0008DF81900D1480088CF490988491C88420FD09DF811009DF8121011EB0020411CD8
:207CE00004A802F008FCC8480088401CC749088016E0C748007801280DD3C5480021017031
:207D00009DF811009DF8121011EB0020411C04A802F0F1FB04E0BE480078401CBC490870C8
:207D2000BC4800884FF6FF71884240F028819A480088142190FBF1F201FB1200002840F0EC
:207D40001E814FF48072002104A802F08BFC55208DF8100000208DF8110004208DF812008E
:207D6000AF208DF813009DF811009DF8121011EB002189B204A8FAF70FFB8DF814009DF812
:207D800011009DF8121011EB0020411C04A802F0B2FBA14800884FF6FF71884240F0E480D3
:207DA0009E4800210180002418E04FF480720021D0A802F057FC4FF48073D0AAA4B24FF4C3
:207DC000807000FB04F010F58051022004F04BFA4FF48071D0A802F025FF641CA4B2904823
:207DE0000068801EB4EB102FDFD3A4B24FF4807000FB04F08A490968891E884227D24FF484
:207E000080720021D0A802F02DFC85480068801EA4B24FF4807101FB04F1431A9BB2D0AA4A
:207E2000A4B24FF4807000FB04F010F58051022004F019FA7A480068801EA4B24FF4807179
:207E400001FB04F1411A89B2D0A802F0EBFE4FF480720021D0A802F005FC0223D0AA704830
:207E6000006800F6FE71022004F0FDF96B4800889DF841139DF8402312EB0121884261D1F2
:207E800000A868490A680260042300AA0021022004F003FA62480068801E000E8DF800006D
:207EA0005F480068801E000C8DF801005C480068801E000A8DF8020059480068801E8DF81C
:207EC0000300042300AA0421022004F0E6F954480068801EC043000E8DF80000504800687C
:207EE000801EC043000C8DF801004D480068801EC043000A8DF8020049480068801EC04386
:207F00008DF80300042300AA0821022004F0C5F91E480021018003221C495D2001F0F4FA1D
:207F20000020ADF804003A2101A803F03BF8BDF8040016490988884203D03A21134803F05F
:207F400050F8FEE71648022101702048002101803048002101801E484FF6FF7101800C48EE
:207F60004FF6FF7101800AE018480021018018484FF6FF71018006484FF6FF7101800DF2C6
:207F8000B44DBDE8F08F00008A6F00205E7F0020727F0020867F00208A7F0020308000088F
:207FA00030800020547F0020527F002098760020567F0020587F002044800008647600202D
:207FC0005A7F002068800008B27F0020687F0020AE7F00204E090020A27F00200B730020BD
:207FE0000C730020A8720020A47F0020C4760020B0760020DC760020C8760020A67F0020B0
:20800000A87F00206E7F0020707F0020B47F00203A800020AA7F0020AC7F00206A7F002033
:20802000A47E00207C800008253036640000000056312E3030332D30322D313730333131DA
:208040000000000061646D696E2C41542B43495053434F4E543D0000534820584420414390
:2080600020504F4C4500000061646D696E2C41542B43495245534554000000005A5A5A5A44
:2080800010B4B84A002306210024230002E002F20C025B1C9BB2062B05D21478A4B280B2C5
:2080A0008442F4D11900080080B210BC704710B4AD4A002304210024230001E010325B1C7B
:2080C0009BB2042B05D21478A4B280B28442F5D11900080080B210BC704738B5A14C0020DD
:2080E000ADF8000000250020050008E000AB0022A168606804F02EFE04F20C046D1CADB2FD
:20810000062DF3D3002000F0A1F831BD38B5964C0020ADF8000000250020050008E000AB5E
:20812000227B92B2A168606804F084FF10346D1CADB2042DF3D331BD1CB50C0000218DF882
:20814000041080B2FFF7B3FF01A9009100230A22210080B2844C14EB0010406805F087F859
:208160009DF80400002802D14FF6FF7000E0002016BD1CB50C0000218DF8041080B2FFF725
:2081800096FF01A9009110230A22210080B2764C14EB0010406805F06AF89DF804000028CC
:2081A00002D14FF6FF7000E0002016BD30B585B00C00150000218DF8081080B2FFF777FFCE
:2081C00002A9019103A900910A230022ADB2290080B2654D15EB0010406804F069FF2060D6
:2081E0009DF80800002802D14FF6FF7000E0002005B030BD30B583B000228DF8042089B273
:208200004FF47A725143594A1268B1FBF2F480B2FFF736FF010089B2062901D1002014E03E
:2082200001A9009100230022210080B20C244D4D04FB0050406804F0C0FD9DF80400002838
:2082400002D14FF6FF7000E000203EBD10B582B000218DF8001080B2FFF712FF010089B27A
:20826000062901D1002011E000AA002180B20C233C4C03FB0040406804F059FE9DF8000072
:20828000002802D14FF6FF7000E0002016BD4FF6FF70704780B500218DF8001000AA00213B
:2082A00080B205F069F89DF80000002802D14FF6FF7000E0002002BD30B58BB0002409A83E
:2082C00005F0A0F9FFF709FFFFF720FF0020040040E009A8089003200790002006900020E0
:2082E0000590A4B228201E4900FB0410008C0490A4B228201A4900FB0410C0690390A4B293
:208300002820174900FB041080690290A4B22820134900FB041040690190A4B228201049F1
:2083200000FB0410007C00900023A4B228200C4900FB0410C268A4B22820094900FB0410D4
:208340008168A4B22820064D00FB0450406805F013FE641CA4B2072CBBD30BB030BD000007
:208360005003002090070020D80700200836010880B500A805F0F1FA01BD50F8041B61B199
:2083800050F8042BD30744BFA9F101039A18002342F8043B091FFAD1EFE7704738B5DFF859
:2083A000EC55002404E0A868804705F21C05641CA4B22E2CF7D30020DFF8D4150880DFF84C
:2083C000D415088006F0E3FA31BD38B50400DFF8BC5500F02BF8A4B2FF2C0CD1DFF8B8058D
:2083E000007878280BD2DFF8B0050078401CDFF8A815087003E0DFF8A0050021017000200B
:2084000002E005F21C05401C80B22E280CD2DFF8801509882A889142F3D1200080B2E968B7
:2084200088474FF6FF7000E0002032BD70B50024DFF85855DFF858050088DFF8581509886C
:20844000884223D0002602E005F21C05761CB6B22E2E1BD2DFF8380500882988884202D112
:2084600028698047641CDFF82C0500882988884202D168698047641CE4B2022CE4D3DFF8DC
:208480001405DFF80C1509880180FFE770BD10B5DFF8F844FFF7CAFFDFF8FC040078782820
:2084A00039D3DFF8EC0400880E2834D0DFF8E00400880F282FD0DFF8D804008810282AD041
:2084C000DFF8CC040088002825D0DFF8C4040088012820D0DFF8B80400880C281BD0DFF8FF
:2084E000680600780E2804D1DFF8A4040E2101800DE0DFF8540600780F2804D1DFF890044F
:208500000F21018003E0DFF8880400210180DFF8880400210170002002E004F21C04401C59
:2085200080B22E280AD2DFF86814098822889142F3D1A06980474FF6FF7000E0002010BD61
:20854000DFF84C1408807047DFF844040088704710B584B0040008000A280DD20A2200A95C
:2085600006F031FB302020702E2060703020A0709DF80000E07005E1B0F10A015A290ED2A1
:208580000A2200A906F01FFB302020702E2060709DF80000A0709DF80100E070F2E0B0F1FA
:2085A00064014FF4617291420FD20A2200A906F00AFB9DF8000020702E2060709DF80100E3
:2085C000A0709DF80200E070DCE0A0F2E83142F22832914212D20A2200A906F0F4FA9DF8AA
:2085E000000020709DF8010060702E20A0709DF80200E0709DF803002071C3E042F21071BF
:20860000411ADFF8A026914215D20A2200A906F0DAFA9DF8000020709DF8010060709DF8E9
:208620000200A0702E20E0709DF8030020719DF804006071A6E0DFF87016411ADFF86C2650
:20864000914218D20A2200A906F0BDFA9DF8000020709DF8010060709DF80200A0709DF814
:208660000300E0702E2020719DF8040060719DF80500A07186E0DFF83816411ADFF834269C
:2086800091421BD20A2200A906F09DFA9DF8000020709DF8010060709DF80200A0709DF8F1
:2086A0000300E0709DF8040020712E2060719DF80500A0719DF80600E07163E0DFF8F81560
:2086C000411ADFF8F82591421BD20A2200A906F07AFA9DF8000020709DF8010060709DF82C
:2086E0000200A0709DF80300E0709DF8040020719DF8050060712E20A0719DF80600E071A0
:2087000040E0DFF8BC15411ADFF8B825914219D20A2200A906F057FA9DF8000020709DF8EE
:20872000010060709DF80200A0709DF80300E0709DF8040020719DF8050060719DF80600A9
:20874000A0711FE0DFF8801588421BD30A2200A906F039FA9DF8000020709DF8010060705C
:208760009DF80200A0709DF80300E0709DF8040020719DF8050060719DF80600A0719DF894
:208780000700E0711FBD80B5022200A91F2000F096FE01220DF102011E2000F090FEDFF829
:2087A0002C050078012818D19DF80000012803D09DF80000022805D1BDF802004FF6FF716C
:2087C00088420AD10221002006F079FA0020FFF7B7FEDFF8FC040121018001BD80B50020F0
:2087E0000090042200A92B2000F069FE009843F2F301084242D0DFF8500300780E283DD076
:20880000DFF8440300780F2838D0DFF83C03007806281DD0DFF8300300780A2818D0DFF867
:2088200028030078072813D0DFF81C03007808280ED0DFF814030078092809D0DFF80803B5
:2088400000780B2804D0DFF8000300780C280DD1DFF880044FF6FF7101800120FFF770FE1F
:20886000DFF86C044FF4FA71018007E00120FFF767FEDFF85C044FF4FA7101800098C0045D
:2088800003D5DFF8AC0A01210170DFF8A40A0078012809D0009850F400500090042200A956
:2088A0002B2000F031FE08E0009830F400500090042200A92B2000F027FE01BDDFF81804EA
:2088C00000210170DFF8140400210170DFF8640A002101707047DFF80004012101707047D2
:2088E000DFF8F803022101707047DFF8F003012101707047DFF8E403002101707047DFF869
:20890000340A022101707047DFF8280A002101707047002008E0C0B23E21DFF81C2A01FB8A
:20892000002100228A87401CC0B20A28F3D37047002008E0C0B21221DFF8002A01FB00219B
:2089400000224A74401CC0B20C28F3D3704770B504000D00160028222021DFF8E40901F02C
:2089600081FEF6B232002900DFF8D40902F013FB01220021F6B2DFF8C809301801F072FE84
:208980002100DFF8BC0906F03BFA70BDE08C0008487F00204A7F00201580002000B591B0D3
:2089A0000020009001A801F05AF804A9002000F0D6FF9DF81100012802D1002006F03AFC9B
:2089C000DFF8800903210170DFF87809AA2101710822DFF87419DFF8740902F0DCFA102231
:2089E000DFF86C19DFF86C0902F0D5FA2022DFF86819DFF8680902F0CEFADFF84809DFF873
:208A00006019097880F89910DFF8380955210172DFF83009DFF84C1909684163DFF84409B5
:208A200000680D9906F088FDDFF81819886305A9DFF8340901F021FA01A9DFF8300901F041
:208A40001CFADFF800090B2180F8981000AA01A905A801F0CFF8DFF8EC080099C16403226D
:208A6000DFF80C19222000F02AFD0022DFF80419062000F024FD0022DFF8FC18002000F037
:208A80001EFD0022DFF8F418012000F018FD0022DFF8EC18022000F012FD0022DFF8E4187D
:208AA000032000F00CFD0022DFF8DC18042000F006FD0022DFF8D418072000F000FD00227B
:208AC000DFF8CC18082000F0FAFC0022DFF8C418092000F0F4FC0022DFF8BC180A2000F008
:208AE000EEFC0022DFF8B4180C2000F0E8FC0022DFF8AC18112000F0E2FC0022DFF8A41856
:208B00000D2000F0DCFC0022DFF89C18122000F0D6FC0022DFF894180E2000F0D0FC00220E
:208B2000DFF88C18132000F0CAFC0022DFF884180F2000F0C4FC0022DFF87C18142000F0AC
:208B4000BEFC11B000BD0000640900202DE9F04184B004000D005FF000080026002700A878
:208B600000F07DFFBDF80000642190FBF1F201FB12004F499DF8022042F210735A4301FB34
:208B800000209DF80310642202FB01009DF80510081880469DF80500401C00FB08F8DFF831
:208BA0001C0810EB08000600DFF8140810EB080007000A20B6FBF0F100FB11603030207073
:208BC0000A20B6FBF0F00A21B0FBF1F201FB1200303060706420B6FBF0F00A21B0FBF1F215
:208BE00001FB12003030A0704FF47A70B6FBF0F00A21B0FBF1F201FB12003030E07042F28E
:208C00001070B6FBF0F00A21B0FBF1F201FB1200303020712448B6FBF0F00A21B0FBF1F2D5
:208C200001FB1200303060710A20B7FBF0F100FB1170303028700A20B7FBF0F00A21B0FB32
:208C4000F1F201FB1200303068706420B7FBF0F00A21B0FBF1F201FB12003030A8704FF453
:208C60007A70B7FBF0F00A21B0FBF1F201FB12003030E87042F21070B7FBF0F00A21B0FBDD
:208C8000F1F201FB1200303028710748B7FBF0F00A21B0FBF1F201FB120030306871BDE864
:208CA000FF810000905F0100A0860100A0BB0D0040420F004054890080969800804A5D052D
:208CC00000E1F50500E9A43500CA9A3B25800020420900209A7F00201D8000201E80002074
:208CE000000000008C7800207FE60008C3E600088FE900088FEA000875E7000801000000CC
:208D0000A0780020093702083B370208955E0208255F02087938020802000000B4780020C1
:208D2000DD8403081F850308AD8B0308458C03087785030803000000C8780020D9E70208C5
:208D40001BE802083FF20208B7F20208B1EB020804000000DC78002049DA03088DDA03085A
:208D600083DD0308B7DD0308B7DA030805000000F078002015F7030847F7030891F90308CB
:208D8000DDF9030867F7030806000000047900204DEA030885EA03083FED0308C5ED030836
:208DA0005BEB0308070000002C79002035B3030877B3030885B80308C7B8030839B60308A2
:208DC000080000004079002025A7030867A703088DAC0308CFAC030841AA030809000000F9
:208DE000547900201D9A03085F9A0308E79F030843A00308619C03080A000000187900207E
:208E000019F403084BF40308ABF6030811F70308E1F403080B00000068790020A5A00308F5
:208E2000E7A0030871A60308C3A60308E9A203080C0000007C790020B5C80308F9C80308FF
:208E4000ADCC03080BCD03084DC903080D0000009079002059D603089BD60308E9D90308D1
:208E600045DA0308D9D603080E000000A47900203D0502086F050208F52D0208552F02083F
:208E8000AD0602080F000000B8790020C1D40108F3D401080D0402085304020831D60108BB
:208EA00010000000CC790020C9C303080BC4030833C80308B1C80308BBC4030811000000A7
:208EC000E07900200575030847750308DF790308BD7B03087375030812000000F479002095
:208EE00065D20308A9D2030893D50308C9D50308D9D3030813000000087A002005FA030818
:208F000037FA030855FC0308A9FC0308BFFA030814000000947A002011060408430604088B
:208F2000C307040801080408C3060408150000001C7A0020F9E103083DE2030859E503084E
:208F4000ADE50308C5E2030816000000C4770020ED1803082F190308FD2003081522030884
:208F6000C11B030817000000EC77002085C40208C7C40208D1CF020839D10208F1C9020806
:208F800018000000007800203DFE02087FFE020881070308E1080308270103081900000082
:208FA000147800204DD102088FD10208FDDD02087DDF0208ADD502081A00000028780020C3
:208FC000292203086B22030879290308D52A0308132603081B0000003C78002095CD03084C
:208FE000D7CD0308C3D103084DD20308AFCF03081C00000050780020A5BE0308E7BE03084E
:20900000BFC20308B9C303085BC003081D000000647800201DF103084FF103089FF30308FD
:20902000FDF3030891F203081E0000009C7700202DDE03086FDE030857E10308E9E10308D0
:2090400045DF03081F000000807A0020B5010408E701040881030408CD0304086702040811
:2090600020000000B0770020D97C03081B7D030899830308C7830308897D030821000000D8
:20908000D8770020C9ED0308FBED030899F00308D9F0030835EE030822000000307A00202B
:2090A0006D520308AF520308E3590308195B03085756030823000000447A002029B903086E
:2090C0006BB9030835BD03088DBE0308EBBA030824000000587A002041FF030873FF030880
:2090E00059010408B1010408FBFF03082500000078780020597302089B730208178502087E
:2091000001870208D97602082600000010770020955F0208D75F02085371020845730208C9
:20912000156302082700000024770020158702084D870208A3980208959A0208658A0208D0
:209140002800000038770020591D0408911D0408951D0408971D0408931D04082900000079
:209160004C7700205D2B03089F2B030891320308E3330308012C03082A0000006C7A00204D
:20918000ADFC0308DFFC0308EFFE03083DFF030891FD03082B00000060770020110404081A
:2091A00043040408B7050408050604085F0404082C000000747700203DF302087FF3020821
:2091C000A9FC020821FE020859F502082D00000088770020498C03088B8C030891920308E3
:2091E00021930308418D030800B585B000200190002000900020039000200290002271494B
:20920000672000F05CF96F4800686F4906F006FA2CD86C4800686D4903F002FD26D2694844
:20922000006806F00DFA5FF03332694B06F030FA06F000FB0090009802900098654903F05D
:20924000EFFC06D200985FF0804106F03BFB019009E0009806F0F4F95F4A604B06F018FA26
:2092600006F0E8FA0190019803903AE055480068564906F0D3F934D852480068584903F037
:20928000CFFC2ED24F480068564906F01BFB06F0D7F90022544B06F0FBF906F0CBFA00909D
:2092A0000098524906F0BAF901D851480090009802900098474903F0B3FC06D200985FF01D
:2092C000804106F0FFFA019009E0009806F0B8F9414A424B06F0DCF906F0ACFA019001987C
:2092E0000390352101A801F07CFE002201A9342000F00AF9362100A801F073FE002200A932
:20930000352000F001F9372103A801F06AFE002203A9362000F0F8F8382102A801F061FE5B
:20932000002202A9372000F0EFF805B000BD0000720900201F800020704E002068040020FC
:209340007875002040680020A1740020496800208A74002059680020A9740020DE68002090
:20936000A0740020607400207C680020846800207068002090680020946800209868002069
:209380009C680020A0680020A4680020A8680020AC680020B0680020B4680020B86800203D
:2093A000C8680020BC680020CC680020C0680020D0680020C4680020D4680020D038030072
:2093C00040E20100547E0020000020410100AA423333E33F0100A0419A9999999999F13FF9
:2093E0000100B442000080C20000044001007C4200007C4201000200030004001300000056
:20940000050006000A0000001400220023002A0007000800090000000B000C001600170058
:20942000180019001B001C001D001E00200021002500260027002800290000000D000E006A
:209440000F0000001000110010B4002304E00C780470401C491C5B1C9342F8D310BC7047BE
:209460000021C0B2002812D0022814D011D3042815D012D3062810D00DD3082811D00ED387
:209480000A2812D00FD30C2813D010D313E0042112E0022110E001210EE002210CE004217B
:2094A0000AE0322108E00C2106E0082104E0022102E0102100E00021080080B2704770B51A
:2094C00006000C0010000025B6B2224911EBC6018978C0B2814214D1B6B21E4931F8361056
:2094E000B6B2B1420DD1C0B2FFF7BAFF0500EDB22A00B6B2174810EBC60041682000FFF7FD
:20950000A3FF2800C0B270BD70B505000E0010000024ADB20F4911EBC5018978C0B28142C7
:2095200014D1ADB20B4931F83510ADB2A9420DD1C0B2FFF795FF0400E4B222003100ADB2B5
:20954000044810EBC5004068FFF77EFF2000C0B270BD0000000000202DE9F0439BB00D0064
:2095600016001F0000245FF000085FF000092A00D2B20DA980B2FFF7A2FF80463A00D2B232
:2095800000A9300080B2FFF79AFF81461FFA88F81FFA89F9C84503D003242000C0B2FCE0C1
:2095A0001FFA88F8424600A90DA801F0C3FC002800F0F180EDB2002D0FD0022D28D019D335
:2095C000042D5DD040D3062D4CD02FD3082D6FD062D3092D00F08880DDE000980D9903F004
:2095E0001FFB03D201200400C0B202E002200400C0B2D0E0BDF80000BDF83410884203D26E
:2096000001200400C0B202E002200400C0B2C2E09DF800009DF83410884203D20120040065
:20962000C0B202E002200400C0B2B4E09DF900009DF93410884203DA01200400C0B202E01A
:2096400002200400C0B2A6E0BDF80000BDF83410884203D201200400C0B202E00220040000
:20966000C0B298E0BDF90000BDF93410884203DA01200400C0B202E002200400C0B28AE02E
:2096800000980D99884203D201200400C0B202E002200400C0B27EE000980D99884203DA99
:2096A00001200400C0B202E002200400C0B272E000200021080000E0401CC0B2322812D212
:2096C000C0B200A9415CC0B20DAA825C914201D2012408E0C0B20DA9415CC0B200AA825C59
:2096E0009142E9D2022456E00DA800A90A8803889A4201D201244DE002880B889A4201D238
:20970000022447E08A7883789A4201D2012441E082788B789A4201D202243BE0CA78C378A0
:209720009A4201D2012435E0C278CB789A4201D202242FE04A7943799A4201D2012429E083
:2097400042794B799A4201D2022423E08A7983799A4201D201241DE082798B799A4201D234
:20976000022417E0CA79C3799A4201D2012411E0C279CB799A4201D202240BE08A6883686C
:209780009A4201D2012405E080688968884201D20224FFE7FFE72000C0B21BB0BDE8F08333
:2097A000C0B2012802D37FF0040007E0C0B234218D4A01FB00200021417000207047C0B20A
:2097C000012802D37FF004000EE0C0B23422864B02FB00320968D161C0B23421824A01FB30
:2097E0000020002181700020704700B502000B00D2B2012A02D37FF004001CE0186859686A
:2098000005F00CFF01D858681860D2B23420764900FB021001218170D2B23420724900FBF2
:2098200002105968C161D2B234206F4900FB021019680162002000BDC0B2012802D37FF0F6
:20984000040015E0C0B23422674B02FB003202239370C0B23422644B02FB00324B68D361B1
:20986000C0B23422604B02FB00300968C162002070473EB504000D00E4B2012C02D37FF0D2
:20988000040029E000A800F0EAF84FF6FF71884220D1E4B23420544900FB04100321817026
:2098A000E4B23420504900FB041003218170E4B234204D4900FB041010300ECD0EC00C3D40
:2098C0000C38E4B23420484900FB0410E968C161002001E07FF005003EBDC0B23421424A84
:2098E00001FB0020022141700020704780B501000020C9B234223C4B02FB01325278022ACD
:2099000007D0C9B23422384B02FB01325278032A23D1C9B23420344A00FB01208078002878
:2099200005D0022808D011D303280AD013E00800C0B205F08FFC10E00800C0B205F028FDF6
:209940000BE00800C0B205F085FD06E00800C0B205F0B7FC01E07FF0050040B202BD10B558
:209960000B003422C0B234211F4C01FB0041180001F011FB002010BDC0B234211A4A01FBEE
:2099800000200521417000207047C0B23421164A01FB00200121417000207047C0B2342145
:2099A000114A01FB00200621417000207047C0B234210D4A01FB002000214170002070479E
:2099C00010B5C0B23421084A01FB002100224A7034220021C0B23423034C03FB004000F0F3
:2099E00041FE002010BD0000DC74002080B505F0ABFF05F0CEFFDFF8A0084FF6FF71018080
:209A0000DFF89408008802BD00B583B0DFF8881809884FF6FF7291421FD10188ADF80010E5
:209A200081788DF80210C1788DF8031001798DF8041041798DF8051081798DF80610C07990
:209A40008DF8070005F0A6FFDDE9000105F0C4FF05F09FFF4FF6FF7000E000200EBD1CB57E
:209A60000400DFF8340800884FF6FF7188421AD100A806F059F8BDF8000020809DF8020002
:209A8000A0709DF80300E0709DF8040020719DF8050060719DF80600A0719DF80700E071A0
:209AA0004FF6FF7000E0002016BD0A8803889A4201D2022042E002880B889A4201D2012022
:209AC0003CE08A7883789A4201D2022036E082788B789A4201D2012030E0CA78C3789A4250
:209AE00001D202202AE0C278CB789A4201D2012024E04A7943799A4201D202201EE042790D
:209B00004B799A4201D2012018E08A7983799A4201D2022012E082798B799A4201D2012028
:209B20000CE0CA79C3799A4201D2022006E0C079C979884201D2012000E0002070470A7891
:209B400003789A4201D2022012E002780B789A4201D201200CE04A7843789A4201D20220C0
:209B600006E040784978884201D2012000E00020704770B504000E001500002028803100CC
:209B80002000FFF7DCFF01280CD130782178401A3C21727801FB00206178401A28804FF6B0
:209BA000FF700BE031002000FFF7C9FF002804D1002028804FF6FF7000E0002070BD4A79D3
:209BC00002708A794270CA79827089684160704710B584B0040000A8FFF741FF002801D10B
:209BE000002005E000A92000FFF7E9FF4FF6FF7004B010BD2DE9F04104000D0016001C27D3
:209C00005FF01E080020306029002000FFF74DFF012873D12088401C2988884204DBA078B1
:209C2000401CA978884201DA002073E028882188491C884207D1A078401CA9780C31884293
:209C400001DA002066E028884FF4C87190FBF1F201FB120000280FD02888642190FBF1F271
:209C600001FB1200002809D02888042190FBF1F202FB1102002A01D11D2700E01C27A07807
:209C8000012811D0A07803280ED0A07805280BD0A078072808D0A078082805D0A0780A28F3
:209CA00002D0A0780C2802D15FF01F0806E0A078022801D1B84601E05FF01E082888218896
:209CC000401A0C21AA7801FB0020A178401A5FFA88F8E97808FB0010E178401A18216A7930
:209CE00001FB00206179401A3C21AA7901FB0020A179401A30604FF6FF700BE0290020008C
:209D0000FFF7D3FE002804D1002030604FF6FF7000E00020BDE8F0812DE9F04104000D00AD
:209D200016001C275FF01E080020306029002000FFF7BBFE012879D12088401C29888842BB
:209D400004DBA078401CA978884201DA002079E028882188491C884207D1A078401CA9787C
:209D60000C31884201DA00206CE028884FF4C87190FBF1F201FB120000280FD028886421B1
:209D800090FBF1F201FB1200002809D02888042190FBF1F202FB1102002A01D11D2700E0D3
:209DA0001C27A078012811D0A07803280ED0A07805280BD0A078072808D0A078082805D0C1
:209DC000A0780A2802D0A0780C2802D15FF01F0806E0A078022801D1B84601E05FF01E0884
:209DE00028882188401A0C21AA7801FB0020A178401A5FFA88F8E97808FB0010E178401AD2
:209E000018216A7901FB00206179401A3C21AA7901FB0020A179401A3C21EA7901FB0020EA
:209E2000E179401A30604FF6FF700BE029002000FFF73BFE002804D1002030604FF6FF7066
:209E400000E00020BDE8F08110B584B0040000A8FFF705FEBDF8000020809DF80200A07052
:209E60009DF80300E0709DF8050020719DF8060060719DF80700A0711FBD0A8802808A78C4
:209E80008270CA78C2704A7902718A794271C97981717047F0B4002301888478C278457941
:209EA0008679C079A1F2B277BFB2822F5CD2631EDBB20C2B58D2531EDBB21F2B54D2EDB2E2
:209EC000182D51D2F6B23C2E4ED2C0B23C284BD2E4B2042C08D0E4B2062C05D0E4B2092CEF
:209EE00002D0E4B20B2C07D1D2B21F2A01D3002330E04FF6FF732DE0E4B2022C28D189B25B
:209F00004FF4C87091FBF0F300FB131000280FD089B2642091FBF0F300FB131000280FD0DF
:209F200089B2042091FBF0F303FB1013002B07D1D2B21E2A01D300230CE04FF6FF7309E0E0
:209F4000D2B21D2A01D3002304E04FF6FF7301E04FF6FF734FF6FF709BB2834202D14FF62E
:209F6000FF7002E0002000E00020F0BC704770B504000D0000260A222900208804F0DEFDE5
:209F80000A22DFF81813A07804F0D8FD0A22DFF81013E07804F0D2FD2D202871DFF8FC02B6
:209FA00000786871DFF8F4024078A8712D20E871DFF8EC0200782872DFF8E40240786872E6
:209FC0002020A8722020E8720A22DFF8D812207904F0B4FD0A22DFF8D012607904F0AEFD05
:209FE0000A22DFF8C812A07904F0A8FDDFF8B40200782873DFF8AC02407868733A20A873A5
:20A00000DFF8A4020078E873DFF89C02407828743A206874DFF894020078A874DFF88C028B
:20A020004078E874002028750020060007E0B6B2132E03D1A87CE8743020A874761CB6B2DF
:20A04000142E23D2B6B2705D0028F7D1B6B2062E04D16879A87130206871EFE7B6B2092E9B
:20A0600004D1287A687230202872E7E7B6B20D2E04D1287B687330202873DFE7B6B2102E8A
:20A08000D5D1E87B28743020E873D7E770BD70B504000D0000260A222900208804F04EFDED
:20A0A0000A228349A07804F049FD0A228149E07804F044FD2D2028717D48007868717C4813
:20A0C0004078A8712D20E8717A48007828727948407868722020A8722020E8720A22764903
:20A0E000607904F02BFD0A227449A07904F026FD0A227349E07904F021FD6F480078287335
:20A100006D48407868733A20A8736C480078E8736A48407828743A20687469480078A8747A
:20A1200067484078E874002028750020060007E0B6B2132E03D1A87CE8743020A874761C97
:20A14000B6B2142E23D2B6B2705D0028F7D1B6B2062E04D16879A87130206871EFE7B6B269
:20A16000092E04D1287A687230202872E7E7B6B20D2E04D1287B687330202873DFE7B6B290
:20A18000102ED5D1E87B28743020E873D7E770BD3EB50400002500A8FFF761FC0A222100E2
:20A1A000BDF8000004F0CAFC0A2246499DF8020004F0C4FC0A2244499DF8030004F0BEFC2B
:20A1C0004048007820713F48407860713E480078A0713D484078E071202020720A223B49BF
:20A1E0009DF8050004F0AAFC0A2239499DF8060004F0A4FC0A2237499DF8070004F09EFC78
:20A2000032480078607231484078A0723A20E0722F48007820732E48407860733A20A0739B
:20A220002C480078E0732B4840782074002060740020050007E0ADB2102D03D1E07B2074C1
:20A240003020E0736D1CADB2112D23D2ADB2285D0028F7D1ADB2052D04D12079607130204C
:20A260002071EFE7ADB2072D04D1A079E0713020A071E7E7ADB20A2D04D1607AA0723020CF
:20A280006072DFE7ADB20D2DD5D1207B607330202073D7E737BD00001E7F0020267F002062
:20A2A000287F0020207F0020227F0020247F0020307F0020327F00202A7F00202C7F002060
:20A2C0002E7F00203A7F00203C7F0020347F0020367F0020387F002038B504000D00200060
:20A2E000FFF7BDFBA07969780818A0716079297808186071A0793C2805D3A0793C38A07127
:20A300006079401C60716079182866D3607918386071E078401CE070A078012811D0A078AD
:20A3200003280ED0A07805280BD0A078072808D0A078082805D0A0780A2802D0A0780C2850
:20A3400009D1E07820283FD3E0781F38E070A078401CA07038E0A07802282CD120884FF4AC
:20A36000C87190FBF1F201FB120000280FD02088642190FBF1F201FB1200002811D02088C7
:20A38000042190FBF1F202FB1102002A09D1E0781E2819D3E0781D38E070A078401CA0700B
:20A3A00012E0E0781D280FD3E0781C38E070A078401CA07008E0E0781F2805D3E0781E389F
:20A3C000E070A078401CA070A0780D2805D3A0780C38A0702088401C208031BD38B5C0B227
:20A3E000032812D201230122C0B20321204C01FB00418978C0B203241D4D04FB00504078BD
:20A4000005F010FC4FF6FF7000E0002032BD10B5C0B2032811D20122C0B20321144B01FB3F
:20A4200000318978C0B20323114C03FB0040407805F079FC4FF6FF7000E0002010BD10B54F
:20A44000C0B2032811D20022C0B20321084B01FB00318978C0B20323054C03FB0040407864
:20A4600005F061FC4FF6FF7000E0002010BD0000F408002080B5354A35480088354941185D
:20A48000012005F0A3FD3248008840F22621884204D22F480088401C2D4908802C48008896
:20A4A00040F22621884202D129480021018001BD7047704780B52648002101802348002176
:20A4C000018001200090002308225FF4E131012005F030FD002801D100200BE01E4B1F4A7E
:20A4E0001F49012005F084FD002801D1002001E04FF6FF7002BD10B50C00220001000120DA
:20A5000005F04DFD002801D1002000E0200010BD0E48002101800E48002101807047114815
:20A520000088704780B200280BD00E4800884FF47A71884208D20B480088401C09490880E6
:20A5400002E008480021018070470000FE7E0020FC7E0020DC500020B3A40008B1A4000832
:20A5600075A4000834090020FF2212EAD05C1DBF12EAD153944593422BE09C44D30780EA3B
:20A5800001021A4043EA002043EA0121A1FB0030410038BF40007CF17F010BDBFE294ADA60
:20A5A0005B0842EAC15153EA006373F1004C51EB10207047D1F1080CDCF120012FDB5B0856
:20A5C00010FA01F10B4373F1004120FA0CF05041704794451CBF02EAD153934280EA010228
:20A5E00002F000421DD0400019D0490017D05BB9634514D00902B1FA81F39940BCEB030C88
:20A60000C00140F00040C1E70002B0FA80FC10FA0CF0B3EB0C0CC90141F00041B6E7100094
:20A62000704740000AD0490008D010F1807F94BF11F1807F02E042F0FF407047D043704700
:20A6400040000DD2010E7F390AD4D1F11F0104D4C00140F00040C84070477FF00000704766
:20A660000020704710B5040010000A000100200005F0D0FC200010BD80B5C0B2012807D2A8
:20A68000C0B214210B4A01FB00200069804700E00A2002BD80B502000800D2B2012A07D2E2
:20A6A00080B2D2B21421034B01FB0231C968884701BD0000801E040838B504000020208019
:20A6C0001C2006F0E4FA05001C2006F0E0FA6560A0606068A1688161606800214161A0684E
:20A6E00000218161A0686168416131BD008870470088142802D14FF6FF7000E000207047B5
:20A700000088002802D14FF6FF7000E000207047F8B504000D00002600272800FFF7E8FF3B
:20A72000002807D02900002000F03BF8002801D1002035E0DFF83005FFF7D8FF0600DFF8C9
:20A74000280540688069002701E080697F1CBFB2B6B2B74206D2217802789142F5D14FF614
:20A76000FF701DE01C2006F092FA0600002E01D1002015E0207830700822A11CB01C00F0B9
:20A780000AFC68688069B06168688069466168687061686886612888401C28804FF6FF70C9
:20A7A000F2BD70B505000C002000FFF7A9FF002801D0002037E02000FFF798FF002D10D10B
:20A7C0002088401E2080A168A0684069A060A06800228261080006F082FB00214FF6FF70BC
:20A7E00021E061688E69002101E0B669491C814218DA2A7833789A42F7D12088401E2080C6
:20A80000A81CB11C082202F043FA7069B1698161B06971694161300006F061FB00264FF6F7
:20A82000FF7000E0002070BD70B4002314E0DBB2022493FBF4F455006D1EDBB2ED1A6D5CDB
:20A840005600761EDBB2F61A761816F8016C15EB0615303D25549B1CDBB2B3EB420FE6D37B
:20A8600070BC704730B4002315E0541EDBB2E41A645CE4B224093034DBB200F81340541ECB
:20A88000DBB2E41A645C14F00F043034DBB210EB43056C705B1CDBB29342E6D330BC704711
:20A8A000002200E0521CD2B28A420ED200230A2B01D300200BE04B1ED2B29B1A1B5C13F0A5
:20A8C0000F030A2BEEDB002001E04FF6FF707047002100E0491CC9B2062907D2C9B20A5C32
:20A8E000303AD2B20A2AF5D3002001E04FF6FF707047C0B2642190FBF1F201FB1200C0B21D
:20A900000A2190FBF1F10901C0B20A2290FBF2F302FB130001430800C0B270470021DFF80A
:20A920004C23B0FBF2F251EA0271DFF84023B0FBF2F302FB1302DFF83833B2FBF3F251EA80
:20A940000261DFF82C23B0FBF2F302FB1302DFF82433B2FBF3F251EA0251DFF81823B0FBC1
:20A96000F2F302FB130242F21073B2FBF3F251EA024142F21072B0FBF2F302FB13024FF47E
:20A980007A73B2FBF3F251EA02314FF47A72B0FBF2F302FB13026423B2FBF3F251EA022182
:20A9A0006422B0FBF2F302FB13020A23B2FBF3F251EA02110A22B0FBF2F302FB1302114340
:20A9C0000800704710B4002211E0D2B211F812301B01D2B21354D2B2135CD2B211EB420452
:20A9E000647814F00F042343D2B21354521CD2B2082AEAD310BC704730B400220EE0C9B240
:20AA00004B1ED2B29B1A1B5CC9B24C1ED2B2A41AD2B2155C2554D2B21354521CC9B202238F
:20AA200091FBF3F3D2B29A42E9DB30BC70472DE9F0438DB004000D0017001E0000A8342114
:20AA400002F05EF9F6B2032EC0F097803222002100A8FFF707FE3F68380006F0A3FC8449B4
:20AA600001FB00F884483900FFF77EFD8146404602F040F80100484604F05EFD06F092FC93
:20AA8000002800D5404203009846380006F08AFC020043460FF2382100A802F011F82900F1
:20AAA000EDB2072D00D30621002000E0401CC0B2F6B2B21E90423BDAC0B200AA825C2E2A4A
:20AAC000F4D1EDB2002D09D1C0B200A920224254C0B200A940182021417029E0C0B2C9B2BD
:20AAE0000A1800ABD21820235370C0B2C9B20A1800ABD21820239370C0B2C9B20A1800ABF5
:20AB0000D2182023D370C0B2C9B20A1800ABD21820231371C0B2C9B20A1800ABD218202373
:20AB20005371C0B2C9B2081800A9401820218171F6B200A8301810F8030C2E2805D1F6B28D
:20AB400000A83018202100F8031CF6B200A83018202100F8021CF6B200A83018202100F8ED
:20AB6000011C002005E0C0B2C0B200A9415C0155401CC0B2F6B2B042F5D30DB0BDE8F0832E
:20AB800030B4002308E0DBB25C5C14F00F043734DBB200F813405B1CDBB2D2B2934227D2D1
:20ABA000DBB25C5CE4B224090A2C09D2DBB210EB4304DBB25D5CEDB22D093035657008E070
:20ABC000DBB210EB4304DBB25D5CEDB22D0937356570DBB25C5C14F00F040A2CD3DADBB27E
:20ABE0005C5C14F00F043034DBB200F81340D2E730BC704710B400220BE092B2130A1202A8
:20AC0000DBB2047863400FF2D00434F813305A40401C0B00591E9BB2002BEED1100080B253
:20AC200010BC704710B415E0144A128892B2120A124B1B881B02114C2380104B1B88D2B2E1
:20AC4000047862400FF2900434F812205A400B4B1A80401C0A00511E92B2002AE4D1074812
:20AC6000008810BC70470000C47C00208096980040420F00A0860100002474496A7F002019
:20AC800010B5ADF5FE6D4FF40050002415E0A4B24FF4806000FB04F010F500504FF4806254
:20ACA000FBA906F0ADFB4FF48061FBA8FFF7A2FFA4B200A921F81400641CA4B2FD2CE6D310
:20ACC0004FF4FD7100A8FFF795FF0DF5FE6D10BD25642E253036640000002110422063308B
:20ACE0008440A550C660E770088129914AA16BB18CC1ADD1CEE1EFF131121002733252220C
:20AD0000B5529442F772D662399318837BB35AA3BDD39CC3FFF3DEE362244334200401144B
:20AD2000E664C774A44485546AA54BB528850995EEE5CFF5ACC58DD553367226111630068B
:20AD4000D776F6669556B4465BB77AA719973887DFF7FEE79DD7BCC7C448E5588668A778BB
:20AD60004008611802282338CCC9EDD98EE9AFF9488969990AA92BB9F55AD44AB77A966A0B
:20AD8000711A500A333A122AFDDBDCCBBFFB9EEB799B588B3BBB1AABA66C877CE44CC55C4B
:20ADA000222C033C600C411CAEED8FFDECCDCDDD2AAD0BBD688D499D977EB66ED55EF44E8B
:20ADC000133E322E511E700E9FFFBEEFDDDFFCCF1BBF3AAF599F788F8891A981CAB1EBA1F7
:20ADE0000CD12DC14EF16FE18010A100C230E3200450254046706760B9839893FBA3DAB30B
:20AE00003DC31CD37FE35EF3B1029012F322D2323542145277625672EAB5CBA5A89589854A
:20AE20006EF54FE52CD50DC5E234C324A01481046674476424540544DBA7FAB79987B8978A
:20AE40005FE77EF71DC73CD7D326F2369106B01657667676154634564CD96DC90EF92FE9BA
:20AE6000C899E9898AB9ABA94458654806782768C018E1088238A3287DCB5CDB3FEB1EFB0A
:20AE8000F98BD89BBBAB9ABB754A545A376A167AF10AD01AB32A923A2EFD0FED6CDD4DCD4A
:20AEA000AABD8BADE89DC98D267C076C645C454CA23C832CE01CC10C1FEF3EFF5DCF7CDF8A
:20AEC0009BAFBABFD98FF89F176E367E554E745E932EB23ED10EF01E80B506F09AFA02BDE6
:20AEE00070B504000D00160000210020FDF782F932002900200006F0A6FA0028F8D0002035
:20AF0000FDF7A4F94FF6FF7070BD70B504000D00160000210020FDF76DF93200290020005D
:20AF200006F07CFA0028F8D00020FDF78FF94FF6FF7070BD0300002013F0030F09D0521EB7
:20AF400022BF13F8010B11F801CBB0EB0C00F3D07047121F22BF53F8040B51F804CB6045DA
:20AF6000F7D0121D0AD200BA9CFA8CFCB0EB0C0038BF6FF0000088BF01207047521E22BFBA
:20AF800013F8010B11F801CBB0EB0C00F6D0521C08BF1046704710B50400200001F078FEC6
:20AFA000200010BD10B50B000024DBB2492B01D2002801D1002411E0DBB2DFF8A81E51F85A
:20AFC00033200100DBB20FF6A46010EBC3004068FFF786FF002801D04FF6FF74200080B2A3
:20AFE00010BD10B50B000024DBB2492B01D2002801D1002411E0DBB20FF6706151F83320AE
:20B000000100DBB20FF6646010EBC3004068FFF77CFF002801D04FF6FF74200080B210BD32
:20B0200030B585B000AC02250320207001212000FFF7D7FF2A00D2B221002120FEF764FAFF
:20B0400003251020208002212000FFF7CAFF2A00D2B221002220FEF757FA022501202070C7
:20B0600003212000FFF7BDFF2A00D2B221002320FEF74AFA02250020207004212000FFF77D
:20B08000B0FF2A00D2B221002420FEF73DFA02250120207005212000FFF7A3FF2A00D2B25E
:20B0A00021002520FEF730FA02250020207006212000FFF796FF2A00D2B221002620FEF758
:20B0C00023FA02250020207007212000FFF789FF2A00D2B221002720FEF716FA0425DFF89B
:20B0E000880D206008212000FFF77BFF2A00D2B221002920FEF708FA00255FF07E502060B1
:20B1000009212000FFF76DFF2A00D2B221003820FEF7FAF900255FF07E5020600A21200067
:20B12000FFF75FFF2A00D2B221003920FEF7ECF900255FF07E5020600B212000FFF751FF65
:20B140002A00D2B221003A20FEF7DEF900255FF07E5020600C212000FFF743FF2A00D2B205
:20B1600021003B20FEF7D0F900255FF07E5020600D212000FFF735FF2A00D2B221003C2030
:20B18000FEF7C2F900255FF07E5020600E212000FFF727FF2A00D2B221003D20FEF7B4F904
:20B1A00000255FF07E5020600F212000FFF719FF2A00D2B221003E20FEF7A6F900255FF03A
:20B1C0007E50206010212000FFF70BFF2A00D2B221003F20FEF798F90B2506202070002016
:20B1E000607011212000FFF7FCFE2A00D2B221004020FEF789F90225022020701F2120005E
:20B20000FFF7EFFE2A00D2B221004E20FEF77CF90B25162020700020607012212000FFF775
:20B22000E0FE2A00D2B221004120FEF76DF902250420207020212000FFF7D3FE2A00D2B2F4
:20B2400021004F20FEF760F90B25032020700020607013212000FFF7C4FE2A00D2B2210062
:20B260004220FEF751F902250320207021212000FFF7B7FE2A00D2B221005020FEF744F9D5
:20B280000B25042020700020607014212000FFF7A8FE2A00D2B221004320FEF735F902256D
:20B2A0000420207022212000FFF79BFE2A00D2B221005120FEF728F90B250520207000208D
:20B2C000607015212000FFF78CFE2A00D2B221004420FEF719F90225012020702321200052
:20B2E000FFF77FFE2A00D2B221005220FEF70CF90B25062020700020607016212000FFF77D
:20B3000070FE2A00D2B221004520FEF7FDF802250220207024212000FFF763FE2A00D2B25E
:20B3200021005320FEF7F0F80B25072020700020607017212000FFF754FE2A00D2B2210056
:20B340004620FEF7E1F802250320207025212000FFF747FE2A00D2B221005420FEF7D4F83A
:20B360000B25082020700020607018212000FFF738FE2A00D2B221004720FEF7C5F8022561
:20B380000420207026212000FFF72BFE2A00D2B221005520FEF7B8F80B2509202070002081
:20B3A000607019212000FFF71CFE2A00D2B221004820FEF7A9F80225012020702721200046
:20B3C000FFF70FFE2A00D2B221005620FEF79CF80B250A202070002060701A212000FFF771
:20B3E00000FE2A00D2B221004920FEF78DF802250220207028212000FFF7F3FD2A00D2B2C7
:20B4000021005720FEF780F80B250B202070002060701B212000FFF7E4FD2A00D2B221004A
:20B420004A20FEF771F802250320207029212000FFF7D7FD2A00D2B221005820FEF764F89E
:20B440000B250C202070002060701C212000FFF7C8FD2A00D2B221004B20FEF755F8022555
:20B46000042020702A212000FFF7BBFD2A00D2B221005920FEF748F80B250D202070002075
:20B4800060701D212000FFF7ACFD2A00D2B221004C20FEF739F80225012020702B2120003A
:20B4A000FFF79FFD2A00D2B221005A20FEF72CF80B250E202070002060701E212000FFF765
:20B4C00090FD2A00D2B221004D20FEF71DF80225012020702C212000FFF783FD2A00D2B230
:20B4E00021005B20FEF710F80025DFF8E80C20602D212000FFF775FD2A00D2B221002C2052
:20B50000FEF702F80025DFF8D00C20602E212000FFF767FD2A00D2B221002D20FDF7F4FF18
:20B520000025DFF8B80C20602F212000FFF759FD2A00D2B221002E20FDF7E6FF0025DFF81D
:20B54000A00C206030212000FFF74BFD2A00D2B221002F20FDF7D8FF0025DFF8880C206017
:20B5600031212000FFF73DFD2A00D2B221003020FDF7CAFF0025DFF8700C206032212000E2
:20B58000FFF72FFD2A00D2B221003120FDF7BCFF0025DFF8580C206033212000FFF721FD52
:20B5A0002A00D2B221003220FDF7AEFF0025DFF8400C206034212000FFF713FD2A00D2B2D8
:20B5C00021003320FDF7A0FF0025DFF8280C206035212000FFF705FD2A00D2B22100342023
:20B5E000FDF792FF00255FF08440206036212000FFF7F7FC2A00D2B221003520FDF784FF13
:20B600000025DFF8F00B206037212000FFF7E9FC2A00D2B221003620FDF776FF00255FF05E
:20B620008440206038212000FFF7DBFC2A00D2B221003720FDF768FF0425002020603921DC
:20B640002000FFF7CEFC2A00D2B221005C20FDF75BFF03257D2020803A212000FFF7C1FCDE
:20B660002A00D2B221005D20FDF74EFF04250A2020603C212000FFF7B4FC2A00D2B2210078
:20B680005F20FDF741FF03250A2020803D212000FFF7A7FC2A00D2B221006020FDF734FF78
:20B6A0000225012020703E212000FFF79AFC2A00D2B221006120FDF727FF02252120207045
:20B6C0003F212000FFF78DFC2A00D2B221006220FDF71AFF02250220207040212000FFF7BD
:20B6E00080FC2A00D2B221006320FDF70DFF02250420207041212000FFF773FC2A00D2B20C
:20B7000021006420FDF700FF02250020207042212000FFF766FC2A00D2B221006520FDF797
:20B72000F3FE02250120207043212000FFF759FC2A00D2B221006620FDF7E6FE0025DFF848
:20B74000B80A206044212000FFF74BFC2A00D2B221006720FDF7D8FE022501202070482184
:20B760002000FFF73EFC2A00D2B221006920FDF7CBFE05B030BD30B585B000AC02250121B3
:20B780002000FFF70FFC2A00D2B221002120FDF7BBFE032502212000FFF704FC2A00D2B2BC
:20B7A00021002220FDF7B0FE022503212000FFF7F9FB2A00D2B221002320FDF7A5FE02255F
:20B7C00004212000FFF7EEFB2A00D2B221002420FDF79AFE022505212000FFF7E3FB2A003B
:20B7E000D2B221002520FDF78FFE022506212000FFF7D8FB2A00D2B221002620FDF784FE1C
:20B80000022507212000FFF7CDFB2A00D2B221002720FDF779FE042508212000FFF7C2FB55
:20B820002A00D2B221002920FDF76EFE002509212000FFF7B7FB2A00D2B221003820FDF75E
:20B8400063FE00250A212000FFF7ACFB2A00D2B221003920FDF758FE00250B212000FFF7A1
:20B86000A1FB2A00D2B221003A20FDF74DFE00250C212000FFF796FB2A00D2B221003B20A1
:20B88000FDF742FE00250D212000FFF78BFB2A00D2B221003C20FDF737FE00250E212000BD
:20B8A000FFF780FB2A00D2B221003D20FDF72CFE00250F212000FFF775FB2A00D2B2210023
:20B8C0003E20FDF721FE002510212000FFF76AFB2A00D2B221003F20FDF716FE0B2511218E
:20B8E0002000FFF75FFB2A00D2B221004020FDF70BFE02251F212000FFF754FB2A00D2B232
:20B9000021004E20FDF700FE0B2512212000FFF749FB2A00D2B221004120FDF7F5FD0225AC
:20B9200020212000FFF73EFB2A00D2B221004F20FDF7EAFD0B2513212000FFF733FB2A008C
:20B94000D2B221004220FDF7DFFD022521212000FFF728FB2A00D2B221005020FDF7D4FD6A
:20B960000B2514212000FFF71DFB2A00D2B221004320FDF7C9FD022522212000FFF712FBBB
:20B980002A00D2B221005120FDF7BEFD0B2515212000FFF707FB2A00D2B221004420FDF713
:20B9A000B3FD022523212000FFF7FCFA2A00D2B221005220FDF7A8FD0B2516212000FFF709
:20B9C000F1FA2A00D2B221004520FDF79DFD022524212000FFF7E6FA2A00D2B22100532016
:20B9E000FDF792FD0B2517212000FFF7DBFA2A00D2B221004620FDF787FD02252521200037
:20BA0000FFF7D0FA2A00D2B221005420FDF77CFD0B2518212000FFF7C5FA2A00D2B22100A9
:20BA20004720FDF771FD022526212000FFF7BAFA2A00D2B221005520FDF766FD0B25192100
:20BA40002000FFF7AFFA2A00D2B221004820FDF75BFD022527212000FFF7A4FA2A00D2B2D3
:20BA600021005620FDF750FD0B251A212000FFF799FA2A00D2B221004920FDF745FD022545
:20BA800028212000FFF78EFA2A00D2B221005720FDF73AFD0B251B212000FFF783FA2A0025
:20BAA000D2B221004A20FDF72FFD022529212000FFF778FA2A00D2B221005820FDF724FD02
:20BAC0000B251C212000FFF76DFA2A00D2B221004B20FDF719FD02252A212000FFF762FA54
:20BAE0002A00D2B221005920FDF70EFD0B251D212000FFF757FA2A00D2B221004C20FDF7FB
:20BB000003FD02252B212000FFF74CFA2A00D2B221005A20FDF7F8FC0B251E212000FFF7A0
:20BB200041FA2A00D2B221004D20FDF7EDFC02252C212000FFF736FA2A00D2B221005B20AD
:20BB4000FDF7E2FC00252D212000FFF72BFA2A00D2B221002C20FDF7D7FC00252E212000EF
:20BB6000FFF720FA2A00D2B221002D20FDF7CCFC00252F212000FFF715FA2A00D2B2210074
:20BB80002E20FDF7C1FC002530212000FFF70AFA2A00D2B221002F20FDF7B6FC00253121DB
:20BBA0002000FFF7FFF92A00D2B221003020FDF7ABFC002532212000FFF7F4F92A00D2B294
:20BBC00021003120FDF7A0FC002533212000FFF7E9F92A00D2B221003220FDF795FC002527
:20BBE00034212000FFF7DEF92A00D2B221003320FDF78AFC002535212000FFF7D3F92A00E0
:20BC0000D2B221003420FDF77FFC002536212000FFF7C8F92A00D2B221003520FDF774FCE1
:20BC2000002537212000FFF7BDF92A00D2B221003620FDF769FC002538212000FFF7B2F9FE
:20BC40002A00D2B221003720FDF75EFC042539212000FFF7A7F92A00D2B221005C20FDF7F8
:20BC600053FC03253A212000FFF79CF92A00D2B221005D20FDF748FC0C253B212000FFF720
:20BC800091F92A00D2B221005E20FDF73DFC0C22DFF868155E20FDF712FC04253C212000F8
:20BCA000FFF780F92A00D2B221005F20FDF72CFC03253D212000FFF775F92A00D2B22100D2
:20BCC0006020FDF721FC02253E212000FFF76AF92A00D2B221006120FDF716FC02253F21F7
:20BCE0002000FFF75FF92A00D2B221006220FDF70BFC022540212000FFF754F92A00D2B2F1
:20BD000021006320FDF700FC022541212000FFF749F92A00D2B221006420FDF7F5FB022550
:20BD200042212000FFF73EF92078022805D30020207042212000FFF754F92A00D2B2210074
:20BD40006520FDF7E1FB022543212000FFF72AF92078042805D30020207043212000FFF704
:20BD600040F92A00D2B221006620FDF7CDFB002544212000FFF716F92A00D2B22100672074
:20BD8000FDF7C2FB032547212000FFF70BF92A00D2B221006820FDF7B7FB0225482120009B
:20BDA000FFF700F92A00D2B221006920FDF7ACFB0222DFF84C146920FDF781FB0222DFF852
:20BDC00044146520FDF77BFB0222DFF83C146620FDF775FB0222DFF830146620FDF76FFBC4
:20BDE0000022DFF828146720FDF769FB0322DFF820146820FDF763FB0222DFF818142520B9
:20BE0000FDF75DFB0721DFF81004FFF7CBF84621DFF80804FFF7C6F80024DFF800040068A5
:20BE2000DFF8FC13FEF7A0FB05F0BCFA0400601EDFF8F013884213D3DFF8E0030021016099
:20BE40004621DFF8D803FFF7CCF80022DFF8CC130520FDF759FB4621DFF8C003FFF7A2F839
:20BE600005B030BD6CBE00082A2C0A00040000000001000001000000040100000200000081
:20BE80000601000001000000080100000100000009010000010000000A0100000100000079
:20BEA0000B010000010000000C010000040000001001000004000000140100000400000036
:20BEC00018010000040000001C0100000400000020010000040000002401000004000000D6
:20BEE00028010000040000002C01000004000000300100000200000034010000020000007A
:20BF0000360100000200000038010000020000003A010000020000003C0100000200000031
:20BF20003E01000002000000400100000200000042010000020000004401000002000000F1
:20BF4000460100000200000048010000020000004A010000020000004C01000002000000B1
:20BF60004E0100000100000050010000010000005101000001000000520100000100000078
:20BF8000530100000100000054010000010000005501000001000000560100000100000047
:20BFA0005701000001000000580100000100000059010000010000005A0100000100000017
:20BFC0005B010000010000005C010000010000005D010000040000006001000004000000DF
:20BFE000680100000400000064010000040000006C01000004000000800100000400000075
:20C00000880100000400000084010000040000008C01000004000000700100000400000004
:20C02000780100000400000074010000040000007C010000040000009001000002000000F6
:20C0400094010000100000009601000004000000A801000002000000AC0100000100000047
:20C06000AE01000001000000AF01000001000000B001000001000000B101000001000000FA
:20C08000B201000001000000B301000004000000B401000016000000B801000004000000AC
:20C0A000D001000002000000D401000001000000D601000000B585B001A800210022002307
:20C0C0000EC00C38FEF708FF3220FCF7E3F80020ADF80000022200A94FF40370FEF715FFE1
:20C0E0003220FCF7D7F80020ADF80000022200A94FF41370FEF709FF3220FCF7CBF84A483D
:20C1000000210170484800214170474800218170032245494FF40570FEF7F7FE3220FCF7F0
:20C12000B9F84148002101703F48002141703E480021817003223C494FF40D70FEF7E5FE00
:20C140003220FCF7A7F8384800210170364800214170354800218170032233494FF40970AD
:20C16000FEF7D3FE3220FCF795F830480021018002222E494FF41370FEF7C7FE03222B4959
:20C180002820FDF7C1F9FEF74BFFFFF7F4FA092201A94AF2E030FEF7B8FE05B000BD80B513
:20C1A00000200090FEF798FE002100A8FEF7FAFE00981F49884207D01D480090002100A82F
:20C1C000FEF70FFFFEF72CFFFFF7D5FAFFF7D3FA01BD0000000072430000684300008443CF
:20C1E00000007E4300004643000050430000044300000E43CDCC0C4233335542347C002016
:20C20000288000202680002027800020547E00205C7F0020258000202E8000207C7E00202F
:20C2200000002041002D3101107E0020627F0020110317020A22002105F0ADB910B50024D1
:20C24000C0B203280CD2C0B20C21214A01FB0020006880474FF6FF71884201D14FF6FF7405
:20C26000200080B210BD70B50400080011001A000025E4B2032C0DD292B2E4B20C23144E0F
:20C2800003FB04635B6898474FF6FF71884201D14FF6FF75280080B270BD70B504000800D5
:20C2A00011001A000025E4B2032C0DD292B2E4B20C23074E03FB04639B6898474FF6FF7130
:20C2C000884201D14FF6FF75280080B270BD00009CCA000800B587B0012141F2040005F0DA
:20C2E000F7FAE020ADF8000003208DF8020018208DF8030000A9DFF88C0705F055FB1020B6
:20C30000ADF8000003208DF8020010208DF8030000A9DFF8700705F047FB1021DFF8640775
:20C3200005F0B3FB0020ADF804004FF48270ADF806000020ADF808000220ADF80A000120F2
:20C34000ADF80C004FF40070ADF80E000020ADF810000020ADF812000720ADF8140001A990
:20C36000DFF8240705F0FCFB0121DFF81C0705F017FC4FF6FF7007B000BD00B587B0012175
:20C38000082005F0A5FA01214FF4804005F0B0FA4FF42040ADF8000003208DF802001C20EF
:20C3A0008DF8030000A9DFF8E40605F0FDFA4FF48040ADF8000003208DF8020004208DF8A4
:20C3C000030000A9DFF8C40605F0EEFA4FF48050ADF8000003208DF8020014208DF8030015
:20C3E00000A9DFF8A80605F0DFFA4FF48051DFF89C0605F04AFB0020ADF804004FF482707C
:20C40000ADF806000020ADF808000020ADF80A000120ADF80C004FF40070ADF80E00382045
:20C42000ADF810000020ADF812000720ADF8140001A9DFF85C0605F093FB0121DFF85006DB
:20C4400005F0AEFB4FF6FF7007B000BD00B587B00121012005F03CFA0121DFF8380605F090
:20C460001AFB01210C2005F033FA01214FF4004005F03EFA3820ADF8000003208DF80200BE
:20C4800018208DF8030000A9DFF8000605F08CFA4FF40040ADF8000003208DF802001020D9
:20C4A0008DF8030000A9DFF8DC0505F07DFA4FF40041DFF8D00505F0E8FA0020ADF8040057
:20C4C0004FF48270ADF806000020ADF808000220ADF80A000120ADF80C004FF40070ADF8B4
:20C4E0000E000020ADF810000020ADF812000720ADF8140001A9DFF8A00505F031FB012139
:20C50000DFF8940505F04CFB4FF6FF7007B000BD80B51021DFF86C0505F0BAFA062000F0DA
:20C520005CFA1021DFF85C0505F0AFFA01BD80B54FF40041DFF84C0505F0AAFA062000F050
:20C5400088FA4FF40041DFF83C0505F09EFA01BD80B51021DFF82C0505F09AFA042000F067
:20C560003CFA1021DFF81C0505F08FFA00F05AF801BD80B54FF40041DFF8080505F088FACA
:20C58000042000F066FA4FF40041DFF8F80405F07CFA00F057F801BD80B51021DFF8E40443
:20C5A00005F076FA502000F018FA1021DFF8D40405F06BFA1021DFF8CC0405F069FA012019
:20C5C00000F00BFA002000F008FA1021DFF8B40405F05BFA00F026F801BD80B54FF40041C5
:20C5E000DFF8A00405F054FA502000F032FA4FF40041DFF8900405F048FA4FF40041DFF870
:20C60000840405F045FA012000F023FA002000F020FA4FF40041DFF86C0405F036FA00F026
:20C6200011F801BD10B50120002401E000F01AF8C0B2C00705D52000441C42F21071884234
:20C64000F4D310BD10B50120002401E000F01EF8C0B2C00705D52000441C42F21071884243
:20C66000F4D310BD10B51021DFF8180405F010FA052000F0B2F900F0ABF904001021DFF8DE
:20C68000040405F002FA2000C0B210BD10B54FF40041DFF8F00305F0FBF9052000F0D9F95F
:20C6A00000F0D2F904004FF40041DFF8D80305F0ECF92000C0B210BDF8B504000D00160078
:20C6C00000271021DFF8BC0305F0E2F90B2000F084F9200CC0B200F080F9200AC0B200F071
:20C6E0007CF92000C0B200F078F9002000F075F904E000F06DF9BFB278557F1CBFB2B6B268
:20C70000B742F6D31021DFF87C0305F0BEF94FF6FF70F2BD70B504000D0000264FF4805151
:20C72000DFF8680305F0B4F914F07F0000F073F904E000F06BF9B6B27055761CB6B2032EA6
:20C74000F7D34FF48051DFF8440305F09EF94FF6FF7070BDF8B504000D00160000274FF432
:20C760000041C84805F094F90B2000F072F9200CC0B200F06EF9200AC0B200F06AF920005C
:20C78000C0B200F066F9002000F063F904E000F05BF9BFB278557F1CBFB2B6B2B742F6D3D0
:20C7A0004FF40041B74805F070F94FF6FF70F2BDF8B504000D0016000027200000F0C6F86C
:20C7C000FFF7EAFEFFF7A4FE1021AE4805F060F9AD2000F002F9200CC0B200F0FEF8200A08
:20C7E000C0B200F0FAF82000C0B200F0F6F8287800F0F3F8687800F0F0F81021A14805F033
:20C8000044F90220070015E0401E0028FCD110219C4805F03DF9AD2000F0DFF8785D00F0D1
:20C82000DCF87F1C785D00F0D8F87F1C1021954805F02BF9B6B2B74201D27820E5E7642016
:20C8400000E0401E0028FCD1FFF782FE10218D4805F01EF9FFF7E6FE4FF6FF70F2BD38B5F3
:20C8600004000D004FF48051884805F011F954F08000C0B200F0CFF8287800F0CCF86878A3
:20C8800000F0C9F8A87800F0C6F84FF480517F4805F0FBF84FF6FF7032BDF8B504000D00F5
:20C8A00016000027FFF799FEFFF741FE4FF40041744805F0EDF8AD2000F0CBF8200CC0B241
:20C8C00000F0C7F8200AC0B200F0C3F82000C0B200F0BFF8287800F0BCF8687800F0B9F864
:20C8E0004FF40041674805F0D0F80220070017E0401E0028FCD14FF40041624805F0C8F8F2
:20C90000AD2000F0A6F8785D00F0A3F87F1C785D00F09FF87F1C4FF400415A4805F0B5F802
:20C92000B6B2B74201D27820E3E7642000E0401E0028FCD1FFF71DFE4FF40041514805F087
:20C94000A7F8FFF77FFE4FF6FF70F2BD10B50400FFF722FEFFF7DCFD10214A4805F098F86C
:20C96000202000F03AF8200CC0B200F036F8200AC0B200F032F82000C0B200F02EF810210A
:20C98000404805F082F8FFF74DFE10BD10B50400FFF723FEFFF7CBFD4FF40041394805F0FA
:20C9A00077F8202000F055F8200CC0B200F051F8200AC0B200F04DF82000C0B200F049F820
:20C9C0004FF400412F4805F060F8FFF73BFE10BD80B5002000F001F802BD10B5040002212A
:20C9E000294805F0EFF80028F9D0E4B2210089B2254805F0E3F80121234805F0E3F8002845
:20CA0000F9D0214805F0DCF8C0B210BD80B5002000F001F802BD10B5040002211C4805F09A
:20CA2000D1F80028F9D0E4B2210089B2184805F0C5F80121164805F0C5F80028F9D01448B9
:20CA400005F0BEF8C0B210BD80B5002000F001F802BD10B5040002210F4805F0B3F80028E4
:20CA6000F9D0E4B2210089B20B4805F0A7F80121094805F0A7F80028F9D0074805F0A0F840
:20CA8000C0B210BD0008014000300140000C01400038004000023000003C0040D5C200088B
:20CAA000B9C60008B1C700087BC3000815C700085FC800084DC4000855C700089BC800086E
:20CAC0000CB41CB5044604A80190009401AB0A4600A907487844183005F07EF8009900228C
:20CAE0000A7000285CBF0098001B16BC5DF80CFB5B020000002840F10880F446404200F0AE
:20CB000004F850F00040604700280AD0B0FA80F18840D1F19D01C905020672F1004241EB06
:20CB20001020704710B5FF2313EAD0541DBF13EAD1529C429A4239E0A41ADA0780EA01032A
:20CB4000134042EA012142EA0020421A3CBF641E01EB4202090AB2FBF1FE01FB1E221202E0
:20CB6000B2FBF1F001FB10226EF30F201202B2FBF1FE4EEA00207F3406DDFE2C24DA53EA66
:20CB8000500050EBC45010BDD4F1020401FB1E2240F08071192C1DDC21FA04F0C4F12004DB
:20CBA000A140114371F10042584110BD9C421ABF03EAD1529A420FE080EA010E0EF00043EA
:20CBC000400004D0490016D143F0FF4010BD490008BFD343180010BD9C4205D1D21AF7D060
:20CBE00001F00041484010BD4A0212BF0846484000F0004010BD4AB90902B1FA81F29140C1
:20CC000044B1A418C00140F000409EE7C90141F0004152420002B0FA80F4A040141B94E733
:20CC20004FF0807C1CEB400F94BF1CEB410F05E040EA010C5FEA4C0C01D28842704718BFD1
:20CC40008142704740EA010C5FEA4C0C07D0884205D14FEA400C1CF1807F98BF80427047AA
:20CC600080B50A480069804702BD80B507484069804702BD80B5C0B20449096A884702BD96
:20CC800080B5C0B20149496A884702BD540800204AB38B0707D0521E11F8013B00F8013B97
:20CCA00021D08B07F7D183071ED1103A07D330B4B1E83810103AA0E83810F9D230BC53079C
:20CCC00024BFB1E80810A0E8081044BF51F8043B40F8043BD20724BF31F8022B20F8022BC7
:20CCE00044BF0B7803707047083A07D3B1E80810083A40F8043B40F804CBF7D25307E4E709
:20CD0000002205F0F9BDFEE7FEE7FEE7FEE7FEE7FEE7704700F10103810704D010F8011BBC
:20CD200089B18107FAD10268B2F10131914311F0803F04BF50F8042FF6E710F8011B11B192
:20CD400010F8011BFBE7C01A70470268531C0360117070472DE9F04105000E0090461C007C
:20CD60000027DFF814020078012803D342F6E160208020E0002D03D145F6C35020801AE026
:20CD800005F0D6FD0700DFF8F4012860C5F814800020A8616E6015F1080000F094FEDFF8C1
:20CDA000E0010088401CDFF8D8110880380005F0C3FD00202080BDE8F0812DE9F04389B021
:20CDC00006000F0091469846109C00256A480078012804D346F2AE10208000207AE0002E50
:20CDE00004D145F6C3502080002073E01FFA89F94846002802D0B0F5004F20D130685F49B5
:20CE0000884221D1B8F1000F02D00020C8F8000005F08EFD0500706900281AD07069401E45
:20CE20007061B8F1000F02D0B069C8F800007669280005F081FD0020208030004AE045F6EF
:20CE400025602080002045E045F6C4502080002040E05FEA094008D57669280005F06CFD65
:20CE600046F2B0102080300034E046480078012807D3280005F060FD46F6635020800020A4
:20CE800028E03B000622310000A800F0D2FD280005F052FD00F0ACFC05F04AFD05003A48C8
:20CEA000006890F83500002805D002282BD014D303281ED033E0B8F1000F04D032480068AA
:20CEC000006CC8F80000002020807669280005F033FD300009B0BDE8F083B8F1000F04D0AD
:20CEE00029480068006CC8F8000046F2A9102080EBE7B8F1000F02D00020C8F8000047F227
:20CF0000D9202080E1E7B8F1000F04D01E480068006CC8F8000045F6C2502080D5E746F645
:20CF20002B602080280005F007FD0020D2E770B504000D001600002C04D145F6C350308081
:20CF4000002011E020680D49884204D045F6C4503080002008E005F052FD0200330029009B
:20CF600089B2200000F012F870BD054900220A8000210180704700003C80002053454D41DA
:20CF8000BE7F002040800020E47E00202DE9F04782B004000D0016001F005FF0000805F0C1
:20CFA000C7FC804614F108000189002918D1606910F1010F07D1404605F0BEFC46F6C55007
:20CFC0003880002033E06069401C6061D4F81490A661404605F0B0FC00203880484626E076
:20CFE000A90502D5B0F8089001E05FF00109D0F800A00BE0DAF80810DAF804A000960023C6
:20D000000022200000F0D5FDB9F101091FFA89F9B9F1000FEED1D4F81490404605F08CFCD2
:20D02000280401D400F0E4FB002038804846BDE8F68700002DE9F04106000F0090461C004A
:20D040000025DFF87C020078012803D342F6E16020802BE0002E03D145F6C350208025E0C6
:20D060001FFA88F8B8F1000F03D146F2945020801CE005F05DFC0500DFF8480230607760F8
:20D08000414689B216F1140005F028FD16F1080000F019FDDFF830020088401CDFF8281286
:20D0A0000880280005F048FC00202080BDE8F0812DE9F04F89B004000D0016001F00DDF808
:20D0C0004880DDF84C905FF0000A7D480078012805D346F2AE10A9F800000020C4E0002CB9
:20D0E00005D145F6C350A9F800000020BCE0002F05D146F2D520A9F800000020B4E0B6B2C0
:20D100003000002802D0B0F5004F1DD120686D4988421FD1B8F1000F02D00020C8F80000A1
:20D1200005F006FC82464B464246390014F1140005F0DEFC8346B9F80000002810D15046DD
:20D1400005F0FAFB58468FE045F62560A9F80000002089E045F6C450A9F80000002083E07B
:20D16000300408D5504605F0E7FB46F2B010A9F80000002078E055480078012808D3504671
:20D1800005F0DAFB46F66350A9F8000000206BE02B000522210000A800F04BFC504605F0ED
:20D1A000CBFB00F025FB05F0C3FB82464848006890F83500002805D0022838D017D3032825
:20D1C00026D045E042480068D0F85CB040480068B0F860003880B8F1000F04D03C48006846
:20D1E000006CC8F800000020A9F8000038E05FF0000B00203880B8F1000F04D03448006888
:20D20000006CC8F8000046F2A910A9F8000027E05FF0000B00203880B8F1000F02D000206D
:20D22000C8F8000047F2D920A9F8000018E05FF0000B00203880B8F1000F04D024480068D1
:20D24000006CC8F8000045F6C250A9F8000007E05FF0000B0020388046F62B60A9F8000033
:20D26000504605F069FB584609B0BDE8F08F2DE9FC4105000E0017009846089C002D03D144
:20D2800045F6C350208013E028680E49884203D045F6C45020800BE005F0B1FB0194009089
:20D2A00043469BB23A0092B23100280000F012F8BDE8F381044900220A800021018070475C
:20D2C0003C80002051554555BC7F002040800020E47E00202DE9F04F83B004000D001600C6
:20D2E0001F00DDF83080DDF834905FF0000A05F01FFB824614F108000189002914D1F8061E
:20D3000001D4002300E01023CDF80490CDF800809BB2320092B2290014F1140005F020FC4E
:20D32000504605F009FB25E0B90502D5B0F808B001E05FF0010B00680DE0816840680190B1
:20D34000CDF8008033009BB22A00200000F031FC0198BBF1010B1FFA8BFBBBF1000FECD139
:20D36000504605F0E9FA380401D400F041FA0020A9F80000BDE8F78FF8B505000E00140043
:20D380000027DFF858020078012803D347F2752020803FE0DFF848020078012803D346F65D
:20D3A0006350208036E0B6B23000002805D0022803D004281ED008281DD1002D03D147F200
:20D3C0007E20208026E005F0B3FA070085480068012180F836102300320092B229008148C0
:20D3E000006805F071FC2088002808D0380005F0A3FA0FE0E7E745F6256020800AE0794829
:20D40000006800F0C0FC380005F096FA00F0F0F900202080F1BDF8B5069C079D00276F4E1D
:20D420003678012E03D347F275202880B0E06C4E3678012E03D346F663502880A8E014F0A3
:20D440000E06B6B23700002F05D0022F03D0042F17D0082F16D1002B0CD192B2002A09D189
:20D4600089B2002906D180B2002803D147F27E2028808DE04FF6E17C14EA0C0F06D100279E
:20D4800005E0F7E745F62560288081E00127FFB2012F03D145F62560288079E0C4F3001497
:20D4A000A4B214F00104E4B2012C1CD04FF47A74A34203D347F27B20288069E092B23C2A03
:20D4C00003D347F27A20288062E089B23C2903D347F2792028805BE080B2642815D347F2AF
:20D4E0007820288054E042F2107489B2A14203D347F2792028804BE04FF47A7480B2A04222
:20D5000003D347F27820288042E0374C246880B24FF4616789B25FF03C0C0CFB01F107FB81
:20D52000001092B210184FF4FA71B1FBF4F1C91801FB04F14FF47A72B1FBF2F104FB00148D
:20D54000002C22D005F0F4F9070026480068012180F836102B00320092B22100214800687B
:20D5600005F0B2FB2888002803D0380005F0E4F90EE01C48006800F006FC380005F0DCF9A6
:20D5800000F036F90020288002E047F27E202880F1BD10B582B005F0B7FD00AA00211348CF
:20D5A00000F000FF0400124800780C21114A01FB002000F037FC10480068401E0E49086002
:20D5C0000D480068002808D10B480C490968016000AA00210A4800F0E5FE13BD3C80002077
:20D5E00040800020E47E002008360108806A00203E800020C85F0020E07E0020DC7E00205B
:20D60000406B002010B5040005F0F9FCDFF8A00800210170DFF89C0800210170DFF89808F7
:20D6200000210170DFF8940800210160DFF8900800210160DFF88C0800210160DFF888081E
:20D6400000210170DFF8840800680A21B0FBF1F0DFF87C180860DFF87C08006800280ED01A
:20D66000DFF874080068002809D0DFF86818096803E0491E00220260001D0029F9D105F053
:20D6800083FD00F001FB200000F09AFE2088002837D1200000F0A5F92088002831D12000FE
:20D6A00005F0C4FA208800282BD1200005F0B0FD2088002825D1200005F0B2FD20880028CF
:20D6C0001FD1200005F0C2F92088002819D1200005F0AEFD2088002813D12000FFF7EAFD5F
:20D6E000208800280DD12000FFF73FFC2088002807D1200005F0A6FD2088002801D105F034
:20D7000019FF10BDDFF8AC07007801280BD1DFF8A0070078FA2806D2DFF894070078401CE7
:20D72000DFF88C170870704710B50024DFF88407007801285BD105F0FBF80400DFF87007EE
:20D740000078002803D1200005F0F6F84FE0DFF860070078401EDFF858170870DFF8500723
:20D760000078012803D3200005F0E6F83FE0DFF848070078012803D3200005F0DDF836E083
:20D7800005F00CFDDFF854170870DFF8500700780C21DFF84C2701FB00200068DFF84417FE
:20D7A0000860DFF840070068DFF83C170968884203D1200005F0C0F819E0DFF8280700680E
:20D7C000D0F88C00401CDFF81C170968C1F88C00DFF818070068401CDFF810170860DFF8E2
:20D7E00010075FF080510160200005F0A5F810BD10B50024DFF8B806007801283ED2DFF80C
:20D80000B8060078012839D205F092F8040005F0C5FCDFF8C8160870DFF8C00600780C21F6
:20D82000DFF8BC2601FB00200068DFF8B8160860DFF8B0060068DFF8B0160968884203D1FD
:20D84000200005F079F819E0DFF898060068D0F88C00401CDFF88C160968C1F88C00DFF8B6
:20D860008C060068401CDFF884160860DFF880065FF080510160200005F05EF810BD38B576
:20D8800004000025DFF828060078012803D346F66250208022E0DFF81C060078012803D0E6
:20D8A00045F68960208019E0DFF80C060078FA2803D345F20920208010E005F039F8050037
:20D8C000DFF8F4050078401CDFF8EC15087000F088FA280005F030F80020208031BD38B502
:20D8E00004000025DFF8C8050078012803D346F66550208030E0DFF8BC050078012803D037
:20D9000045F68960208027E0DFF8AC050078002803D146F6645020801EE005F009F80500B7
:20D92000DFF894050078401EDFF88C150870DFF888050078012806D3280004F0FDFF46F67F
:20D940006350208008E000F056FA280004F0F4FFFFF74EFF0020208031BD10B50400DFF8AC
:20D9600054050078002826D105F018FCDFF86C150870DFF88005DFF8641509780170DFF869
:20D980005C0500780C21DFF8582501FB00200068DFF850150860DFF85005DFF84815096834
:20D9A0000160DFF810050121017005F04FFE43F69920208002E045F68A60208010BD80B50A
:20D9C000002104F0B5FF0100DFF82C050068401CDFF824251060080004F0AEFF05F00EFB7A
:20D9E000EFE700B589B0DFF8101500220A600890032007900020069000200590002004906A
:20DA0000DFF8F80400680390DFF8F40400680290DFF8F00400680190132000900023DFF8EE
:20DA2000E8240FF24051DFF8E40400F0A5FA09B000BD70B504000D001900DFF8AC04006846
:20DA400080F83420DFF8A0040068002280F83520DFF89404006800F05BFA002D0ED015F1FB
:20DA60000806E56001222100DFF87C04006800F010F82100300000F02DF809E0DFF86804C6
:20DA800000680021C187DFF8600400680021016370BD10B4C287016300230EE000244C600E
:20DAA00000240C6000240C6100244C6100240C830024CC61886020315B1C9BB292B293425A
:20DAC000ECD310BC7047002101600021416000210181704710B48A6892F837200389002B18
:20DAE00008D10122028100224A6000220A600160416024E003895B1C0381046800E06468AA
:20DB0000002C05D0A36893F83730D2B29A42F6D2002C06D100224A6042680A6051604160AA
:20DB20000DE02268002A05D1216000220A604C60016004E022680A604C605160216010BCD2
:20DB4000704770B50400266BE58F06E0F0680830310000F00AF820366D1EADB2012DF5D212
:20DB60000020E0870020206370BD0289012A04D1002202600022426013E00A68002A04D117
:20DB80004B6800221A6003600BE04A68002A04D10A6800235360426003E00A684B68536092
:20DBA0001A600289521E02810020486000200860704738B505000C00049894F836100029D1
:20DBC0000BD002290AD008D3042906D006D3062925D002D3072922D042E041E094F8341080
:20DBE000032906D100909BB22100280000F039F803E0E265A4F860302064002D02D02000E2
:20DC0000FFF79FFF200000F0A0F9002084F83600002084F83500002084F8340020E094F8C8
:20DC20003410032906D100909BB22100280000F018F803E0E265A4F860302064200005F088
:20DC4000D1F8002D02D02000FFF77BFF042084F83600002084F83500002084F83400FFE70F
:20DC600031BD70B4039C0D6BC98F01E02035491E89B2012906D3EE68B042F7D128616A61E4
:20DC80002B83EC6170BC704700200BE0C0B20C21934A01FB002100220A8100220A600022A7
:20DCA0004A60401CC0B21428F0D3704710B5040094F8370005F082FA94F837008D4909781F
:20DCC000884203D1200000F022F802E0200000F001F810BD90F837100C22814B02FB0131CC
:20DCE0000A89002A08D101220A810022C260002202610860486009E00A89521C0A810A6820
:20DD0000C260002202610A6810610860704790F837100C22724B02FB01310A89002A08D1DB
:20DD200001220A810022C260002202610860486008E00A89521C0A810022C2604A6802618F
:20DD4000D0604860704710B40189002902D0022901D00BD215E0016842680A610023CB6051
:20DD600000231361D160026041600AE001684268CB6800241C610024CC600A61D1600360B8
:20DD8000416010BC704710B5040094F837000C21534A01FB00202169E268002913D1002AE2
:20DDA0000AD100210181002101600021416094F8370005F016FA0FE00189491E0181002156
:20DDC0001161026008E003895B1E0381CA60002A01D1416000E01161002020610020E060E4
:20DDE00010BD80B534480078012803D104F007FE3249086001BD80B52F480078002810D169
:20DE000004F0FDFD2D490968401A2D490968814201D22B4908602B490968814201D229498D
:20DE2000086001BD38B5040000252748007801283CD104F07DFD05002068002803D128006A
:20DE400004F07AFD32E03149884203D1280004F073FD2BE0816D002902D0816D491E816572
:20DE6000806D002803D0280004F066FD1EE02089022803D2280004F05FFD17E00E48007858
:20DE8000012803D3280004F057FD0FE02000FFF75AFF2068416D002903D10D4909688165D5
:20DEA00001E0416D8165280004F046FD31BD00003C8000203D80002040800020B87E0020B1
:20DEC000BC7E0020C07E00204180002008360108C47E0020F0350108EC3501083F800020C9
:20DEE000C85F0020E87E0020E47E0020C87E002004ED00E03E800020B47E0020E43501084A
:20DF0000E0350108DC350108BFD90008C069002010B582B00400002910D000AB02222000ED
:20DF200004F0D2FEBDF80000002803D1032084F8360006E0022084F8360002E0022084F85D
:20DF400036002000FFF71FFF13BD10B50400200004F048FF94F83600400702D42000FFF76E
:20DF6000A5FE10BD75432F4F532D4949492049646C65205461736B002DE9FE4F82B00500B5
:20DF80000F9EDDF84090119FDDF84C80159CDDF858A05FF0000BDFF83C040078012804D377
:20DFA00047F24A10AAF80000ABE0002D04D147F2AD10AAF80000A4E00398002804D147F2B2
:20DFC0004F10AAF800009CE0002E04D146F62C60AAF8000095E0DFF820050068874204D2DF
:20DFE00046F62D60AAF800008BE0B94504D346F62E60AAF8000084E09DF83800142804D3C6
:20E0000046F27320AAF800007BE09DF83800132808D1DFF8E804854204D046F27320AAF88C
:20E0200000006EE0280000F0D9F90020AAF80000E0070AD5A00708D53000002103E0002246
:20E040000260001D491CB942F9D316EB8909A4B2019400974B4632000499039804F0DCFF36
:20E060000399A9620499E962029929629DF8381085F837102860C5F80890C5F85480B8F133
:20E08000000F04D1DFF834050068A86501E0C5F85880149868606E62AF63AC87002005E013
:20E0A00080B215EB80010022CA67401C80B20028F6D0BDF8481015F1640004F00FFD28003F
:20E0C00004F0A7FF04F034FC834695F8370005F075F82800FFF71BFEDFF8E4040088401CB9
:20E0E000DFF8DC140880DFF8DC040078012803D0584604F021FC04E0584604F01DFCFFF772
:20E1000077FB05B0BDE8F08FF8B505000C000026DFF8C0020078012803D347F24E10208089
:20E1200044E0DFF8D803854203D147F24C1020803CE0002D08D104F0FBFB0600DFF89802B6
:20E140000568300004F0F8FB04F0F2FB060095F8360000280BD002282ED029D3042826D048
:20E160002AD3062828D023D3072825D03AE02800FFF709FE15F1640004F08EFC070028000C
:20E1800004F048FFDFF838040088401EDFF830140880280000F022F9FF2085F83600300073
:20E1A00004F0CAFBFFF724FB00202080F1BDE1E7280004F017FEDDE7280004F013FE95F8AC
:20E1C0003400002808D0401E07D0401E04D0401E032802D9001F04D103E02800FFF7B1FC9E
:20E1E000FFE7C7E7300004F0A7FB46F62A602080DCE72DE9F0410700884616001C00002529
:20E20000DFF8D0010078012804D346F2AE1020800020C5E0002E01D00020306004F088FB5D
:20E220000500DFF8A4030068406C00283CD0DFF898030068406C401EDFF88C13096848649C
:20E24000DFF884030068476C002E04D0DFF878030068006C306004F0D2FBDFF86C13096805
:20E26000096C401ADFF860130968C1F8A800DFF858030068D0F8AC00DFF84C130968D1F835
:20E28000A810884209D2DFF840030068DFF838130968D1F8A810C0F8AC10280004F04CFBB4
:20E2A0000020208038007BE05FEA084007D5280004F042FB46F2B0102080002070E0DFF866
:20E2C0000C030078012807D3280004F035FB46F663502080002063E03B00072200210020D1
:20E2E000FFF7A7FB280004F027FBFFF781FA04F01FFB0500DFF8D002006890F835000028CE
:20E3000004D001282ED0032837D03EE0002E26D0DFF8B4020068006C306004F070FBDFF867
:20E32000A8120968096C401ADFF89C120968C1F8A800DFF894020068D0F8AC00DFF88812D2
:20E340000968D1F8A810884209D2DFF87C020068DFF874120968D1F8A810C0F8AC10002086
:20E36000208015E0002E04D0DFF85C020068006C306046F2A91020800AE0002E01D00020D3
:20E38000306047F2D920208002E046F62B602080DFF834020068476C280004F0CDFA38008F
:20E3A000BDE8F08170B504000D00160004F027FB02003300290089B2200000F0A1F870BD76
:20E3C0007F4900220A80824900220A6000210180704700003C800020E47E002010B50400F2
:20E3E000002020600020A060002060600020E06000202061002060610020A0610020E06119
:20E400000FF2D0102062002060620020A0620020E062002020630020E08700202064002045
:20E42000E0650020A4F86000002114F1640004F055FB002060670020A0670020C4F8800043
:20E440000020A4F888000020C4F88400002005E0C0B214EB80010022CA67401CC0B20028D8
:20E46000F6D0002060640020C4F8A8000020C4F8AC000020A063002084F88A000020C4F8C1
:20E48000B4000020C4F8B0000020A0875FF00040A0640020E0640020206500206065002054
:20E4A000A065002084F88B000020C4F88C000020C4F8900004F0A3FAC4F89400002000213A
:20E4C000C4E926010020C4F8B800002084F83400002084F83500002084F83600142084F8B1
:20E4E000370010BD80B53848006804F094FD00A90020FFF709FE01BD04360108C069002066
:20E500002DE9F04182B007000C0090461E00002504F00EFA0500002F01D12B480768C7F8B3
:20E5200040800020308097F8360000280BD002281DD008D3042806D019D3062817D002D3B9
:20E54000072814D030E0786C10F1010F07D1280004F0F2F946F6C550308000202CE0786CB3
:20E56000401C78647E6C280004F0E6F923E097F83400072810D1CDF80080002300223900E5
:20E580000020FFF716FB7E6C280004F0D5F9200409D4FFF72DF906E0786C401C78647E6C77
:20E5A000280004F0C9F906E0280004F0C5F946F62A60308000263000BDE8F681C47E002073
:20E5C000C07F00203D800020E47E002040800020C87E00203F5461736B00000080B5002010
:20E5E0008DF80000012200A91820FAF768FF02220DF101011F20FAF762FF01220DF1020161
:20E600001E20FAF75CFFBDF802004FF6FF71884222D19DF8010000281ED19DF800000028DD
:20E620000DD1DFF878040078552803D1DFF86C04AA210170DFF86804552101700CE0DFF870
:20E6400060040078552803D1DFF85404AA210170DFF8480455210170DFF848040078AA28AB
:20E660000CD1DFF844040078052807D3DFF83404552101700221002005F08EF901BDDFF8D5
:20E680002C0400210180DFF8240400214180DFF81C040021C180DFF8140400218180DFF886
:20E6A0000C0400214181DFF8040404210181DFF8FC0300210161DFF8F403DFF8F413C160BB
:20E6C000704780B580B2002809280ED90C3816D0401E1CD0401E0DD0401E05D00B3801288E
:20E6E00041D9103833D03FE03EE0DFF8C8035521017039E0DFF8BC03AA21017034E00320CD
:20E70000F9F71EFFDFF8B003012101802CE0DFF8980300210170DFF89C030078AA2811D10D
:20E72000DFF898034FF6FF71018006220021DFF89003FBF797FF1220F9F702FFDFF8780381
:20E7400001210180DFF86C03552101700CE0DFF87403AA2101700620F9F7F2FEDFF858033B
:20E760000121018000E0FFE7DFF85C034FF6FF71018001BD10B588B0DFF850030078401E09
:20E78000DFF844130988002900F0FF80CE480021018000A9C548C08805F05DF94FF41B7251
:20E7A0002021CB48FBF75EFFFAF7B3F8BE480078052806D3C74800210170C6490220F9F7D4
:20E7C000BBFCB9480078401CB7490870FAF706F8FFF704FF0222C0496920FAF770FEBF4831
:20E7E00000884FF6FF7188420BD0BB480078022807D0B9480078032803D0B74800780428A1
:20E8000005D10120F9F79CFEAB480121018001A8FBF7BEFC4FF41B722021AD48FBF722FF73
:20E82000FAF777F8AE4800780C21AE4A01FB0020027AAB4800780C21AA4B01FB00304168EB
:20E84000A74800780C23A74C03FB00400078A04B13EB40003E30FAF77AF8A14800780C21F1
:20E86000A04A01FB002090F820209D4800780C219C4B01FB0030C169994800780C23994C96
:20E8800003FB0040007E924B13EB4000FAF75FF8934800780C21934A01FB002090F8382000
:20E8A0008F4800780C218F4B01FB0030416B8C4800780C238B4C03FB004090F83000844B13
:20E8C00013EB40007C30FAF742F8854800780C21854A01FB002090F83820814800780C2178
:20E8E000814B01FB0030416B7D4800780C237E4C03FB004090F83000754B13EB4000BA3060
:20E90000FAF725F80F220DF10601754800780C23754C03FB004090F848006D4B13EB40008A
:20E92000BA30FAF714F8002010E0C0B2009911EB0011C0B23E22664B02FB00328A60C0B2BA
:20E940000101009A4FF6FF738B52401CC0B20428EBD3009800214173009810214177009849
:20E96000202180F82D100098302180F83D100098302180F84D10F9F7AEFF0221002000F065
:20E980009EF90221022000F09AF908B010BD10B582B000244C484FF6FF7101804248002103
:20E9A00001704FF41B7220214948FBF75BFEF9F7B0FF3A4855210170394855210170002069
:20E9C000FAF7EEFEC02200214848FBF74BFE00200090002200A90020FAF796FD002200A9A2
:20E9E0000120FAF791FD002200A90220FAF78CFD002200A90320FAF787FD002200A90420BE
:20EA0000FAF782FD3A48AA2101703A48AA2101702C48552101703848552101703748552153
:20EA20000170374855210170364855210170402200213548FBF716FE402200213348FBF7A4
:20EA400011FE392200213248FBF70CFE314855210170314855210170304800210170304873
:20EA600000210170082200212E48FBF7FBFD2E48002101602D48002101602D48552101700E
:20EA80002C48002101702C480021017013BD214855210170204855210170704762090020B9
:20EAA000630900205E090020168000208C780020F49300085409002042090020547F0020FF
:20EAC000F87C00206A0900204C7F00202B800020704E0020AC7C002028800020687F002064
:20EAE00026800020A0BB010890BC01084068002068090020690900206B0900206C09002083
:20EB00006E090020700900206074002020740020A074002064090020650900201B80002013
:20EB20001C800020F07C00203C7E0020407E002073090020068000200780002030B589B0CE
:20EB40000300080000AC911E232901D3002038E00A2A03D1002B01D5012500E00025EDB224
:20EB6000002D01D05B4203E002E030312170641C002B02D100A98C420BD1B3FBF2F102FBE4
:20EB80001131B3FBF2F30A29EFDB37312170641CEEE7002805D100A8201A2818401C02F0E7
:20EBA00076F80100002D07D02D220A70491C03E0641E22780A70491C00AAA242F8D300225B
:20EBC0000A7009B030BD10B58AB00300080000AC911E232901D3002026E002E03031217096
:20EBE000641C002B02D100A98C420BD1B3FBF2F102FB1131B3FBF2F30A29EFD337312170F3
:20EC0000641CEEE7002804D100A8201A401C02F03EF8010003E0641E22780A70491C00AAB3
:20EC2000A242F8D300220A700AB010BD38B5C0B2042812D201230122C0B20321524C01FB1C
:20EC400000418978C0B203244F4D04FB0050407800F0E8FF4FF6FF7000E0002032BD10B5F7
:20EC6000C0B2042811D20122C0B20321464B01FB00318978C0B20323434C03FB004040787E
:20EC800001F051F84FF6FF7000E0002010BD10B5C0B2042811D20022C0B203213A4B01FB3A
:20ECA00000318978C0B20323374C03FB0040407801F039F84FF6FF7000E0002010BD80B539
:20ECC000C0B2002830D1C9B2012914D12F490978002958D1C0B2FFF7DAFF2D4802684FF461
:20ECE0007A71092004F0F0FE092005F01FF927480121017047E025490978012943D1C0B220
:20ED0000FFF7C5FF092005F011F9002301220721012000F087FF00220721012001F003F8B5
:20ED20001A48002101702EE0C0B202282BD1C9B201291BD117480078002803D01648007800
:20ED4000012820D10220FFF78AFF0320FFF787FF4FF47A70F9F79EFA0220FFF798FF0D48A0
:20ED6000012101700C48002101700CE009480078012808D10220FFF78AFF0320FFF787FF23
:20ED800004480021017001BDE8080020EE7F0020547E0020EF7F0020E87F002070B40122EC
:20EDA00040F24B135FF0FF3100E0621C1BB212B2934221DB5FF0FF3409B2A1421CD11BB2AA
:20EDC00012B2D418022594FBF5F424B222253E4E05FB046535F8225C80B28542E5D324B2A0
:20EDE0002223394D03FB045333F8223C80B2984201D2631EDAE7611E080000B270BC70472D
:20EE000070B504000D00002613E0305D00280DD0305D4FF480713219527801FB002080B2ED
:20EE2000FFF7BCFF00F200102880AD1CB61C00202880305D002809D0102E07DA305DA12811
:20EE4000E3D2305D2880AD1C761CF0E770BDF0B4049C059D89B2102934D180B2802804D359
:20EE600042F2200680B2B0421DD1198080B2C1B20C26164F06FB017109891B8891FBF3F139
:20EE8000118080B2C1B20C22104B02FB0131897A298080B2C0B20C210C4A01FB00204068ED
:20EEA0002060F0BC7047102119800221118010212980074980B22222034B02FB00300818B6
:20EEC0002060EEE7EDE70000A873010834AD030802DEFFFF38B5040000200090002200A9AF
:20EEE000E4B23420DFF83C3600FB0430C0785023DFF8345603FB0050406980B2FAF704FB8B
:20EF0000002200A9E4B23420DFF8183600FB0430C0785023DFF8105603FB0050806980B297
:20EF2000FAF7F2FA002200A9E4B23420DFF8F43500FB0430C0785023DFF8EC5503FB0050FF
:20EF4000C06980B2FAF7E0FA002200A9E4B23420DFF8D03500FB0430C0785023DFF8C8552C
:20EF600003FB0050006A80B2FAF7CEFA002200A9E4B23420DFF8AC3500FB0430C0785023A7
:20EF8000DFF8A44503FB0040406A80B2FAF7BCFA31BD70B58EB00400002001900020099031
:20EFA00000200890002007900020069000200D9000200C9000200B9000200A90002000908E
:20EFC000002005900020049000200390002002900025002209A9E4B23420DFF8483500FB31
:20EFE0000430C0785023DFF8406503FB0060806980B2FAF764FA002208A9E4B23420DFF85A
:20F00000243500FB0430C0785023DFF81C6503FB0060C06980B2FAF752FA002207A9E4B207
:20F020003420DFF8003500FB0430C0785023DFF8F86403FB0060006A80B2FAF740FA00221C
:20F0400006A9E4B23420DFF8DC3400FB0430C0785023DFF8D46403FB0060406A80B2FAF71C
:20F060002EFA00220DA93820FAF729FA00220CA93920FAF724FA00220BA93A20FAF71FFAAB
:20F0800000220AA93B20FAF71AFADFF8A0040021016009990D98FBF767FA059008990C98CA
:20F0A000FBF762FA049007990B98FBF75DFA039006990A98FBF758FA02900999089800F006
:20F0C00001FC079900F0FEFB069900F0FBFB01900599049800F0F6FB039900F0F3FB029964
:20F0E00000F0F0FB0090002205A90720FAF70CFA002204A90820FAF707FA002203A90920D7
:20F10000FAF702FA002202A90A20FAF7FDF90199DFF81C0400F0D6FBE4B23421DFF80424E8
:20F1200001FB042188620099DFF8040400F0CAFBE4B23421DFF8EC2301FB04214862E4B265
:20F140003420DFF8E01300FB0410816ADFF8E403FBF70AFAFBF774FA05000A20B5FBF0F1C3
:20F1600000FB115005280ED3A81DFDF7CDFCDFF8C413FDF7D7FCE4B23421DFF8A82301FBA5
:20F18000042188620DE0A81CFDF7BEFCDFF8A413FDF7C8FCE4B23421DFF8882301FB04212D
:20F1A0008862E4B23420DFF87C1300FB0410416ADFF88003FBF7D8F9FBF742FA05000A20E1
:20F1C000B5FBF0F100FB115005280DD3A81DFDF79BFCDFF86013FDF7A5FCE4B23421D14A00
:20F1E00001FB042148620BE0A81CFDF78DFCD149FDF798FCE4B23421CA4A01FB04214862AC
:20F20000E4B23420C74900FB0410806A0190002201A90020FAF778F9E4B23420C14900FB2D
:20F220000410406A0090002200A90620FAF76CF90EB070BD80B5C0B23421BA4A01FB002032
:20F24000001DFAF70CFC002802D17FF0050000E0002002BD1CB50400E4B23420B14900FBB6
:20F2600004104078022815D12000C0B2FFF7E2FF10F1060F02D17FF0050021E0E4B2342001
:20F28000A84900FB0410032141702000C0B2FFF721FE14E0E4B23420A24900FB0410407862
:20F2A00003280CD100A8FAF793FC002802D17FF0050005E000A92000C0B2FFF76AFE002011
:20F2C00016BD1CB50400E4B23420964900FB04104078022815D12000C0B2FFF7ABFF10F1B3
:20F2E000060F02D17FF0050051E0E4B234208D4900FB0410032141702000C0B2FFF7EAFD6E
:20F3000044E0E4B23420874900FB0410407803283CD100A8FAF75CFC002802D17FF00500B0
:20F3200035E000A92000C0B2FFF733FEE4B234207C4900FB0410416A7C48006800F0C2FA15
:20F340000100E4B23420774A00FB0420006AFDF767FC1BD2E4B23420724900FB0410103040
:20F36000FAF77DFB002802D17FF005000FE0E4B234206C4900FB041005214170E4B2342057
:20F38000684900FB0410022180F83010002016BD1CB50400E4B23420624900FB04104078AE
:20F3A000022815D12000C0B2FFF744FF10F1060F02D17FF005004CE0E4B23420594900FB62
:20F3C0000410032141702000C0B2FFF783FD3FE0E4B23420534900FB04104078032837D19D
:20F3E00000A8FAF7F5FB002802D17FF0050030E000A92000C0B2FFF7CCFDE4B2342049498F
:20F4000000FB0410806AE4B23421464A01FB0421C96A00F003F91BD8E4B23420414900FBD6
:20F4200004101030FAF71BFB002802D17FF005000FE0E4B234203B4900FB041005214170BF
:20F44000E4B23420374900FB0410032180F83010002016BD30B585B00400E4B234203149E2
:20F4600000FB04104078022815D12000C0B2FFF7E1FE10F1060F02D17FF005004FE0E4B22C
:20F480003420284900FB0410032141702000C0B2FFF720FD42E0E4B23420224900FB041098
:20F4A000407803283AD100A8FAF792FB002802D17FF0050033E000A92000C0B2FFF769FD1F
:20F4C00002A8FAF7CCFA002802D17FF0050026E0E4B23420134900FB041010F1100102A845
:20F4E000FAF7E3FA022819D1E4B234200D4900FB0410103002A92CC92CC00C390C38E4B2F0
:20F500003420084900FB041005214170E4B23420044900FB0410042180F83010002005B068
:20F5200030BD0000DC74002040070020047E0020ACC5A73700401C4690EA010F44BF81F076
:20F54000004100F0C6B9431A4FF000423EBF5340C01AC918D3095FEAD05C13EB400F34BF41
:20F56000B3EB410F40E07CEBD1530CD342EA012122D8D1EB402009D3400A28BF5FEA500108
:20F5800040EBCC507047401A15D04002B0FA80F2521C9040400A4FEA3C23B3EB026384BF6A
:20F5A00000EB730007E040F400001A16DB07C2F10102D04018437047182BFCDC31FA03F2AD
:20F5C00002FA03F3591A38BF42F00102D2EB40203CBF4000ACF1010C5FEACC5CC20572F1FD
:20F5E00000414CEB5020704713EB400F0FD24B0009D0ACEBD153022B03DB4902172BDDDD0D
:20F6000070479143401A4300D5D10020704713EB410FD0D36FF00000704700004FF0807C03
:20F620001CEB400F94BF1CEB410F05E040EA010C5FEA4C0C01D28142704718BF8842704768
:20F640005FF0FF0C1CEAD05114BF614506E0C110400721F0E04101F16051704779B900F004
:20F66000004100020AD0B0FA80FC00FA0CF001F16051A1EB0C5101EBD021400570474102A9
:20F680000CBF40F4E0016FF00001002070470000B0B581EA030C0CF0004C40F2FF7515EA87
:20F6A00011541DBF15EA1357AC42AF4239E0E41923EA455343F48013C90241F0004141EAD4
:20F6C000505EC7021100A7FB020200284FF00000EEFB01204FF00001E3FB072118BF42F03C
:20F6E0000102401800214941E3FB0E01A4F580640F0302D252004041494154F101046CDDC4
:20F70000470872F1004250F1000051EB0451A1F580115CBF41EA0C01B0BD4CEA0551002090
:20F72000B0BD05EA1357AC4214BFAF4241E050EA410E1CBF52EA430E02E061460020B0BD29
:20F7400024423C441BD15FEA070EF6D0090302BF01460020AEF1140EB1FA81F7AEEB0704F7
:20F7600001FA07FE0C37C7F1200100FA07F7C8404EEA000E23EA455343F48013A2E733F00C
:20F780000043B3FA83F704BFB2FA82FE77440B3FE41BB7F1200E2FBF02FA0EF3BB40C7F198
:20F7A000200E22FA0EFE38BF43EA0E03BA40641C82E750EA410E14BF52EA430E6FF0000192
:20F7C0004FF4001717EB430F8ABF194617EB410FB5E74CEA05510020B0BDD4F10104B4F15D
:20F7E00020070FDAC4F12007520828BF42F0010210FA07F501FA07F7E1BF2A43E040384300
:20F80000E1400FE0352C98DCC7F1200452EA400220FA07F218BF42F0010231FA07F0A14087
:20F820000A43002172F1004250F1000051EB0C01B0BD00004FEAF17CBCF1E04C2CBFBCF5A3
:20F84000001F11E05FEA4C0C34BFBCF17F5F2EE05FEA9C0C4FEA0C1C4FEA3C0CC10071F175
:20F8600000414CEB50707047C90241EA5051C00218BF41F0010141F000414FEA6C50C0F11E
:20F880000900212810D240EACC7CCCF1200C11FA0CF070F10040CCF1200C21FA0CF00CF035
:20F8A000004C40EB0C0070474FEACC707047490011F5001F04D84FEACC10FF30C0057047D8
:20F8C000C817704790EA010F44BF81F00041FFF73ABE421A3CBF801A89184FF0004CC0F395
:20F8E000C752FF2A24D0C1F3C75313B3D21AD2F1190327DD4CEA01214CFA03F321EA0303CA
:20F90000D140C20D4CEA0020401834BF20EA0C004CEA5000D20553EA006373EB0C0C52EBA0
:20F920001020420012F1807F38BF7047C00DC0057047490212BF9A4200EB5120F8E7D2F166
:20F940001703D9D57047000080B501215FF0C05001F0CEFF012004F00BFB012001F003FF85
:20F96000412001F0D5FF0028FAD04FF4807001F00FFF012001F012FF04F039FB04F032FBD1
:20F9800004F030FB47F6FF7004F01EFB04F02AFB01BD7047704780B2042190FBF1F202FB88
:20F9A0001102002A16D180B2642190FBF1F201FB120100290CD180B24FF4C87190FBF1F2CD
:20F9C00001FB1200002801D1012004E0002002E0012000E0002070472DE9F34F81B0002493
:20F9E000BDF804509DF806609DF807709DF809809DF80A909DF80BA0A5F2B27080B28228D5
:20FA000001D3012055E040F2B27B03E07C4804191BF1010B1FFA8BFBADB2AB4508D258461B
:20FA200080B2FFF7B8FF0028F0D076480419EFE7761E5FF0000B17E01FFA8BFB0FF2D810E1
:20FA40001BF80000704901FB0044280080B2FFF7A2FF002806D01FFA8BFBBBF1010F01D17E
:20FA6000694804191BF1010B3000C0B21FFA8BFB80B28345E0D3FFB2781E634901FB00447F
:20FA80005FFA88F84FF4616000FB08445FFA89F93C2000FB09445FFA8AFA1AEB040404F0E5
:20FAA0006DFA200004F084FA04F06FFA04F09AFA0020BDE8FE8F30B480B2642390FBF3F308
:20FAC00080B2642490FBF4F504FB1500DBB2142B00D36430C0B2C0B2042390FBF3F31B1802
:20FAE0009BB2072493FBF4F504FB1533D2B2C9B20FF218140C1914F8014CA218D318C0B20F
:20FB0000042290FBF2F404FB1204002C03D1C9B2032900D25B1E9BB2072093FBF0F100FB69
:20FB20001130C0B230BC7047F8B5040000260025002704F032FA06003348B6FBF0F0050015
:20FB400040F2B270070002E0A5F26D157F1CB5F5B67F0BD9380080B2FFF71DFF0028F3D08A
:20FB6000B5F5B77F02D3B5F5B775EFE72780002701E01D3D7F1C1C2D16D32088FFF70BFFA6
:20FB8000002805D0BFB2012F02D11D2DF1D20BE0BFB20FF28400385C854205D3BFB20FF261
:20FBA0007800385C2D1AE5E7781CA070681CE0701548B6FBF0F100FB11654FF46160B5FB9A
:20FBC000F0F060714FF46160B5FBF0F100FB11503C21B0FBF1F0A0714FF46160B5FBF0F1F4
:20FBE00000FB11503C21B0FBF1F201FB1200E071E278A1782088FFF75EFF2071F1BD0000B2
:20FC00008033E1010085E201805101000003030601040602050003051F1C1F1E1F1E1F1FFC
:20FC20001E1F1E1F70B582B004000D001600E4B2012C0AD02DD3032C11D00BD3052C18D028
:20FC400012D3072C1FD019D323E00121042001F03FFE1EE00121082001F03AFE19E00121AE
:20FC6000102001F035FE14E00121202001F030FE0FE00121402001F02BFE0AE00121802084
:20FC800001F026FE05E001214FF4807001F020FEFFE70120A840ADF80000F6B2012E03D1C7
:20FCA00010208DF8030009E0F6B2002E03D104208DF8030002E014208DF8030002208DF808
:20FCC0000200E4B2012C0AD02CD3032C11D00BD3052C18D012D3072C1FD019D322E000A9E1
:20FCE000844801F061FE1DE000A9834801F05CFE18E000A9814801F057FE13E000A9804818
:20FD000001F052FE0EE000A97E4801F04DFE09E000A97D4801F048FE04E000A97B4801F03A
:20FD200043FEFFE773BD80B5C0B201280BD0C0F08F8003282DD019D3052850D03CD3072863
:20FD400073D05FD384E0D2B2002A07D1012010FA01F189B2674801F09BFE06E0012010FAA2
:20FD600001F189B2634801F090FE71E0D2B2002A07D1012010FA01F189B25F4801F088FEDF
:20FD800006E0012010FA01F189B25B4801F07DFE5EE0D2B2002A07D1012010FA01F189B2FA
:20FDA000564801F075FE06E0012010FA01F189B2524801F06AFE4BE0D2B2002A07D101203E
:20FDC00010FA01F189B24E4801F062FE06E0012010FA01F189B24A4801F057FE38E0D2B253
:20FDE000002A07D1012010FA01F189B2454801F04FFE06E0012010FA01F189B2414801F026
:20FE000044FE25E0D2B2002A07D1012010FA01F189B23D4801F03CFE06E0012010FA01F10A
:20FE200089B2394801F031FE12E0D2B2002A07D1012010FA01F189B2344801F029FE06E09C
:20FE4000012010FA01F189B2304801F01EFEFFE701BD10B51400C0B201280AD048D303288D
:20FE600019D00FD3052828D01ED3072837D02DD33EE0012010FA01F189B21E4801F0FAFDA7
:20FE8000207035E0012010FA01F189B21A4801F0F1FD20702CE0012010FA01F189B21748D1
:20FEA00001F0E8FD207023E0012010FA01F189B2134801F0DFFD20701AE0012010FA01F1B2
:20FEC00089B2104801F0D6FD207011E0012010FA01F189B20C4801F0CDFD207008E001204A
:20FEE00010FA01F189B2094801F0C4FD2070FFE710BD000000080140000C0140001001409E
:20FF00000014014000180140001C0140002001400749002201E01831521C0B78FF2B01D1EC
:20FF2000002004E00B78C0B28342F4D108007047C80600202DE9F0410E0017009846069CA5
:20FF4000C0B2FFF7E5FF0500002D01D1002013E02300DBB24246D2B23900C9B230006C68CA
:20FF60002468A047002129724FF6FF7180B2884201D10121297280B2BDE8F08110B50C00F9
:20FF8000C0B2FFF7C5FF0100002901D1002005E02000C0B249684968884780B210BDF8B5C5
:20FFA00004000D00160000270AE0BFB2795D2000C0B2FFF7E3FF4FF6FF71884200D17F1C6D
:20FFC000BFB2B742F1D34FF6FF70F2BD38B50C001500C0B2FFF79CFF0200002A01D1002061
:20FFE00005E02900200052689268904780B232BD70B50C0015001E00C0B2FFF789FF0028AB
:020000040801F1
:2000000001D1002004E004614661C5604FF6FF7070BD000062F30F2262F31F42401810F064
:20002000030308D0C91A1FD3DB0748BF00F8012D28BF20F8022D130030B4144615461039DB
:2000400028BF20E93C00FAD8490728BF20E90C0048BF40F8042D890028BF20F8022D48BF28
:2000600000F8012D30BC7047C91818BF00F8012DCB0728BF00F8012D70470000DFF8A406C2
:20008000016899B94FF4803181604FF4805141604FF0FF31C160016104214161DFF88816ED
:2000A0000422C1F8B821DFF8841601600120704701F1080313F0070308BF002307D001F121
:2000C000080303F00703C3F1080303F007035918D21A8161C26042F001034B605118282267
:2000E0004A60DFF840160969C16170472DE9F04101F1080414F0070408BF002407D001F1D6
:20010000080404F00704C4F1080404F00704611802F1080414F0070408BF002407D002F1D8
:20012000080404F00704C4F1080404F00704A5185A186C1AE41A43F003034B60AA4201D39D
:2001400003F06CBF6E68F307FAD5102CF8D383699D4207D1C368E318C360826143F00100D8
:20016000506042E143699D4208D18368E3188360426143F0010050609B5036E106F00303FA
:20018000012B40F0A080F308DB004FEAD30EBEF1200F26D2AF68D5F80CC06545D0D0BD4224
:2001A000CED0674506D10668012707FA0EF7BE43066086E04FEA4E0600EB860606F1280E84
:2001C000774503D0D0F810E07745B9D32836B44502D00669B445B3D3C7F80CC0CCF80870B2
:2001E0006FE0AF69EE68AE420AD0D5F808C0D0F810E0F445A4D3CCF80C60C6F808C024E0C1
:2002000005F2140CDCF8006046B905F1100CDCF80060D6B102E0F446DCF8006006F2140E5D
:20022000DEF80080B8F1000FF5D106F1100EDEF80080B8F1000FEED1D0F810E0F445FFF424
:200240007FAF4FF0000ECCF800E0002F39D0D5F81CC000EB8C0C0CF2301CDCF800E0754563
:200260000BD1CCF800609EB946680127D5F81CC007FA0CF7BE43466023E0D0F810C06745B6
:20028000FFF45EAFD7F810C0AC450CBF3E617E61BEB1D0F810C06645FFF452AFB7612F692F
:2002A00037B1D0F810C06745FFF44AAF3761BE616F6937B1D0F810C06745FFF441AF7761B0
:2002C000BE615D191C196B685B085B006B6044F001035360A450E308202B1BD25D0000EBAE
:2002E000850505F228052E46102CFFF429AF012707FA03F304681C4204BF2343036004D08C
:20030000AE6800698642FFF41BAFAA60F2609660D5606AE0230A08BF002523D0B3F5803F95
:2003200028BF1F251ED2A3F580752D0C05F00805AB40A3F58056360C06F00406B340A3F5B4
:2003400080473F0C07F00207C5F10E05AD1BED1BBB4005EBD333DD1D24FA05F505F00105F4
:2003600005EB430500EB850303F23013D561002656611661012707FA05F64768374207D1EC
:2003800046EA070444601A609361D26092602CE01B681F2D0EBF00256D08C5F1190504FAD8
:2003A00005F500E033465E68F608F600A6420ED0EE0F03EB860606F110076D003E68002EA4
:2003C000F0D100698742FFF4BBAE3A60DCE79C6800698342FFF4B4AE8442FFF4B1AEE26090
:2003E0009A609460D3600020906101F10800BDE8F0812DE9FE4F0446A56904F2BC102E46CA
:2004000001688E4203D3426851188E4202D380680028F5D14168006801EB0008A8F12F0072
:2004200000F1080111F0070108BF002107D000F1080101F00701C1F1080101F0070101EB67
:20044000000A05F11000824538BFAA460AF1080B0AF1180900270198A0F12802009920463A
:20046000FFF726FE1BF0070022D11B20CAF8040004F2BC10B0E80E10ABE80E10ABF1100B7C
:200480000098C4F8BC010198C4F8C0010298C4F8C801C4F8C4B100E0814609F10400072118
:2004A000C9F804107F1C011D4145F5D3022F01DA03F0B4BDAA4500F09380AAEB0600411909
:2004C0004A68520852004A6040F0010169604051C108202919D24A0004EB820202F22802B0
:2004E00013461028E4D3012606FA01F02168014206D1084320609560DD60AB60EA606FE058
:20050000936820698342F6D2D2E7010A08BF002223D0B1F5803F28BF1F221ED2A1F5807225
:20052000120C02F008029140A1F580531B0C03F004039940A1F58046360C06F00206C2F11E
:200540000E02D21A921BB14002EBD131CA1D20FA02F202F0010202EB410204EB820101F293
:200560003011EA6100236B612B61012606FA02F366681E4207D143EA060060600D60A961E8
:20058000ED60AD602CE009681F2A0EBF00225208C2F1190200FA02F200E019464B68DB0861
:2005A000DB0083420ED0D30F01EB830303F1100652003368002BF0D120698642FFF478AF1B
:2005C0003560DCE7886822699142FFF471AF9042FFF46EAFC5608D60A860E9600020A861F4
:2005E00000F052BBF8B504460D464E4E306808B9FFF744FD03F018FD010000F091800A680C
:2006000011F1010F00F08C80D4F8B0011018C4F8B001D4F8B401D4F8B031984238BF18465D
:20062000C4F8B401A06968BB206908B1814200D22161C4F8BC11C4F8C0210020C4F8C801F9
:20064000306860624FF0FF3020622046202300F22806F660B66008305B1EF8D13248844261
:2006600004D1283A2046FFF723FD48E054F8040CC00814EBC00008385118091AA1F1280234
:200680000146EFE704F2BC10034600E09B68BBB15E681F68F619B142F8D11E7B36070FD412
:2006A0003E46A769B7420BD35F68D4F818C0BE19B44505D2D0195860E0681218A169D1E7E8
:2006C0002369994238BF21610346501800E09B688BB11E688642FAD1187B00070BD4304662
:2006E00019605E6892195A602B460246204601B0BDE8F040FAE400232046FFF77AFEE06894
:2007000085420DD2401BE060A1696A18A26140F00100506045F00300486001F10800F2BD9F
:200720000020F2BDE0760020E45C00206859883C2DE9F04100224B420C0A08BF002423D0A5
:20074000B4F5803F28BF1F241ED2A4F580752D0C05F00805AC40A4F58056360C06F00406B1
:20076000B440A4F580473F0C07F00207C5F10E05AD1BED1BBC4005EBD434E51D21FA05F536
:2007800005F0010505EB440400EB8405D5F8305155B31F2C0EBF00266608C6F1190601FADF
:2007A00006F6002700E07600D5F804C04FEADC0C4FEACC0CACEB010C9C4502D22A4663468B
:2007C0007BB1D5F814C04FEAD67E05EB8E052D69BCF1000F02D0AC4518BF6746002DE2D1C3
:2007E0003D4675BB002A3DD1012505FA04F4640065422C4345682C4000F0518165422C4089
:20080000651E2C0B04F0100425FA04F6750905F00805EE40B70807F00407FE404FEA560CB5
:200820000CF0020C26FA0CF6C6F3400E2C193C196444744426FA0EF52C1900EB8404D4F8E4
:2008400030517DB100E025466C68E408E400641A9C423CBF23462A462C69002CF3D16D696F
:20086000002DF1D1002A00F01A818468641AA34280F0158116460469A64206D38C18CD186C
:200880005768FF08FF00AF4201D003F0C7BBA642FBD29769D66896420AD0D2F808C0D0F85D
:2008A00010E0F445F1D3CCF80C60C6F808C023E002F2140CDCF8006046B902F1100CDCF868
:2008C0000060CEB102E0F446DCF8006006F2140EDEF80080B8F1000FF5D106F1100EDEF810
:2008E0000080B8F1000FEED1D0F810E0F445CCD34FF0000ECCF800E0002F35D0D2F81CC0A6
:2009000000EB8C0C0CF2301CDCF800E072450BD1CCF8006096B946680127D2F81CC007FAD3
:200920000CF7BE4346601FE0D0F810C06745ACD3D7F810C094450CBF3E617E61A6B1D0F86B
:2009400010C06645A1D3B76117692FB1D0F810C067459AD33761BE6157692FB1D0F810C090
:20096000674592D37761BE61102B08D245F003005060A818416841F0010141608CE041F098
:200980000301516043F0010161601B51D908202918D24B0000EB830303F228031E460125C6
:2009A00005FA01F105680D4204BF2943016004D09E6800698642FFF468AF9C60F460A6608F
:2009C000E36069E0190A08BF002623D0B1F5803F28BF1F261ED2A1F580752D0C05F0080541
:2009E000A940A1F58056360C06F00406B140A1F580473F0C07F00207C5F10E05AD1BED1B2E
:200A0000B94005EBD131CD1D23FA05F505F0010505EB410600EB860101F23011E6610025A6
:200A2000656125610125B54047682F4207D13B462B4343600C60A161E460A4602CE0096892
:200A40001F2E0EBF00257508C5F1190503FA05F500E031464E68F608F6009E420ED0EE0F53
:200A600001EB860606F110076D003E68002EF0D100698742FFF409AF3C60DCE78B68056951
:200A8000A942FFF402AFAB42FFF4FFAEDC608C60A360E1600020A06102F1080000E00020B2
:200AA000BDE8F0812DE9F041426813465B421A40531E1A0B02F01002D3405C0904F00804CD
:200AC000E3409D0805F00405EB405E0806F00206F340C3F34007A218AA18B218BA18FB403E
:200AE0009A1800EB8202D2F8304123466268D208D200521A07E06568ED08ED006D1A95425B
:200B00003CBF2A4623462569002D14BF2C466469002CF0D11E460469A64206D3CC188D182C
:200B20005F68FF08FF00AF4201D003F077BAA642FBD29F69DE689E420AD0D3F808C0D0F8EA
:200B400010E0F445F1D3CCF80C60C6F808C023E003F2140CDCF8006046B903F1100CDCF8C3
:200B60000060CEB102E0F446DCF8006006F2140EDEF80080B8F1000FF5D106F1100EDEF86D
:200B80000080B8F1000FEED1D0F810E0F445CCD34FF0000ECCF800E0002F35D0D3F81CC002
:200BA00000EB8C0C0CF2301CDCF800E073450BD1CCF8006096B946680127D3F81CC007FA2F
:200BC0000CF7BE4346601FE0D0F810C06745ACD3D7F810C09C450CBF3E617E61A6B1D0F8C1
:200BE00010C06645A1D3B7611F692FB1D0F810C067459AD33761BE615F692FB1D0F810C0DE
:200C0000674592D37761BE61102A08D245F003005860E818416841F00101416030E041F00A
:200C20000301596042F001016160125187682FB341694FEAD70CBCF1200FBFF476AF4FEA1B
:200C40004C0500EB850505F228052E46102FFFF46CAF012707FA0CF7D0F800C01CEA070F19
:200C600004BF47EA0C07076004D0AE680769BE42FFF45BAFA960F1608E60CD6082604461B3
:200C800003F10800BDE8F08103B0BDE8F08FF8B50446012003F0F4F9F52C80F0D3800B2C58
:200CA00031BF102404F10B00C408E400E308DFF8F006016821FA03F515F0030233D0EA43F2
:200CC00002F00102D3185A0000EB820202F22805AA68DC005668F608F600A64201D003F0FE
:200CE0009DB99668AA42FAD0B242F8D05768FF08FF00A742F3D1B54205D1012505FA03F3D4
:200D00009943016004E000698642E8D3AE60F56044F003005060A018416841F00101416047
:200D200002F10805D6E08268A24280F09E80002D00F07F80012202FA03F6760005FA03F302
:200D4000754235432B405D422B405D1E2B0B03F0100325FA03F6750905F00805EE40B708B3
:200D600007F00407FE404FEA560C0CF0020C26FA0CF6C6F3400EEB18FB186344734426FAD1
:200D80000EF5ED186B0000EB830303F22806B368EF00D3F804C04FEADC0C4FEACC0CBC4580
:200DA0009DD1D3F808C0B34299D0634597D0664502BF02FA05F5A943016006D001698C4505
:200DC0008DD3C6F808C0CCF80C60391B44F003055D60E41841F001056560095186681EB39F
:200DE0004569F708202FBFF47AAF4FEA470C00EB8C0C0CF2280CE646102EFFF470AFBA4064
:200E00000668164204BF3243026005D0DCF808E002699645FFF463AFCCF80850CEF80C5058
:200E2000C5F808E0C5F80CC08160446103F1080550E0416800293AD02146FFF733FE05005E
:200E400013D047E014F1400F28BF4FF0FF340CD204F10B00C408E400DFF84405416821B1B2
:200E60002146FFF765FC050034D1DFF834058268A2421CD3131B4169102B0AD362184261D0
:200E8000836043F0010050609B5044F0030048600AE000238360436142F0030048605018E8
:200EA000426842F00102426001F1080512E0C1688C420BD2091BC1608269A318836141F0EC
:200EC0000101596044F00300506029E72146FFF789FB0546012003F0F5F82846F2BD0028EE
:200EE00000D17047F8B5A0F10804012003F0C8F8DFF8AC542A6994421ED3636803F003005A
:200F0000012819D0D808C0000119DE0729D4266813F0030300F0E280301873421C19944232
:200F20000AD36B699C4200F0CA80F308202B67D2A668E768BC4201D103F070B8B442FBD060
:200F4000D4F804C04FEADC0C4FEACC0CBCEBC30FF2D1BE4243D12A68012606FA03F39A43F3
:200F60002A608C42E8D24A68D307E5D5930700F15481AB69994240F0B580E9684018E86074
:200F8000AC6140F00101616069698C4202D100216961A960E969814280F0A080DFF8FC036F
:200FA000006808B9FFF76AF8A869002800F09680E96829290BD305F2BC121368984203D300
:200FC0005468E318984202D39268002AF5D1E869884280F083804FF0FF30E8617EE05B00C3
:200FE00005EB830303F1280C664501D09642A3D328339F4201D097429ED3F760BE60B0E726
:20100000A669E368A34205D0A768974294D3FB609F601DE004F214073B6833B904F110076A
:201020003B68ABB101E067463B6803F2140CDCF800E0BEF1000FF6D103F1100CDCF800E06E
:20104000BEF1000FEFD19742FFF476AF00223A60002E86D0E26905EB820202F2301217686D
:20106000BC4208D113607BB96A680123E669B3409A436A6075E72A699642FFF45DAF3269B2
:20108000A2420CBF33617361002B3FF46AAF2A699342FFF451AF9E6122692AB12E69B24277
:2010A000FFF44AAF1A6193616269002A3FF459AF2E69B242FFF440AF5A61936151E70A79CE
:2010C00002F00302032A7FF44CAFA8604A68520852004A6040F0010161600051012002F017
:2010E000F1FFF1BD6B69994204D1A9684018A8606C61EFE7D208D2001018D308202B24D2CA
:201100008E68CF68B9423FF417AFB1423FF414AFBE4205D1296801229A409143296073E0B1
:20112000590005EB810101F12802964203D02A699642FFF401AF28318F4203D029698F42AF
:20114000FFF4FAAEF760BE605EE08B69CA688A4207D08E682F69BE42FFF4EEAEF260966013
:201160001EE001F21406326832B901F110063268B2B101E03E46326802F21407D7F800C03D
:20118000BCF1000FF6D102F11007D7F800C0BCF1000FEFD12F69BE42FFF4CEAE00273760F2
:2011A00093B3CE6905EB860606F230163768B9420BD1326016468EB96A680123C96903FA28
:2011C00001F122EA010169601EE02E69B342FFF4B3AE1E698E420CBF1A615A61A2B12E6926
:2011E000B242FFF4A9AE93610B692BB12E69B342FFF4A2AE13619A61496929B12B69994234
:20120000FFF49AAE51618A6140F001016160005169698C4208D1A86060E7520852004A6094
:2012200040F0010161600051C10820291BD24A0005EB820202F2280213461028FFF47CAEE1
:20124000012606FA01F02968014204BF0843286004D0936828698342FFF46EAE9460DC60A8
:20126000A360E2603AE7010A08BF002223D0B1F5803F28BF1F221ED2A1F58072120C02F00C
:2012800008029140A1F580531B0C03F004039940A1F58046360C06F00206C2F10E02D21AC5
:2012A000921BB14002EBD131CA1D20FA02F202F0010202EB410205EB820101F23011E2619D
:2012C000002363612361012606FA02F36E681E4207D143EA060068600C60A161E460A460C8
:2012E0002CE009681F2A0EBF00225208C2F1190200FA02F200E019464B68DB08DB008342AE
:201300000ED0D30F01EB830303F1100652003368002BF0D128698642FFF40EAE3460DCE759
:2013200088682A699142FFF407AE9042FFF404AEC4608C60A060E1600020A061286A401ED6
:2013400028627FF4CBAED5F8C40118B94FF0FF302862C3E680680028FCD1F7E738B5002447
:2013600060B101FB00F441EA0002120C120405D0B4FBF0F0884218BF4FF0FF342046FFF738
:2013800086FC050008D015F8040C10F0030003D02146284602F0A4FE284632BDE0760020BF
:2013A000E45C00204100090E7F3915D4D1F11F0114D4400007D2C00140F00040C84048BFB1
:2013C0006FF000407047C00140F00040C8404CBF4FF00040404270470020704700424FF063
:2013E000004058BFC04370474FF6FF70704780B50B000100180002F080FE4FF6FF7002BD35
:2014000080B50B000100180002F06DFE4FF6FF7002BD80B502F098FE80B202BD30B583B0DD
:201420000C00150000AA01A902F0CEFE002801D1002007E02B00220000990198C0B202F095
:2014400036FF80B23EBD30B583B00C00150000AA01A902F0B9FE002801D1002007E02B00C8
:20146000220000990198C0B202F04BFF80B23EBD2DE9F04F85B080460D4616461F001CBF44
:2014800000203860444600E0641C2078A0F109010529F9D32028F7D02D2801D02B2802D122
:2014A00014F8019B01E04FF02B09002E03D4012E01D0252E04DB0DB1C5F80080002067E097
:2014C000012E0BDB102E16D12078302813D1607840F0200078280ED1A41C0CE020783028BB
:2014E00018BF0A2607D1607840F02000782808BF1026F1D0082603942078302803D114F8F2
:20150000010F3028FBD04FF0000A02940FF28C008DF8040009E0CDF800A09DF80410401A52
:201520005FFA80FB06FB0ABA641C2178A1F141001A2838BF203132460FF2600002F00EFFC4
:201540000028E8D10398A042B5D00298201A0FF27401715C401A13D4012807DABAEB0B0096
:2015600004D3B0FBF6F00099884209D002F022FF222101600FB1012038604FF0FF3A04E03B
:20158000B9F12D0F08BFCAF1000A05B12C60504605B0BDE8F08F00236AE7000030313233EE
:2015A0003435363738396162636465666768696A6B6C6D6E6F707172737475767778797AC5
:2015C0000000000000002115110E0D0C0B0B0A0A09090909090808080808080807070707F2
:2015E000070707070707070707000000DFF86403006850F00100DFF85C130860DFF85803E5
:201600000068DFF858130840DFF84C130860DFF844030068DFF848130840DFF838130860B0
:20162000DFF83003006830F48020DFF828130860DFF82403006830F4FE00DFF81C13086004
:20164000DFF82003002101607047DFF80813096831F48031DFF8FC221160DFF8F812096866
:2016600031F48021DFF8EC221160B0F5803F03D0B0F5802F09D011E0DFF8D802006850F49C
:201680008030DFF8D012086008E0DFF8C802006850F4A020DFF8BC120860FFE7704780B5A5
:2016A0000020009000200021312000F031F901000098401C0090C9B2002903D10098B0F594
:2016C000A06FF1D1312000F023F9002801D0012000E00020C0B202BD0022DFF87C321B6867
:2016E0001A0032F47C1208430243DFF86C0202607047DFF87412C0B2086070470021DFF848
:20170000582212681100890889000143DFF8480201607047DFF84002006810F00C007047E9
:201720000021DFF834221268110031F0F0010143DFF82402016070470021DFF81C221268B5
:20174000110031F4E0610143DFF80C02016070470021814A1268110031F4605151EAC00188
:201760007D4801607047824900220A70804900220A70C0B2012802D0042804D007E07C48A8
:201780000121017003E07A4805210170FFE770477749096808437649086070477549C0B253
:2017A00008607047F0B500250026002100270022002300245FF0000CDFF89CE1DEF800E004
:2017C0001EF00C0E7546002D04D0042D05D0082D06D03DE0684901603CE06849016039E09E
:2017E0005D49096811F47011890C891C5A4A126812F48037002F03D1614A5143016026E08E
:201800005A4A126812F48032584B1B6813F00F035B1C002A06D1594AB2FBF3F201FB02F11B
:20182000016014E0514A1268C2F30312541C4F4A1268C2F3032212F1020C504AB2FBF4F2D9
:201840000CFB02F2B2FBF3F201FB02F1016001E0494901604049096811F0F0052D090FF2B0
:2018600034116E5C0168F14041603B49096811F4E0652D0A0FF21C116E5C4168F1408160F5
:201880003549096811F46055ED0A0FF208116E5C4168F140C1603049096811F44045AD0B9D
:2018A0000FF200116E5CC168B1FBF6F10161F0BDC9B2002905D033490968084331490860EE
:2018C00005E03049096831EA00002E4908607047C9B2002905D02C49096808432A49086003
:2018E00005E02949096831EA0000274908607047C9B2002905D025490968084323490860FF
:2019000005E02249096831EA000020490860704710B4002200230021C0B24409E4B22200C2
:20192000012A02D10B490B6806E0022A02D110490B6801E016490B68C0B210F01F020120CA
:201940009040034201D0012100E000210800C0B210BC704700100240041002400000FFF8E2
:20196000FFFFF6FE08100240600042422C100240201002403C04424200127A00001BB70025
:2019800000093D0014100240181002401C1002402410024000000000010203040102030439
:2019A0000607080902040608F0B400220026002400250023002791F803C01CF00F0C62465B
:2019C00091F803C05FEACC6C01D58B781A430B781B0621D00368002406E0CD78482D02D16D
:2019E0000125A5400561641C082C14D20125A5400E882E40AE42F6D1A5000F2616FA05F730
:201A0000BB4312FA05F52B43CD78282DE5D10125A5404561E7E703600B884FF48074A34273
:201A200026D34368002420E0012514F10806B5400E882E40AE4217D1A5000F2616FA05F7EE
:201A4000BB4312FA05F52B43CD78282D04D1012514F10806B5404561CD78482D04D101251C
:201A600014F10806B5400561641C082CDCD34360F0BC70470022806880B2084201D0012215
:201A800000E000221000C0B2704789B20161704789B24161704770B4002200240023002571
:201AA0002D4E36683300C0F30346350086B2320010F44016B6F5401F08D133F07063264C9A
:201AC000246834F07064244D2C600FE0C40205D50324AC40A34353F0706307E0440DE4B219
:201AE000240112FA04F4A34353F07063C9B2002905D0400DC0B2000112FA00F003431648E8
:201B0000036070BC704710B400220F2311F00304E4B2A400A3401A00C9B28B100F4C54F86B
:201B2000233033EA0202C9B28B100C4C44F82320C9B28A10094B53F82220C0B211F00303D5
:201B4000DBB29B0098401043C9B28910034A42F8210010BC70470000040001400800014065
:201B600010B4002203881A0012F441520B884C8823438C882343CC8823430C8923434C8970
:201B800023438C892343CC8923431A430280828B4FF2FF731A408283098A018210BC704712
:201BA000C9B2002904D0018851F04001018004E001884FF6BF7211400180704781817047FC
:201BC0008089704700220089084201D0012200E000221000C0B270472DE9F04FA1B017461E
:201BE0001C4601AD6860A9600020E86211AE4FF00A096FF0004802E0E86A401CE862387858
:201C000018B9E86A21B0BDE8F08F252807D100206861A861E86128626862A8620CE017F8F3
:201C2000011BA8686A689047A8600028E4D14FF0FF30E7E740F0010017F8011F2029F9D03C
:201C400023290DD02B2904D02D2906D030290AD00CE040F0020080B2EEE740F00400FAE79A
:201C600040F00800F7E740F01000F4E72A290DD12268111D216011686963002904D54942F7
:201C8000696340F0040080B27F1C10E00021696307E0696B414503D009FB0121303969632B
:201CA0007F1C3A78A2F13001C9B20A29F1D339782E291CBF4FF0FF3129631BD117F8011FA8
:201CC0002A2906D12268111D2160116829637F1C10E00021296307E0296B414503D009FB8C
:201CE0000121303929637F1C3A78A2F13001C9B20A29F1D3288739780FF6D83002F060FB90
:201D000008B117F8010B8DF83E009DF83E00682804D1387868280AD1622005E06C2806D107
:201D200038786C2803D171208DF83E007F1C11A828613A781046253825D01C3877D0001F46
:201D4000022874D9133800F09E8009386FD0801E00F03681401E00F0DF80401E022866D97A
:201D6000001F00F0D980401F36D0401E00F08B80401E23D0C01E0CD0801E00F08480C01EC2
:201D800000F0818024E16869411C69612521815528E12168081D20600868E8602A6B002A8B
:201DA00008D4002102F0DAFA00281ABFE968401A286B01E0FAF7AEFFA86113E12168081DF7
:201DC000206008680021CDE9000111A8E860782100A800F097F905E19DF83E0062281FD047
:201DE00068280DD06A2812D06C2802D071280ED074282168081D20600868E96A0160F1E066
:201E0000E86A2268111D216011680880EAE0E86AC11723681A1D22601A68C2E90001E1E00F
:201E2000E86A2268111D216011680870DAE02068C01D20F007002060034603F108002060AB
:201E4000D3E90001CDE90001002904D56869411C69612D210DE0288F810704D56869411C93
:201E600069612B2105E0C00704D56869411C696120218155686911A94018E860114600A88E
:201E800000F0CFF9AEE09DF83E006C280FD0712801D06A280BD12068C01D20F007002060E2
:201EA000034603F108002060D3E9000104E02168081D206008680021CDE900019DF83E0073
:201EC00068280CD0622806D0742801D07A280CD1DDE9000106E0DDE90001C0B202E0DDE9BC
:201EE000000180B20021CDE9000195F83800000760D5DDE9000109B900285BD042F02000A8
:201F0000782857D16869411C6961302181556869411C696182554DE09DF83E0062280CD0A5
:201F2000682810D06A281AD06C2824D0712816D0742820D07A280CD01DE02168081D206079
:201F400091F900001BE02168081D2060B1F9000015E02168081D20600868002110E02068F8
:201F6000C01D20F007002060034603F108002060D3E9000104E02168081D20600868C11711
:201F8000CDE90001DDE9000100290EDB288F810704D56869411C69612B210AE0C00709D5C6
:201FA0006869411C6961202103E06869411C69612D218155686911A94018E860114607E779
:201FC0006869411C69612268111D21601168DEE66869411C6961252181551AB16869411C86
:201FE000696182557F1C686B6969401A296A401AA969401A696A401AE969401AA96AA0EBD6
:20200000010A95F83800400711D420208DF84000BAF1010F0BDBD346012210A900A800F091
:202020003FFC00287FF403AEBBF1010BF4D16A6911A900A800F034FC00287FF4F8AD3020B7
:202040008DF84000D5F820B0BBF1010F0ADB012210A900A800F024FC00287FF4E8ADBBF10D
:20206000010BF4D1AA69E96800A800F019FC00287FF4DDAD30208DF84000D5F824B0BBF1F7
:20208000010F0ADB012210A900A800F009FC00287FF4CDADBBF1010BF4D1EA69A869E9688B
:2020A000411800A800F0FCFB00287FF4C0AD30208DF84000D5F828B0BBF1010F0ADB0122B2
:2020C00010A900A800F0ECFB00287FF4B0ADBBF1010BF4D195F8380040077FF590AD202056
:2020E0008DF84000BAF1010FFFF689AD012210A900A800F0D5FB00287FF499ADBAF1010A5A
:20210000F4D17CE52DE9FA4786B00546686900909DF818006F2808BF082705D040F0200001
:20212000782814BF0A2710273C24D5E90001064689469DF81820642A01D0692A04D10029CD
:2021400002DA764269EB4909B9F1000F0DD166B9686B50B9082F3FD195F83C0000073BD58C
:20216000641E00983021215436E0A4F101084446F817CDE9047030464946DDE9042302F024
:2021800035F9CDE90201B246DDE90223DDE90401A0FB02695046801B3030C0B23A2803D369
:2021A0009DF8181051390818009908F80100DDE90269B9F1000F00D126B1286900996118E9
:2021C0008842D2D3082F07D195F83C00000703D50098205C3028C3D1C4F13C00E861009906
:2021E00061182961696B884207DA081A6862A88F4FF6EF710840A88710E000290ED595F895
:202200003C1001F01401102908D1A96BAA69891A6A6A891A0C1A012CA8BF6C6208B0BDE834
:20222000F0872DE9F24F8EB0054604AFD5E90001CDE902019DF8380040F020008DF800007A
:2022400061280BD0686B002848BF062005D405D19DF80000672801D1012068636968C1F3DC
:202260000A5040F2FF72904225D0012819DA284602F04AF9012814DB002400209DF80010DA
:20228000612940D12A69511C29613021117029694A1C2A619DF83820612A0CBF782258226D
:2022A0002DE040F2FE316A6861F31E526A60441A4FF0FF30E2E7080301D1286870B103200A
:2022C000E8619DF838006138C0B21A2811D30FF2106103222869FAF7DBFC9EE10320E861DC
:2022E0009DF838006138C0B21A2805D30FF2F851EFE70FF2E851ECE70FF2E851E9E70A703B
:20230000A969891CA96110B90026B0467BE19DF80000612840F09780686B00284CBF212609
:20232000461C36B2771CD5E900ABDDE902010022002302F00BF93ABF8BF00040CDE902A047
:20234000CDE902ABA4F104088DF810200DF11109012F33DBDDE902010022002302F00EF967
:202360002CD21C2102A802F021F9DDE9020102F0A9F90446FF1F012F09DB02F0CFF9024691
:202380000B46DDE9020102F0E1F9CDE9020109F207000721012C0BDB491E5EBF04F00F02D8
:2023A00000F8012D2411F5D502E0002200F8012D491EFAD500F20709012FCBDA0DF11100B2
:2023C000A9EB00010DF11107B142B8BF0E4636B2002E31D43046884206DA04A94118497892
:2023E000082928BF0F2100D2002104AA821800E0761E401E12F801398B42F9D00F2904D1A1
:2024000004A941184A78521C4A70002803D504AF761C08F1040836B2701E0DD4C1190A78CF
:202420003032D2B23A2A03D39DF838303A3B9A1801F80129401EF2D5686B002840F1E38081
:20244000701E6863DFE0DDE902010022002302F07DF805D2DDE9020181F00041CDE90201E4
:2024600024B247F2975060436D4990FBF1F80FFA88F8C8F107040027DFF8A891012C19DBF4
:20248000DDE902ABE00707D5504659463A464B46FDF7FEF882468B466410384649463A463C
:2024A0004B46FDF7F5F807468946002CEAD1CDE902AB21E064429246DFF86CB114D0E00706
:2024C00007D5504659463A464B46FDF7E1F882468B466410384649463A464B46FDF7D8F81E
:2024E00007468946002CEAD1DDE9020152465B4602F0ECF9CDE902019DF8000066280CBF59
:2025000008F10A000620696B4618142EA8BF132630208DF810000DF11104444F012E2FDBBA
:20252000DDE9020102F0E4F804F1080104220A23B0FBF3F403FB1400303001F8010DB4FBF9
:20254000F3F003FB1043303301F8013D521EEED101F10804083E012EE0DBDDE9020102F095
:20256000C7F802F0E5F802460B46DDE9020102F0EDF800223B46FDF78BF8CDE90201CFE70B
:202580000DF11100201A0DF111079DF81110302906D1401EA8F1010817F8011F3029F8D0A6
:2025A0009DF80010662904BF0FFA88F808F1010103D065290CBF012100216A6B8E1836B2CE
:2025C000B042B8BF064636B2002E1CD43146814204DAC85D352828BF392000D23020CA1961
:2025E000521E00E0761E491E12F801398342F9D0392802D1C85D401CC855002903D57F1E4E
:20260000761C08F101080FFA88F0009033B23A469DF83810284600F00BF80FB0BDE8F08F8F
:20262000A0860100000024400000F03F84D797412DE9F04385B00546894617461E46BDF99E
:202640003040D5F83480012E02DA01260FF29C2749F0200066280AD0672840F086806FF0AE
:2026600003018C42C0F28780444580F28480641C66280CD095F83C00000702D44645B8BF3E
:20268000B04624B2B8EB040848BF4FF000082869E96924B2012C25DA4A1C30230B54B8F1CB
:2026A000010F03DA95F83C10090702D52E211154521CEA6118EB040FB8BFC8F1000424B2E0
:2026C0006142A962A044B045B8BF464636B22E6232463946EB691818FAF7DAFAA8EB06001F
:2026E000E862C6E00818A64218DA32463946FAF7CFFAE9697118E961A01BA862B8F1010F9C
:2027000003DA95F83C00000705D528692E220A54286A401C2862C5F82C80AAE022463946A1
:20272000FAF7B6FAE8692018E861361BB8F1010F03DA95F83C10090704D5411CE961296944
:202740002E22425436B2B045B8BF464636B23246E119E8692B69C018FAF79AFAE86930187E
:20276000E861A8EB0600A86283E0B9F1610F16D14FF0700918E0464504DA95F83C10090707
:2027800058BFB046B8F1010848BF4FF00008B9F1670F14BF4FF045094FF0650904E0B9F171
:2027A000410F08BF4FF05009E9694A1C286917F8013B0B54B8F1010F03DA95F83C100907F8
:2027C00002D52E211154521CEA61B8F1010F11DB761E36B2B045B8BF464636B232463946BD
:2027E000EB691818FAF754FAE8693018E861A8EB0600A862E8692969471807F8019B002C88
:202800005CBF2B2007F8010B03D52D2007F8010B644200260DF1080824B2012C0EDB0A2225
:20282000214600A802F075F9019808F8010B009C761C24B2012CF2DA022E06DA49F020001E
:20284000652804BF302007F8010B1EB9302007F8010B09E0012E07DB761E02A8305C303077
:2028600007F8010B012EF7DAE86929694018381A286295F83C0000F0140010280DD1A86942
:20288000E9690818A96A0818296A0818E96A0818A96B8842BCBF081A686205B0BDE8F0835B
:2028A00070B504460D4616460020002E10D015F8011BE068A2689047E060002802D14FF000
:2028C000FF3070BD206B401C20630020761EEED170BD0000686A6C747A4C00006E616E00DD
:2028E0004E414E00696E6600494E46003000000062F30F2262F31F4200B5130096469446F7
:20290000103928BFA0E80C50FAD85FEA417C28BF0CC048BF40F8042BC90728BF20F8022BAE
:2029200048BF00F8012B00BD72B6704762B67047EFF3108072B6704780F310887047B0FA44
:2029400080F0704790FAA0F0704730BF704720BF7047000080B502F0FDF8FEF747FE5FF49A
:202960008030FEF772FEFEF79AFEC0B20128FAD1C0B2012825D10020FEF7D2FE0020FEF7C4
:20298000E7FE4FF48060FEF7D7FE022002F03CFA102002F049FA5FF480115FF48030FEF7DA
:2029A0009BFE0120FEF7A5FE3920FEF7B1FF0028FAD00220FEF7A2FEFEF7ACFE0828FBD183
:2029C00001BDFEE700B585B000A8FEF7EBFE019805B000BD80B50B48006850F08070094967
:2029E00008600948002101600848006850F0010006490860FFF7E6FF02F02FFB01BD0248ED
:202A000000687047FCED00E0041000E0001000E010B4020010324B1E002109E002600024E9
:202A20004460002404810024C46010301032491C89B29BB29942F1D30021016000214160AF
:202A4000002101810021C16010BC704710B504006A480068002803D145F21E7020801AE0D0
:202A600067480088002803D145F21D70208012E06348018861480068FFF7CAFF5E485F497B
:202A8000096801605C485E49098881805A480021C1800020208010BD41894289012A1AD349
:202AA0000268554B1B6813604268534B1A60524AD2884389D21A504BDA804F4A9288438932
:202AC0009A184D4B9A8000224281002282810022026000224260080080B2704701810021AC
:202AE0004181002181810021016000214160704770B44489002C0AD100200880002A01D05B
:202B00000020106046F292501880002026E045686C682E890E80002A01D0E9681160296839
:202B200041604168002904D1002101600021418102E04189491E41812F48006828602E4836
:202B400005602D488088401C2B4988802A48C088401E2949C88000201880200070BC70472E
:202B6000F0B4049D059C46890789BE4203D346F2935020803DE0204EB688002E03D145F27D
:202B80001D70208035E01C4E36681B4FD6F800C0C7F800C0184FBF887F1EDFF85CC0ACF892
:202BA0000470154FFF887F1CDFF84CC0ACF806704789002F04D106604660012343810DE069
:202BC000DB0605D403681E6000233360066002E043683360466043895B1C4381838947898D
:202BE000BB4201D24389838171603281F56000202080F0BC70470000007D0020003601085D
:202C0000F835010800B583B000AB01AA00210020FBF7EFFABDF800100029F5D1DFF89803FE
:202C200000780128F0D100F0FEF8EDE710B58AB00400DFF8880300210160DFF88403002112
:202C4000016000F02DF8DFF87C030078132803D346F27320208021E008940320079000203D
:202C600006900020059000200490DFF85C0300680390DFF8580300680290DFF85403006862
:202C80000190DFF84003007800900023DFF844230FF25431DFF84003FBF76EF90AB010BDA0
:202CA00000200BE080B2DFF8341311EBC00100220A6000228A800022CA80401CC8490988DA
:202CC00080B28842EED3704730B492B2042A29D1BA4A12688A1A521EC24CA24209D30021AF
:202CE000C164002101650021C16147F27E20188076E0C164511C0165C16CB94A1288B1FBB2
:202D0000F2F402FB141189B2B44A12EBC1018A88002A32D10022426100228261086001221F
:202D20008A8054E000291ED092B2082A15D1826C8C18A24A1268A21A521E8A4201D2C464F7
:202D400003E09E4A12688918C164C16C9B4A1268891A0165C16C8164CEE7984A12688A180E
:202D6000C2640165C8E70021C164002101650021C16147F27E20188032E00A6805E0946933
:202D800084614261606190610022002A1CD0D46C8A4D2D68641B1465146D056DAC420AD260
:202DA0005469002C01D05269EFE700244461826150610022E9E79469002CE0D10024846196
:202DC000426190610860DFE78A88521C8A80CA888C88A24201D28A88CA80C1610020188054
:202DE00030BC7047C16900291CD0002202650A68824206D142690A60002A08D0002393612D
:202E000005E0826943695361002B00D09A6100224261002282610022C2610022C264888825
:202E2000401E888070472DE9F0410024FFF780FD0400FFF7E4FD050060480068401C5F49A3
:202E400008605E48006866490988B0FBF1F201FB120080B2614911EBC000D0F8008000261A
:202E600000E0B846F6B2002E40F09780B8F1000F00F09180D8F8147098F8360000280BD081
:202E8000022809D009D3042806D01CD3062803D042D3072856D0E4E7E3E7D8F84C004749B6
:202EA0000968401AC8F8500044480068D8F84C10884206D1002088F836004046FBF745F8EB
:202EC00000E00126CDE7D8F84C003C490968401AC8F8500039480068D8F84C10884219D1F2
:202EE0000020C8F85C000020A8F86000FFF787FDC8F840004046FAF724FE4046FBF725F8CE
:202F0000002088F83600032088F83500002088F8340000E00126A4E7D8F84C0027490968A0
:202F2000401AC8F8500025480068D8F84C10884206D1042088F836004046FFF753FF00E0FD
:202F400001268EE7D8F84C001C490968401AC8F850001A480068D8F84C10884219D10020AF
:202F6000C8F85C000020A8F86000FFF748FDC8F840004046FAF7E5FD4046FFF733FF0420AF
:202F800088F83600032088F83500002088F8340000E0012665E7012664E7FFF730FD401B8C
:202FA00007490968814201D2054908602000FFF7C3FCBDE8F08100003D800020CC7E0020D2
:202FC000D07E00200C360108183601081436010810360108052C0108806A00201073002058
:202FE000203601080100FFFF75432F4F532D494949205469636B205461736B00704757482E
:2030000000685749096811EB8000001F55490860704770477047704710B40400019812EB5C
:203020008000001F5FF080720260001F0460001F4D4A0260001F5FF012320260001F5FF031
:2030400003320260001F5FF002320260001F0360001F0160001F5FF011310160001F5FF054
:2030600010310160001F5FF009310160001F5FF008310160001F5FF007310160001F5FF028
:2030800006310160001F5FF005310160001F5FF00431016010BC704738B5FFF7B0FC02007B
:2030A0003248006832490968884217D02F480068D0F89400101A2D490968C1F890002B4889
:2030C0000068D0E9264529480068D0F89000002120186941254B1B68C3E926012448006896
:2030E000C0F8942021480068D0F8B80021490968884205D21D4800681E490968C0F8B81072
:203100001C480021016031BD704710B50024FFF70FFC040018480078401C1749087020000A
:20312000FFF70AFCFAF735FAFAF7FEFA10BD401E12490860124800680002000A104908600D
:203140001048006850F005000E4908600D48006850F002000B49086070470000F03501080B
:20316000EC350108AC7E0020E5E40008E47E0020E87E0020C07E00203C80002014E000E0F4
:2031800020ED00E010E000E0002004E01F49002241F82020401C0028F8D0704710B500247F
:2031A0001A4801E02034001D01680029FAD00068FFF7C5FB04192000C0B210BDC0B24209A8
:2031C000C0B210F01F010120D1F11F018840D2B20E4951F822100843D2B20C4941F82200BD
:2031E0007047C0B24209C0B210F01F010120D1F11F018840D2B2054951F8221031EA000096
:20320000D2B2024941F8220070470000B07E0020024900220A80002101807047B67F0020DA
:20322000024900220A80002101807047B87F0020034900220A800021018070470000000096
:20324000BA7F002000B589B0A6490968002908D0A5490968A34A1268B1FBF2F1A34A116013
:2032600006E0A14909680A22B1FBF2F19F4A11609F499E4A12680A60994900220A609D49F0
:2032800000220A6000210AE089B29B4A12EBC102002393800023D38000231360491C974A2F
:2032A000128889B29142EFD395490968002903D147F2463101802DE092490968924A126878
:2032C000914203D247F24631018023E08F490978132903D346F2732101801BE008900320A4
:2032E0000790002006900020059000200490854800680390864800680290814800680190C6
:203300008248007800900023824A0FF210218248FAF732FE09B000BD10B4022280F82A20AF
:2033200089B2012905D1416A6D4A1268511881610DE0016A002905D1416A694A1268511893
:20334000816104E0016A664A12685118816181696A4A1288B1FBF2F302FB131189B2664AF2
:2033600012EBC1010A68002A07D100220261002242610860012088802EE08269584B1B6820
:20338000D21AC2610B6805E05A6942610361106158610023002B1CD09A69514C2468121B3F
:2033A000DA61DA69C469A2420AD21A69002A01D01B69EFE700220261436118610023E9E735
:2033C0005A69002AE0D100224261036158610860DFE78888401C8880C8888A88904201D2C4
:2033E0008888C88010BC70478169444A1288B1FBF2F302FB131189B23F4A12EBC1010A6839
:20340000824206D102690A60002A08D00023536105E0426903691361002B00D05A6101221A
:2034200080F82A2000220261002242618888401E88807047F0B583B00BE0FFF7E0FA041BA1
:2034400000A8FAF74CFA2B480068A04201D22948046000AB01AA00210020FAF7CAFE0500D3
:2034600000A8FAF70CFAFFF7CAFA04001C480068401C1B4908601A48006820490988B0FB8C
:20348000F1F201FB120080B21B4911EBC0000668002700E00127FFB2002FCED1002EF9D0D6
:2034A00035690F480068B169884216D13000FFF79BFF308D022804D101213000FFF72CFFF5
:2034C00002E0032086F82A00B2681000002802D0F168300090472E00DDE70127DBE70000DF
:2034E000D87E00202C36010808360108DC7E0020E07E0020D47E00207873002040360108B0
:20350000303601083836010804360108283601083436010835340108406B002075432F4F35
:20352000532D4949492054696D6572205461736B000000000FF210100FF2A00108000FF290
:20354000A00108000FF29C0108000FF29C0108000FF2980108000FF2980108000FF294019C
:2035600008000FF2940108000FF2900108000FF2900108000FF28C0108000FF28C01080045
:203580000FF2880108000FF2880108000FF2840108000FF2840108000FF2800108000FF260
:2035A000800108000FF27C0108000FF27C0108000FF2780108000FF2780108000FF27401FC
:2035C00008000FF2740108000FF2700108000FF2700108000FF26C010800704714550020BB
:2035E0000C0000007D000000F4010000085700207D000000F40100006400000040060000B2
:20360000F039002040000000E803000010000000FC5800200C0000007D000000F401000034
:203620000D00000068000000120000000A000000F05A00200C0000007D000000F401000011
:203640000D00000068000000E00E00001748FF210170002080F309881548016881F3088829
:2036600014481549016062B6FEE772B6EFF3098028B1203880E8F00F10490968086000B520
:203680000F4880475DF804EB0E480F490A7802700A480E490A680260106890E8F00F20306A
:2036A00080F309884EF0040E62B6704722ED00E0AC7E002004ED00E000000010E47E00204B
:2036C000993001083E8000203F800020E87E002038B5040001212020FEF7FAF8E4B2012CD8
:2036E00040D200230122E4B20520C14900FB04108178E4B20520BE4D00FB04504078FCF7E5
:2037000091FA00230122E4B20520B94900FB04100179E4B20520B64D00FB0450C078FCF75A
:2037200081FA0022E4B20520B14900FB04108178E4B20520AE4B00FB04304078FCF7F3FAB4
:203740000022E4B20520AA4900FB04100179E4B20520A74B00FB0430C078FCF7E4FA4FF6E6
:20376000FF7000E0002032BD10B584B00400E4B2012C80F082800122E4B205209C4900FBFB
:2037800004100179E4B20520994B00FB0430C078FCF7C9FA02A8019000200090642300224B
:2037A00000210020F9F737FE0122E4B20520904900FB04108178E4B205208D4B00FB043022
:2037C0004078FCF7B0FA02A80190002000904FF41673002200210020F9F71DFE0022E4B2B7
:2037E0000520834900FB04108178E4B20520804B00FB04304078FCF796FA02A80190002085
:2038000000906423002200210020F9F704FE0122E4B20520764900FB04108178E4B20520DC
:20382000734B00FB04304078FCF77DFA02A80190002000904FF4FA73002200210020F9F78B
:20384000EAFD0022E4B20520694900FB04108178E4B20520664B00FB04304078FCF763FA47
:2038600002A80190002000906423002200210020F9F7D1FD4FF6FF7000E0002004B010BD80
:2038800010B584B00400E4B2012C80F082800022E4B20520564900FB04100179E4B2052036
:2038A000534B00FB0430C078FCF73DFA02A80190002000906423002200210020F9F7ABFD6C
:2038C0000122E4B205204A4900FB04108178E4B20520474B00FB04304078FCF724FA02A880
:2038E0000190002000904FF41673002200210020F9F791FD0022E4B205203D4900FB041068
:203900008178E4B205203A4B00FB04304078FCF70AFA02A8019000200090642300220021DB
:203920000020F9F778FD0122E4B20520304900FB04108178E4B205202D4B00FB0430407889
:20394000FCF7F1F902A80190002000904FF4FA73002200210020F9F75EFD0022E4B2052064
:20396000234900FB04108178E4B20520204B00FB04304078FCF7D7F902A801900020009018
:203980006423002200210020F9F745FD4FF6FF7000E0002004B010BD10B50400E4B2012C4A
:2039A00025D2C9B2012911D112480078002804D02000C0B2FFF7D8FE19E0F4F7C5FD21286E
:2039C00015D12000C0B2FFF7CFFE10E009480078002804D02000C0B2FFF752FF07E0F4F74C
:2039E000B3FD212803D12000C0B2FFF749FF10BD080900202780002080B52E484FF6FF7105
:203A0000018001F03DFB4FF6FF7001F091FC02F0F7F801BD80B501F048FB01BD80B5254862
:203A200000884FF6FF71884214D0234800680090FFF7F0FF22481F49098801801D48008882
:203A4000002803D11C48006801F021FB19484FF6FF71018001BD38B504000D004FF41B726E
:203A600020211848F6F7FEFDF4F753FF114800884FF6FF71884201D0002011E0A4B2002CBC
:203A80000DD1A02200210D48F6F7ECFD0B48286009490860074804804FF6FF7000E000201E
:203AA00032BD80B506480088002801D101F004FB01BD00003E7F0020147E002050700020F5
:203AC000407F0020704E002070B58EB004001600E4B2102C01D3002026E23000DFF868145B
:203AE000FBF79CFD05D930005FF08041F9F798F801D2002018E2E4B20C20DFF8501400FBB8
:203B000004104068DFF84814884205D101214FF40060FDF7DDFE2DE0E4B20C20DFF82C149C
:203B200000FB04104068B0F1804F04D101210120FDF7DEFE1EE0E4B20C20DFF8101400FBC0
:203B400004104068DFF80C14884204D101210220FDF7CEFE0EE0E4B20C20DFF8F01300FB8A
:203B600004104068DFF8F013884203D101210420FDF7BEFE01210C20FDF7AAFEE4B2002C6F
:203B80001FD0022C3DD02CD3042C58D048D3062C71D062D3082C00F08A807AD30A2C00F040
:203BA000A280C0F092800C2C00F0B980C0F0A9800E2C00F0D280C0F0C1800F2C00F0DC80F3
:203BC000E9E04FF48070ADF8000018208DF8030003208DF8020000A9DFF88003FDF7E4FE01
:203BE000D9E04FF40070ADF8000018208DF8030003208DF8020000A9DFF86003FDF7D4FEA1
:203C0000C9E04FF48060ADF8000018208DF8030003208DF8020000A9D048FDF7C5FEBAE0B7
:203C20004FF40060ADF8000018208DF8030003208DF8020000A9C948FDF7B6FEABE00120C4
:203C4000ADF8000018208DF8030003208DF8020000A9C248FDF7A8FE9DE00220ADF80000C4
:203C600018208DF8030003208DF8020000A9BB48FDF79AFE8FE00420ADF8000018208DF8AD
:203C8000030003208DF8020000A9B448FDF78CFE81E00820ADF8000018208DF80300032043
:203CA0008DF8020000A9AD48FDF77EFE73E04020ADF8000018208DF8030003208DF80200AD
:203CC00000A9A648FDF770FE65E08020ADF8000018208DF8030003208DF8020000A99F4867
:203CE000FDF762FE57E00120ADF8000018208DF8030003208DF8020000A99948FDF754FE39
:203D000049E00220ADF8000018208DF8030003208DF8020000A99248FDF746FE3BE04FF430
:203D20008050ADF8000018208DF8030003208DF8020000A98B48FDF737FE2CE04FF4005060
:203D4000ADF8000018208DF8030003208DF8020000A98448FDF728FE1DE04FF48040ADF820
:203D6000000018208DF8030003208DF8020000A97C48FDF719FE0EE04FF40040ADF800004B
:203D800018208DF8030003208DF8020000A97548FDF70AFEFFE74FF4187530007249F8F7C7
:203DA0003FFF06D271483100F6F7DEFBFDF7FAFA050008A8FDF7F6FC4FF47A70ADF81800D0
:203DC0004720ADF814000020ADF81A000020ADF8160005A9E4B20C205C4A00FB042040682C
:203DE00002F036F8E4B20C20584900FB0410007A01281DD16020ADF804000120ADF80600AB
:203E0000ADF80A500220ADF80C0001A9E4B20C204E4A00FB0420406802F035F80821E4B227
:203E20000C204A4A00FB0420406802F03FF970E0E4B20C20454900FB0410007A02281DD190
:203E40006020ADF804000120ADF80600ADF80A500220ADF80C0001A9E4B20C203B4A00FBAF
:203E60000420406802F04BF80821E4B20C20374A00FB0420406802F022F94AE0E4B20C2015
:203E8000324900FB0410007A03281DD16020ADF804000120ADF80600ADF80A500220ADF84A
:203EA0000C0001A9E4B20C20284A00FB0420406802F068F80821E4B20C20244A00FB042087
:203EC000406802F006F924E0E4B20C201F4900FB0410007A04281CD16020ADF8040001202F
:203EE000ADF80600ADF80A500220ADF80C0001A9E4B20C20154A00FB0420406802F084F845
:203F00000821E4B20C20114A00FB0420406802F0E9F80121E4B20C200C4A00FB04204068C0
:203F200002F0B6F84FF6FF700EB070BD80B50121C0B20C22054B02FB0030406802F09AF8A2
:203F40004FF6FF7002BD00000100C64208060020002C014000040040000800400008014075
:203F6000000C0140001401400000C842000020410149C0B20860704720000E4222480088F7
:203F800050F010002049088070471F4800884FF6EF7108401C490880704700201B49098894
:203FA00008001B49098889B280B250EA0140704710B50400FFF7E2FF200C15490880134858
:203FC0000480FFF7E2FF10BD10B50400FFF7D6FF200C10F00F000F4908800F480480FFF739
:203FE000D4FF10BD084800888006FBD57047064800884FF6F77108400349088002480088CB
:204000000007FBD570470000042800401C28004018280040082800400C28004080B5012068
:2040200002F06AB800BF000006490868002801D000207047044808600449C908C900091A60
:2040400001607047F07E002048A1002048C2002010B5224C206890B1201D02F058F804F117
:20406000080002F054F804F10C0002F050F804F1100002F04CF804F1140002F048F810BD7C
:2040800038B50446154D286890B9281D02F03EF805F1080002F03AF805F10C0002F036F8FD
:2040A00005F1100002F032F805F1140002F02EF801202860052C04D205EB8400001D02F089
:2040C00027F831BD052800D3704780B5034901EB8000001D02F01DF801BD0000F8760020BF
:2040E0000022FBF79BBF03E00B680370401C491C13005A1E002BF7D17047F8B505000C00D5
:20410000170004208DF8000000F09EFEBE080420B7FBF0F101FB1071002909D0761C07E0DE
:204120002968200000F0A4FE8DF80000241D2D1D3000461E80B2002803D09DF800000428AA
:20414000EED000F08CFEF1BD10B5002400E0641C032C36D214200FF2E40100FB0410C068A8
:2041600014210FF2D80201FB0421096814220FF2CC0302FB043292685118491E884201D0FF
:20418000002020E0601C03280FD214200FF2AC0100FB0410C06814210FF2A00201FB042165
:2041A0004969884201D300200DE014200FF28C0100FB0410007900F05FF80028C7D1002031
:2041C00001E04FF6FF7010BD30B4002300E05B1C032B2FD214240FF2640504FB035424686C
:2041E000A042F4D314240FF2540504FB0354E4688442ECD314240FF2440504FB0354248AD7
:20420000002C01D1002016E0002906D014240FF22C0504FB035424790C60002A07D014218C
:204220000FF2180401FB03410968401A10604FF6FF7000E0002030BC70470000000000008F
:204240000200000000000100FFFF0000FFFF0000000001000300000000000100FFFF01005B
:20426000FFFF0000000000100100000000000800FFFF07100000000038B5040000200025DC
:2042800010E0EDB22421344A01FB05210978E4B28C4206D1EDB224202F4900FB05104069DA
:2042A00080476D1CEDB2032DEBD380B232BD2DE9F04104000D0016001F0000205FF00008FC
:2042C00017E05FFA88F82421234A01FB08210978E4B28C420BD13A00310028005FFA88F80A
:2042E0002423DFF874C003FB08C3DB68984718F101085FFA88F8B8F1030FE2D380B2BDE84F
:20430000F0812DE9F04104000D0016001F0000205FF0000817E05FFA88F824210E4A01FBBF
:2043200008210978E4B28C420BD13A00310028005FFA88F82423DFF820C003FB08C31B69DC
:20434000984718F101085FFA88F8B8F1030FE2D380B2BDE8F0810000381C0408C9B2830776
:2043600006D0521E22D310F8013B9942F7D11FE0083A13D302F1040241EA012141EA014141
:2043800050F8043B121F21BF4B40A3F1013C2CEA030C1CF0803FF3D0C9B2001F083210F89A
:2043A000013B521E28BF91EA030FF8D818BF0120401E7047014801F0ADBE0000F47E0020C9
:2043C0000278C9B28A421AB11CBF10F8012FF9E718BF00207047000013F0004C03D55B42EC
:2043E000524263F100039CEA210C15D11B4229D109424CD12AB18446B0FBF2F002FB10C279
:20440000704701F089BEFCD30022002370470B00020000210020704710B5644603D349420D
:20442000404261F10001FFF7E1FF640004D34942404261F10001244203D55B42524263F173
:20444000000310BD904271EB030CE0D370B5B1FA81F4B3FA83F52C1BA340C4F1200532FA02
:2044600005F63343A2405FF00046E64002E05B085FEA3202841A71EB030524BF20462946B2
:204480007641F4D302000B003000002170BD012AB9D970B5140C20D0B1FA81F4B2FA82F5DE
:2044A000C4F120046419B4F12006D6D3B2405FF00044F440002502E052085FEA3303C61AB9
:2044C00071EB020E24BF3046714664416D41F3D302000B002000290070BD0C46B1FBF2F1E3
:2044E00002FB11452D0445EA1045B5FBF2F402FB145580B240EA0545B5FBF2F002FB105221
:2045000040EA044070BD000070B4416801F0004201210D4B44681C40446001D104686CB17F
:2045200004684568E60F46EA4505456064000460491EEC02F4D544682340436043681A43AE
:204540004260084670BC7047FFFF0F004FF4001C1CEB410F94BF1CEB430F09E041EA030CF6
:2045600050EA4C0C52EA0C0C03D2994208BF9042704714BF8B428242704700004FF4001CDB
:204580001CEB410F94BF1CEB430F09E041EA030C50EA4C0C52EA0C0C03D28B4208BF8242E2
:2045A000704714BF994290427047000070B504460D466068C0F30A5040F2FF71884209D130
:2045C0006068000302D12068002801D0022070BD012070BD30B92046FFF796FF012801DB40
:2045E000002070BD012D0EDB40F2FF71091A8D4209D36068002847BF00202F4900202F49C1
:20460000C4E90001E4E74142A942616806DA2C4A1140401941EA0050606049E001F0004154
:2046200062681203120B42F480126260401E451905F13500352803D361600020206070BD4C
:20464000002215F11F0F05DA203522686068206000206060684213D0521E9241D243C0F188
:20466000200325689D4055EAD2722568C540666806FA03F32B432360636823FA00F060604B
:20468000606808436060B2F1004F03D80AD12078C00707D52068401C2060206810B96068E7
:2046A000401CB9E76068884202D12068002897D04FF0FF3070BD00BF0000F0FF0000F07FCA
:2046C000FFFF0F80F446400D40EAC120490006D200F013F8004248BF6FF00040604700F020
:2046E0000CF84FF0004188428CBF084640426047400D40EAC12049000CD240F00040490D65
:20470000A1F58061491C05D4D1F11F0154BFC840C01770474FF0000070470000010040F131
:204720000880F446404200F004F851F000416047010009D0B0FA80F18840C91CC1F58461E3
:20474000090501EBD02140057047000070B44FF0004591EA030F44BF6B4001F0E8BC841A5C
:2047600071EB030604D26E40001BB141121973414FF4001C1CEB410F34BF7CEB430684E0A7
:204780000C0DA4EB1356362E7DDC012E43DC45EAC32343EA525312BFD20292025B08240551
:2047A00045EAC12141EA5051D2EBC020994125D407D1B0FA80F610FA06F164D00020203609
:2047C00008E0B1FA81F6B140C6F1200220FA02F21143B0404FEAF474B4EB465434F00106AE
:2047E0004FEA74040AD8D6F50016760D04F00044F04061FA06F25040F1404840C00A40EACA
:20480000415021F0004128BF5FEA500550F1000044EBD12137E045EAC323DB0A45EAC121AC
:20482000C90AB6F120050EDD42EA0242120CC5F1200603FA06F6EB4042EA06056D429841A1
:2048400061F100010DE062FA06F5F240554063FA06FC82EA0C02F3405A406D42904161EB88
:20486000030111F4801F05D1641E620502D06D004041494121F48011430875F1004350F1AC
:20488000000041EB045170BC70471CEB410F15D223F0004352EA43060BD04FEA4C0CBCEB88
:2048A000410F04D80C0D661E342EB7DDEBE7801A994150EA410608BF0021E4E708BF1CEBF1
:2048C000430F28BF6FF00001DDE70000F0B540F2FF7581EA030C0CF0004C15EA11541DBF2E
